:020000040800F2
:10000000187E012061020008D34C0008C34100089B
:10001000D14C0008970A00082D5800080000000085
:10002000000000000000000000000000A101000826
:10003000A50A000800000000FD0100083D5100086D
:100040007B0200087B0200087B0200087B0200089C
:100050007B0200087B0200087B020008A70A000858
:100060007B0200087B0200087B0200087B0200087C
:100070007B0200087B0200087B0200087B0200086C
:100080007B0200087B0200087B0200087B0200085C
:100090007B0200087B0200087B0200087B0200084C
:1000A0007B0200080D5200087B0200087B0200085A
:1000B0007B020008195200087B0200087B0200083E
:1000C0007B0200087B0200087B0200087B0200081C
:1000D0007B020008D9570008F157000809580008AA
:1000E0007B0200087B0200087B0200087B020008FC
:1000F0007B0200087B0200087B0200087B020008EC
:100100007B0200087B0200087B0200087B020008DB
:100110007B0200087B0200082552000841520008BB
:10012000990A00087B0200087B0200087B02000895
:100130007B0200087B0200087B0200087B020008AB
:100140007B0200087B0200087B0200087B0200089B
:100150007B0200087B0200087B020008155800089B
:100160007B0200087B0200087B0200087B0200087B
:100170007B0200087B0200087B02000800000000F0
:100180007B0200087B020008DFF810D000F0FCFBC7
:10019000004800470D9A0208AFF30080187E012046
:1001A0002C4B19680868B0E8F04F80F30988BFF35A
:1001B0006F8F4FF0000080F311887047000000003F
:1001C00008480068006880F308884FF0000080F35A
:1001D000148862B661B6BFF34F8FBFF36F8F00DF35
:1001E00000BF00BF08ED00E0DFF80C00016841F43B
:1001F00070010160704700BF88ED00E0EFF30980F7
:10020000BFF36F8F134B1A681EF0100F08BF20ED5D
:10021000108A20E9F04F106009B44FF0500080F3CD
:100220001188BFF34F8FBFF36F8F32F05BFC4FF03D
:10023000000080F3118809BC19680868B0E8F04F25
:100240001EF0100F08BFB0EC108A80F30988BFF3CE
:100250006F8F7047B4000020EFF3058070470000F7
:100260000648804706480047FEE7FEE7FEE7FEE750
:10027000FEE7FEE7FEE7FEE7FEE7FEE7FD510008CA
:10028000890100082DE9F05F0546002092469B4653
:1002900088460646814640241BE02846414647469C
:1002A000224600F03AFA53465A46C01A914110D3FA
:1002B00011461846224600F021FA2D1A67EB010874
:1002C0004F4622460120002100F018FA17EB0009E2
:1002D0004E41201EA4F10104DFDC484631462A4687
:1002E0004346BDE8F09F10B5431A934209D28318E4
:1002F000881803E010F8011D03F8011D521EF9D201
:1003000010BD40EA01039B0703D009E008C9121F92
:1003100008C0042AFAD203E011F8013B00F8013BBF
:10032000521EF9D210BD421C10F8011B0029FBD14E
:10033000801A704710B5002200E0521C835C8C5C70
:10034000A34201D1002BF8D1D8B2E1B2401A10BDBE
:10035000034611F8012B00F8012B002AF9D11846A9
:1003600070472DE9FE4F804681EA0300C00F0C461E
:10037000009021F0004123F00045B8EB0200A941B4
:1003800005D24046214690461C460B46024623F0C5
:100390000040104347D0270DC7F30A00C3F30A51AA
:1003A0000290401A019040286BDAC3F3130040F426
:1003B000801B0098924620B10023D2EB030A63EB26
:1003C0000B0B01985946C0F14002504600F096F9D7
:1003D00006460D4650465946019A00F0AEF910EB1C
:1003E00008006141002487EA115284EAE7731A4346
:1003F00040D0009A62B3019A012A4FEA075215DCF5
:10040000001B61EB02014FF0004202EA0752CDE906
:100410000042001C41F5801132462B4600F0E5F900
:1004200003B0BDE8F08F40462146F9E7001B61EBC1
:100430000201001C41F5801300185B412018A2F551
:10044000001747EB030140EAD570B6196D4111E082
:100450006D084FEA360645EAC0754FEA0752001BA1
:1004600061EB0201001C41F5801149084FEA3000A0
:100470000019514132462B4603B0BDE8F04F00F061
:10048000A5B90098012240000023D0EB020263EBE3
:10049000E073009821464FEAE074B8EB000061EB8E
:1004A0000401E9E783F000435BE781F0004158E78E
:1004B0002DE9FE4F81EA030404F0004421F00041DD
:1004C00000944FF0000B23F0004350EA01045ED08B
:1004D00052EA03045BD0C3F30A54C1F30A552C4417
:1004E000A4F2F3340194A0FB0254C1F3130141F4CC
:1004F0008011C3F3130343F4801301FB024400FB98
:10050000034E840A970A44EA815447EA8357A4FBBE
:10051000076802958D0A05FB07854FEA932C04FBBB
:100520000C542705029D4FEA065847EA1637B5EBEB
:1005300008056EEB070C870E920E47EA811742EA18
:100540008312A7FB0201B6EB0B0164EB00042B0D39
:1005500043EA0C335E1844EB1C50DA465146E7FB85
:100560000201C5F313044FEA0B3343EA14534FEA75
:100570000432019C43EA0603A4F10C040294009C9B
:10058000CDE900B400F031F903B0BDE8F08F0020F0
:100590000146F9E72DE9F04D81EA030404F0004B30
:1005A00021F0004514464FF0000A23F0004150EAC4
:1005B000050220D054EA01021DD0C5F30A570246B5
:1005C000C5F31303C1F31300C1F30A5640F48015B9
:1005D00043F48013A7EB0608101BD64608F2FD383B
:1005E00073EB050002D308F1010801E092185B41AA
:1005F000B8F1000F03DA00200146BDE8F08D0020BD
:100600004FF48011064684460EE0171B73EB050776
:1006100005D3121B63EB050306434CEA010C4908A2
:100620004FEA300092185B4150EA0107EDD152EADF
:10063000030012D082EA040083EA0501084305D0D2
:10064000101BAB4106D20122002306E000224FF02E
:10065000004302E06FF0010253101AEB06004CEB6E
:10066000085110EB0A0041EB0B01BDE8F04D00F022
:10067000ADB800F0004230F000400AD0C10D01F5E5
:100680006071C0F3160042EA0151C20840071143ED
:10069000704700200146704701F0004330B421F05C
:1006A000004150EA010206D00A0DA2F56072C1F3C2
:1006B0001301002A02DC30BC00207047440F44EADA
:1006C000C104C100E01830BC00EBC25000F047B8D4
:1006D00030B50B46014600202022012409E021FA12
:1006E00002F59D4205D303FA02F5491B04FA02F50F
:1006F0002844151EA2F10102F1DC30BD202A04DBE2
:10070000203A00FA02F1002070479140C2F1200324
:1007100020FA03F3194390407047202A04DB203A63
:1007200021FA02F00021704721FA02F3D040C2F111
:1007300020029140084319467047202A06DBCB1758
:10074000203A41FA02F043EAE07306E041FA02F38C
:10075000D040C2F120029140084319467047002959
:10076000A8BF7047401C490008BF20F00100704737
:1007700010B4B0FA80FC00FA0CF050EA010404BF97
:1007800010BC704749B1CCF1200421FA04F411FAED
:100790000CF118BF012121430843A3EB0C01CB1D31
:1007A0004FEA00614FEA102042BF002010BC7047A2
:1007B00000EBC35010440029A4BF10BC7047401C7C
:1007C000490008BF20F0010010BC704710B5141E8E
:1007D00073F1000408DA401C41F1000192185B41FA
:1007E0001A4301D120F0010010BD2DE9F04D9246D1
:1007F0009B4611B1B1FA81F202E0B0FA80F22032E8
:100800009046FFF77BFF04460F4640EA0A0041EAA4
:100810000B0153465A46084313D0114653EA0100D0
:1008200019D0C8F140025046FFF777FF05460E4643
:10083000504659464246FFF761FF084305D0012064
:1008400004E020463946BDE8F08D0020054346EA25
:10085000E0762C4337430A986305E40AA0EB0800CE
:100860000022FD0A44EA47540A3002D5002001461E
:10087000E9E7010510196941DDE9084500196941F9
:10088000BDE8F04DA2E72DE9F04D00231A461B1AF2
:100890008A4103DB00200146BDE8F08DC1F30A5216
:1008A000C1F3130141F480154FF0000BD10702D1C1
:1008B00000186D41521E0027044640F2FF113846D1
:1008C00001EB620A3E468046024600204FF480114A
:1008D000FFF723FFC2197141BB1846EB0100B4EBCF
:1008E000030C75EB000C04D3E41A65EB0005174606
:1008F0000E46241908F101006D4180463428E3DDDD
:10090000F91946EB0600091BA84103D24FF0FF324C
:10091000134601E0002213461BEB070046EB0A5189
:10092000BDE8F04DFFF752BFC1F30A52C1F3130106
:1009300040F2FF3341F480119A4202DA002001466E
:10094000704740F233439A42A2F2334202DC5242F1
:10095000FFF7E3BEFFF7D2BE30B5041E71F100040D
:1009600004DB4FF00044404264EB0101141E73F1BC
:10097000000405DB1C464FF00043524263EB0403C6
:10098000994208BF904230BD064C074D06E0E06832
:1009900040F0010394E8070098471034AC42F6D3C6
:1009A000FFF7F6FB48E9040868E9040870B58C18FD
:1009B00010F8015B15F0070301D110F8013B2A1173
:1009C00006D110F8012B03E010F8016B01F8016B60
:1009D0005B1EF9D12B0705D40023521E0DD401F85C
:1009E000013BFAE710F8013BCB1A921C03E013F825
:1009F000015B01F8015B521EF9D5A142D8D300205A
:100A000070BD10B50246806B016C11F0500F016C87
:100A100005D011F0100F28D000F000F910BD41F4FE
:100A20000071016401688A6812F0405F04BF027EB1
:100A3000002A17D1CA6A12F4700F1CBF8A6812F418
:100A4000806F0FD14A6822F020024A60016C21F4C5
:100A500080710164016C11F4805F03D1016C41F07D
:100A60000101016400F0D8F810BD806BC16CBDE8D5
:100A700010401046084710B5806B40210164416C5E
:100A800041F00401416400F0C9F810BD10B5806B5D
:100A900000F0C3F810BDFEE7014800F0F9BB00000C
:100AA000640900207047022000F0FCBD72B6FEE72A
:100AB00038B44FF0000CCDF800C090F83C20012A6B
:100AC00002BF022038BC7047012280F83C200A682F
:100AD00007240368092A13D9DD680A3A02EB4202A7
:100AE00004FA02F225EA0202DA600A788B680A3A0E
:100AF00002EB420293400268D4682343D36010E0C3
:100B00001D6902EB420204FA02F225EA02021A61AE
:100B10000A788B6802EB420293400268146923430F
:100B200013614A681F24072A15D203685D6B521EA1
:100B300002EB820204FA02F225EA02025A630A88F0
:100B400093B20A79521E02EB820293400268546B00
:100B5000234353632BE003680D2A14D21D6BD21F6D
:100B600002EB820204FA02F225EA02021A630A8800
:100B700093B20A79D21F02EB820293400268146B8F
:100B80002343136313E0DD6A0D3A02EB820204FA99
:100B900002F225EA0202DA620A8893B20A790D3A71
:100BA00002EB820293400268D46A2343D362174B5C
:100BB0000468154A9C4204BF0C68122C03D1546887
:100BC00044F48004546004689C4218D10B68102BD4
:100BD00018BF112B13D1536843F400035360096805
:100BE00010290CD10A490B4A0968B1FBF2F101EB5B
:100BF00081014900009102D0491E0091FCD180F88A
:100C00003CC038BC00207047002301400020014058
:100C1000B000002040420F0070477047704700004E
:100C20002DE9F04104004FF0000504BF0120BDE8AC
:100C3000F081564F206C002628B9204600F0AEF80F
:100C4000666484F83C60206C10F0100F18BF01251A
:100C500004D084F83C602846BDE8F081206C20F484
:100C6000885040F0020020644948416821F4403136
:100C7000416041686268114341602068416821F425
:100C80008071416020684168226941EA0221416027
:100C90002068416821F04071416020684168A26885
:100CA000114341602068816821F4006181602068FF
:100CB0008168E26811438160A06AB8422068816857
:100CC00021F0706181602068816808BF21F0405187
:100CD0000BD0A26A114381602068816821F04051E5
:100CE000816020688168E26A1143816020688168C0
:100CF00021F00201816020688168227E41EA420180
:100D0000816094F8200000282068416808BF21F421
:100D100000610ED041F4006141602068416821F417
:100D200060414160206841681A4B626A03EB4232BD
:100D3000114341602068C16A21F47001C1622068DA
:100D4000C16AA28B144B03EB02521143C1622068AB
:100D5000816821F4007181602068816894F83020F6
:100D600041EA422181602068816821F480618160CC
:100D700020688168626941EA822181606664206C32
:100D800020F0020040F00100206462E70100000F43
:100D90000023014000E0FFFF0000F0FF70B586B0C7
:100DA000002400940194029403940494016806467C
:100DB000A1F18040B0F590301CBF06B070BD1A485C
:100DC000016841F480710160006800F48070059052
:100DD0001648016841F0010101600068694600F0B1
:100DE000010005900120009003200190104800F0C0
:100DF00065FC114D0F48C5E900040015AC60C5E95C
:100E00000340400068618000A8614011C5E9070403
:100E100028466C6200F02CFB002818BFFFF746FE46
:100E2000B563AE6306B070BD44380240303802404E
:100E300000000240106402406409002038B500231D
:100E40000446009390F83C00012804BF022038BDFE
:100E5000012084F83C002068D0F808C01CF0010F85
:100E600012D1D0F808C04CF0010CC0F808C04A48B4
:100E7000DFF828C10068B0FBFCF010EB40000090E8
:100E800002D0401E0090FCD12068D0F808C01CF4AD
:100E9000807F05D0D0F808C02CF4807CC0F808C052
:100EA0002068D0F808C01CF0010F6BD0D4F840C007
:100EB0002CF0010C2CF4C06C4CF4807CC4F840C0C5
:100EC000406810F4806F05D0206C20F4005040F48E
:100ED00080502064206C10F4805F08BF636403D0EE
:100EE000606C20F00600606484F83C30A36B2D48F1
:100EF0002B4DD863A36B2C481864A36B2B48D86484
:100F000023686FF0220018602068436843F0806314
:100F100043602068836843F48073836020681346CD
:100F200000F14C0C0A466146A06B00F04DFB68686E
:100F30001F4910F01F0F206806D0884204BF816847
:100F400011F0405F19D025E0884212D0194A904232
:100F500004BFD1F8042312F01F0F0AD0A0F1804281
:100F6000B2F5913216D1D1F8041301F01F01102906
:100F700010D2816811F0405F0CD1816841F080414E
:100F8000816007E0206C40F010002064606C40F04D
:100F900001006064002038BDB000002040420F0016
:100FA00000230140030A00088D0A0008770A0008A0
:100FB00000200140002101407047002812BF002995
:100FC000012070474379012B04BF0220704730B4E1
:100FD00001244471022303710368D3F800C002F0B6
:100FE000100240F6FE7595402CEA050CD1E900513F
:100FF0002943914041EA0C01196001680B684FF0E8
:10100000C00C0CFA02F223EA02020A600471002109
:10101000417130BC0846704770472DE9F0410446E5
:1010200000680668456B16F4005F4FF0040718BFB0
:1010300015F4005F0FD02771216941F00101216192
:101040004FF4005141632068016821F48051016030
:101050002046FFF7E1FF16F0005F14BF15F0005FB8
:10106000BDE8F0812771206940F00200206121680D
:101070004FF0005048632068016821F08051016002
:101080002046BDE8F041FFF797BF002804BF0120CC
:10109000704770B504460079002518B9657120467F
:1010A00000F008F802202071256101202071002045
:1010B00070BD000000B587B0002100910191029140
:1010C000039104910168A1F18040B0F5E8401CBF94
:1010D00007B000BD1148016841F00051016000688F
:1010E00000F0005005900E48016841F001010160D8
:1010F0000068694600F00100059010200090032070
:101100000190084800F0DAFA00220521362001F0AB
:101110004BF8362001F038F807B000BD40380240E7
:10112000303802400000024081B04FF0000CCDF892
:1011300000C0002802BF012001B070470068009085
:10114000002910440CBF08301430009003600020C8
:1011500001B07047002804BF012070474279012A7E
:1011600004BF0220704730B44FF0010C80F805C076
:101170000222027103681C6801F010020CFA02F5E9
:101180002C431C603C230029016812D00C6803FA30
:1011900002F204F47014944204BF4A6842F002025E
:1011A00000D14A6080F804C00021417130BC08467B
:1011B00070470A6833EA020204BF4A6842F001023B
:1011C000F0D1EEE72DE9F0410446866D00F09AFB80
:1011D000054694F835000027022806D08020606577
:1011E00084F834700120BDE8F0812068016821F0A6
:1011F000160101602068416921F080014161206C85
:10120000002804BFA06C002804D02068016821F0E9
:10121000080101602068016821F001010160206877
:10122000006810F0010F12D000F06CFB401B052885
:1012300008D920206065032084F8350084F83470D4
:10124000BDE8F0812068006810F0010FECD194F83F
:101250005C003F2101FA00F0B060012084F8350005
:1012600084F834700020BDE8F08190F83510022930
:1012700003D08021416501207047052180F8351099
:101280000068016821F00101016000207047000042
:101290002DE9F84304464FF00008CDF8008073486C
:1012A0004FF41651A56D0068B0FBF1F72E6894F865
:1012B0005C00082101FA00F0304211D02068026879
:1012C00012F0040F0CD0026822F00402026094F8BD
:1012D0005C0001FA00F0A860606D40F001006065FC
:1012E00094F85C004FF0010909FA00F0304209D08F
:1012F0002168496911F0800F04D0A860606D40F04A
:101300000200606594F85C1004208840304209D0E7
:101310002168096811F0020F04D0A860606D40F0E8
:101320000400606594F85C1010208840304220D0A2
:101330002168096811F0080F1BD0A86020680168B7
:1013400011F4802F09D0006810F4002F02D0A16C96
:1013500079B10CE0216C51B90BE0016811F4807F88
:1013600003D1016821F008010160216C09B1204618
:10137000884794F85C102020884030424AD0216889
:10138000096811F0100F45D0A86094F835000528C1
:101390002068016809D011F4802F2BD0006810F468
:1013A000002F24D0E16B21B332E021F0160101605F
:1013B0002068416921F080014161206C002804BF50
:1013C000A06C002804D02068016821F008010160A9
:1013D00094F85C004FF03F0101FA00F0A86084F837
:1013E000359084F83480216DD1BBBDE8F883616C01
:1013F00071B90FE0016811F4807F07D1016821F015
:101400001001016084F8359084F83480E16B09B1F3
:1014100020468847606D002808BFBDE8F883606DEE
:1014200010F0010F17D04FF0050084F83500206848
:10143000016821F001010160009800F101000090B5
:10144000B84204D82068006810F0010FF4D184F885
:10145000359084F83480E16C002908BFBDE8F8833A
:10146000204601B0BDE8F04308470000B00000206E
:1014700070B5044600F046FA0646002C04BF012071
:1014800070BD022084F83500002584F834502068AF
:10149000016821F0010101602068006810F0010F6F
:1014A0000FD000F02FFA801B052805D92020606599
:1014B000032084F8350070BD2068006810F0010F2B
:1014C000EFD1216808683D4A1040D4E901231A434E
:1014D000D4E9033C43EA0C031A4363691A43A36942
:1014E0001A43E3691A43236A1A431043626A042ABF
:1014F00003D1D4E90B231A431043086026687069AE
:10150000012320F00701606A40EA010204283AD171
:10151000A16AE06A0A4330B3D4F818C0BCF1000FE6
:101520000AD0BCF5005F14D000291CBF0129022994
:1015300021D003291CD026E019B1012905D00229A8
:1015400021D110F0807F1ED015E0B0F1C07F1AD1FC
:1015500011E081B1012907D002290CD0032908BF6D
:10156000B0F1C07F07D00EE010F0807F03D10AE019
:1015700010F0807F07D04FF04000606584F8353070
:101580004FF0010070BD726120680D4AC1B2A1F137
:101590001001A2FB01210B4A4FEA11110329525CF1
:1015A000E2656FF3090088BF001D3F219140A065EF
:1015B0008160656584F83530002070BD3F8010F093
:1015C000ABAAAAAA5839030870B490F834C0002412
:1015D000856DBCF1010F02BF022070BC70474FF057
:1015E000010C80F834C090F835604FF0000C012EEB
:1015F0001CBF80F834C0022402D0204670BC704763
:10160000022680F83560C0F854C0D0F800C0DCF87D
:10161000006026F48026CCF80060D0F800C0CCF83A
:1016200004308368402B036803BF9A600268D1606E
:1016300099601CBF0168CA6090F85C103F2202FAF2
:1016400001F1A96001680A6842F016020A60016CA3
:1016500021B101680A6842F008020A600068016866
:1016600041F001010160C8E770B5044600F04AF995
:101670000546B4F1FF3F02D004480078044400F06E
:1016800041F9401BA042FAD370BD0000A400002025
:10169000022818BF704701200149087070470000F8
:1016A0008D00002004490A68024208BF704710B547
:1016B0000860FFF7EDFF10BD143C01402DE9F84F25
:1016C000DFF818A20022DFF810924FF0010E032776
:1016D0004FF00F080AF1040B0B680EFA02FC03EA44
:1016E0000C03634540F0F2800C7904F00304012CF4
:1016F00018BF022C18D185684FEA420407FA04F695
:1017000025EA0605CE6806FA04F444EA0504846076
:10171000446824EA0C0C0C79C4F3001404FA02F4B3
:1017200044EA0C0CC0F804C0D1F804C037EA0C0C31
:101730000CD0C4684FEA420C07FA0CF5AC438D6834
:1017400005FA0CFC4CEA040CC0F80CC091F804C07B
:101750000CF0030CBCF1020F12D14FEAD20C00EBDB
:101760008C04256A4FEA427C4FEADC6C08FA0CF6DE
:10177000B5430E6906FA0CFC4CEA050CC4F820C00F
:1017800004684FEA420C07FA0CF5AC430D7905F0FA
:10179000030505FA0CFC4CEA040CC0F800C0D1F8B3
:1017A00004C01CF4403F7CD0D9F800C04CF4804CFD
:1017B000C9F800C0D9F800C00CF4804CCDF800C0C6
:1017C00022F0030C0CF1804505F59835D5F808C8D2
:1017D0009407240F08FA04F62CEA0606A0F1804CC0
:1017E000BCF5003C38D0A0F1804CBCF5013C08BFF2
:1017F0004FF0010C30D0A0F1804CBCF5023C08BF8A
:101800004FF0020C28D0A0F1804CBCF5033C08BF7F
:101810004FF0030C20D0A0F1804CBCF5043C08BF75
:101820004FF0040C18D0A0F1804CBCF5053C08BF6B
:101830004FF0050C10D0A0F1804CBCF5063C08BF61
:101840004FF0060C08D0A0F1804CBCF5073C0CBF53
:101850004FF0070C4FF0080C0CFA04FC4CEA060C95
:10186000C5F808C8DAF800C04C682CEA030C14F478
:10187000801F18BF4CEA030CCAF800C0DBF800C098
:101880004C682CEA030C14F4001F18BF4CEA030C3C
:10189000CBF800C0124CD4F800C04D682CEA030C01
:1018A00000E013E015F4003F18BF4CEA030CC4F845
:1018B00000C00C4CD4F800C04D682CEA030C15F4A1
:1018C000803F18BF4CEA030CC4F800C0521C102A19
:1018D000FFF402AFBDE8F88F44380240083C0140F5
:1018E000043C0140003C0140426921EA02031140EE
:1018F00043EA014181617047002A08BF0904816100
:10190000704700000148806870470000A400002074
:10191000002804BF0120704770B5044690F83D00D0
:10192000002520B984F83C50204600F06BFB2420B1
:1019300084F83D002068016821F001010160206801
:10194000016841F4004101602068016821F4004110
:10195000016000F03FFD544B6168994203D8534940
:10196000814203D804E05249814201D9012070BD6F
:1019700050492268B0FBF1F1D2F804C02CF03F0CC2
:101980004CEA010CC2F804C06268934228BF4A1CAA
:1019900007D24FF4967251434FF47A72B1FBF2F1D1
:1019A0004A1C2168D1F820C02CF03F0C42EA0C02FE
:1019B0000A6261688B420FD34900401EB0FBF1F20E
:1019C000521CC2F30B02042A31BF0420B0FBF1F019
:1019D000401CC0F30B0022E0A268002A52D001EBA9
:1019E000C10303EB0113A0F1010CBCFBF3F35B1C7F
:1019F00043F480431B051B0D08BF01200FD0002AB4
:101A000048D001EBC10202EB0111401EB0FBF1F026
:101A1000401CC0F30B0040F4804040F400402168BB
:101A2000CA6922F0FF0222F44F421043C861D4E990
:101A3000070101432068026822F0C00211430160DF
:101A4000D4E9031001432068826822F0FF0222F4E7
:101A5000034211438160D4E9050101432068C26853
:101A600022F0FF021143C1602068016841F00101CA
:101A700001602564202084F83D00256384F83E50F1
:101A8000002070BD01EB4103A0F1010CBCFBF3F39E
:101A90005B1CAFE701EB4101401EB0FBF1F0401CC5
:101AA000C0F30B00B9E70000A086010080841E008F
:101AB00000093D0040420F002DE9F84F984692463C
:101AC0000E4604460A9FFFF71DFF054694F83D00A9
:101AD000202840F06D8119230122B7492046009546
:101AE00002F070FB002840F0638194F83C0001286C
:101AF00000F05E81012084F83C002068016811F04C
:101B0000010F03D1016841F0010101602068016803
:101B100021F400610160222084F83D00102084F847
:101B20003E004FF00009C4F84090C4F824A0A4F887
:101B30002A80608D2085A148E062E06A21680A68F9
:101B400042F480620A6008281CBF012810F5803F1B
:101B500002D0206B112804D12068016841F4807103
:101B600001603B4600224FF001112046009502F033
:101B700029FB4FF4007A30B12068006810F4807FB0
:101B800000F0DF803DE02069DFF834B2B0F5804F2F
:101B900010D0062000EAD618206848F0F001016154
:101BA0002B463A460BF10601204602F075FB38B190
:101BB00000F0C7B8F0B240F001012068016127E0F1
:101BC0002068F1B201612B463A465946204602F0A0
:101BD00063FB002848D12068416981690091016850
:101BE00041F4807101603B4600224FF00111204614
:101BF000009502F0E7FA38B12068006810F4807FA1
:101C000032D0C4F840A09CE0206848F0F1010161A6
:101C10002B463A465946204602F03EFB002823D187
:101C2000208D10B3012829D00228206801682BD00C
:101C300041F4806101602068416980690090208DD5
:101C4000002818BF5F4E72D080B2032873D80128D5
:101C500027D002283B464FF000023146204600952F
:101C600026D002F0AFFAE8B36BE0206841698169E1
:101C70000091016841F400710160E0E720680168AB
:101C800021F480610160F0E721F480610160206847
:101C9000016841F400610160206841698069009039
:101CA000CDE72A463946204602F06CFBF0BB64E0E3
:101CB00002F088FAD0BB2068016841F4007101602D
:101CC00020680069616A0870606A401C6062218D4A
:101CD000491E2185618D491E618521680969017050
:101CE000606A00E008E0401C6062208D401E208594
:101CF000608D401E60854DE02068016821F48061A0
:101D0000016020680069616A0870606A401C606256
:101D1000208D401E2085608D401E60853B46002240
:101D200031462046009502F04DFA02E009E035E028
:101D300001E030B9BFE72A463946204602F022FBCF
:101D400010B10120BDE8F88F20680069616A087051
:101D5000606A401C6062208D401E81B22185608DCA
:101D6000401E60852068426912F0040F12D00329DA
:101D700003D1016821F48061016020680069616A13
:101D80000870606A401C6062208D401E2085608D56
:101D9000401E6085208D00287FF456AF202084F8F7
:101DA0003D0084F83E9084F83C900020BDE8F88F18
:101DB0000220BDE8F88F0000020010000000FFFFC5
:101DC00002000100040001002DE9F84F99469246F7
:101DD0000E4604460A9DFFF795FD074694F83D0020
:101DE000202840F0048119230122824920460097CF
:101DF00002F0E8F9002840F0FA8094F83C0001284D
:101E000000F0F580012084F83C002068016811F0A2
:101E1000010F03D1016841F00101016020680168F0
:101E200021F400610160212084F83D00102084F835
:101E30003E004FF00008C4F84080C4F824A0A4F885
:101E40002A90608D20856C48E062E06A08281CBFFB
:101E5000012810F5803F02D0206B122804D12068A1
:101E6000016841F4807101602B4600224FF001119E
:101E70002046009702F0A6F940B12068006810F4EF
:101E8000807F1CBF4FF400702064ADE02069B0F586
:101E9000804F0ED0062000EAD61040F0F0012068F6
:101EA00001613B462A465549204602F0F5F928B122
:101EB0009AE0206806F0FE01016102E02068F1B2BC
:101EC00001613B462A464E49204602F0E5F90028CA
:101ED0007AD12068416980690090208D4FF02009F7
:101EE000002863D03A462946204602F08FFA40B1D6
:101EF000206C042878D12068016841F400710160E9
:101F000072E0606A216800780861606A421C62625F
:101F1000608D401E6085208D401E81B22185206825
:101F2000436913F0040F18BF00290DD01178016127
:101F3000606A00F101006062608DA0F101006085BF
:101F4000208DA0F10100208520683E46406910F0F8
:101F5000040F28D12068406910F4806F10D02168E8
:101F60006FF480604861C4F8308084F83D9084F854
:101F70003E80206C40F00400206484F83C8030E017
:101F8000B5F1FF3F0AD0FFF7BDFC811BA94200D885
:101F900025B92068406910F0040F16D02068406908
:101FA00010F0040FD6D0208D00289BD12068016846
:101FB00041F40071016084F83D9084F83E8084F81B
:101FC0003C800020BDE8F88F0EE0C4F8308084F833
:101FD0003D9084F83E80206C40F02000206484F81E
:101FE0003C80206C042886D00120BDE8F88F0220B8
:101FF000BDE8F88F020010000000FFFF080001009C
:102000000200010000B587B000210091019102910A
:10201000039104910068A0F18041B1F5A8411CBF73
:1020200007B000BD0F48016841F00201016000687F
:10203000694600F002000590C02000901220019037
:1020400003200390042004900748FFF737FB07485C
:10205000016841F400110160006800F4001005906F
:1020600007B000BD30380240000402404038024052
:10207000024881680278114481607047A400002002
:102080000B4810B5016841F400710160016841F42A
:1020900080610160016841F480710160032000F0FB
:1020A000B5F80F2000F006F800F050F8002010BD41
:1020B000003C024030B505461F4887B00024016847
:1020C00041F020010160006806A900F020000590A1
:1020D000684600F05FF90398A8B100F07BF9400072
:1020E0001649174AB0FBF1F0411E1648026040F253
:1020F000E732C0E90324C0E90114846101F073F8F8
:10210000040016D102E000F065F9E9E70D4801F09E
:1021100001F904000DD1372000F036F8102D28BF4A
:10212000012406D200222946372000F03DF8064857
:10213000056007B0204630BD4038024040420F00E5
:102140000014004038130020A80000200C4882B082
:10215000016841F480410160006800F48040009013
:102160000848016841F0805101600068002200F0D9
:10217000805000900F21901E02B000F015B80000B2
:1021800044380240403802400028B8BF704700F091
:102190001F01012202FA01F14009800000F1E02054
:1021A000C0F8001170470000174B10B41B68C3F350
:1021B0000223C3F1070CBCF1040F88BF4FF0040CDD
:1021C0001C1D072C34BF0023DB1E012404FA0CFC69
:1021D000ACF1010C0CEA0101994004FA03F35B1E17
:1021E0001A40114300284FEA0111A1BF00F1E0207D
:1021F00080F8001410BC704700F00F0000F1E020E0
:1022000080F8141D10BC70470CED00E0074A00F088
:10221000070011684FF6FF03194041EA002040F023
:10222000FD7040F080601060704700000CED00E031
:10223000002804BF012070472DE9F047DFF83C91EA
:1022400004460D46D9F80000CFB200F00700A842BE
:1022500007D289F80070D9F8000000F00700A84202
:1022600063D12068464E10F0020F14D010F0040F16
:1022700003D0306840F4E0503060207810F0080F50
:1022800003D0306840F4604030603068A16820F0CE
:10229000F00008433060207810F0010F37D06068FC
:1022A0003849012823D0022818BF0328096823D001
:1022B00011F0020F39D0316821F0030141EA00002A
:1022C0003060FFF71FFB80463068616800F00C004B
:1022D000B0EB810F18BF41F2883A18D0FFF712FB1C
:1022E000A0EB080050450BD90320BDE8F087096832
:1022F00011F4003FDFD118E011F0007FDBD114E0D2
:102300003068616800F00C00B0EB810FE6D1D9F8BD
:10231000000000F00700A8420AD989F80070D9F837
:10232000000000F00700A84202D00120BDE8F087BD
:10233000207810F0040F05D03068E16820F4E050F8
:1023400008433060207810F0080F06D0306821690B
:1023500020F4604040EAC100306000F05BF8316872
:10236000094AC1F30311515CC84008490860084894
:102370000068FFF79FFE0020BDE8F087003C0240A8
:10238000083802400038024060390308B0000020DD
:10239000A80000200F2202600C4A136803F0030318
:1023A0004360136803F0F0038360136803F4E053A1
:1023B000C36012684FF4E05303EAD202026104489A
:1023C000006800F00700086070470000083802400D
:1023D000003C02400448054900680968044AC1F30A
:1023E0008221515CC8407047B0000020083802408C
:1023F000703903080448054900680968044AC1F3B4
:102400004231515CC8407047B0000020083802409B
:10241000703903081848006810F00C01174808BF0D
:102420007047174B042904BF18467047082918BF86
:10243000704710B5134C216801F03F02216811F478
:10244000800F08D02068C0F38810A0FB0301002390
:10245000FDF718FF07E021680023C1F38811A1FBF5
:102460000001FDF70FFF2168C1F30141491C49003C
:10247000B0FBF1F010BD0000083802400024F40069
:1024800000C0A80004380240002804BF01207047A3
:102490002DE9F84F04460078F84E10F0010FA6F130
:1024A000040556D0301D016801F00C01042908D044
:1024B000006800F00C0008280CD1306810F4800F80
:1024C00008D0286810F4003F43D06068002800F06E
:1024D000D1813EE06068B0F5803F19D0B0F5A02F03
:1024E00028680CBF40F4802020F4803028602868E1
:1024F0000CBF40F4803020F4802028606068B8B1C0
:10250000FFF700FA0746286810F4003F05D020E0E6
:10251000286840F480302860F0E7FFF7F3F9C01B2B
:10252000642800F24181286810F4003FF5D010E0E3
:10253000FFF7E8F90746286810F4003F09D0FFF7D5
:10254000E1F9C01B642800F22F81286810F4003FD5
:10255000F5D12078CA4F10F0020F4FF0000948D093
:10256000C848016811F00C0F15D0006800F00C008D
:10257000082804BF306810F4800F0CD0E06828B33E
:102580004FF001003860FFF7BDF98046286810F071
:10259000020F09D012E0286810F0020F1CBFE0689B
:1025A00001280BD000F066B9FFF7ACF9A0EB0800EA
:1025B00002287DD8286810F0020FF5D0286821691C
:1025C00020F0F80040EAC100286012E0C7F800904F
:1025D000FFF798F98046286810F0020F09D0FFF73E
:1025E00091F9A0EB0800022862D8286810F0020FC9
:1025F000F5D1207810F0080F2FD0A348DFF88CA277
:102600006169A9B101210160FFF77CF98046DAF820
:10261000000010F0020F20D1FFF774F9A0EB0800C2
:10262000022845D8DAF8000010F0020FF4D014E0C8
:10263000C0F80090FFF766F98046DAF8000010F065
:10264000020F0AD0FFF75EF9A0EB080002282FD88E
:10265000DAF8000010F0020FF4D1207810F0040F27
:102660007ED08B484FF00008006810F0805F0AD1E0
:102670008748016841F08051016000684FF001080F
:1026800000F080500090DFF80CB2DBF8000010F48E
:10269000807F1AD1DBF8000040F48070CBF8000096
:1026A000FFF730F98246DBF8000010F4807F00E08D
:1026B0007AE00AD1FFF726F9A0EB0A00022873D8C6
:1026C000DBF8000010F4807FF4D0A068DFF8C8B118
:1026D00001281DD00528DBF800000CBF40F00400E5
:1026E00020F00100CBF80000DBF800000CBF40F048
:1026F000010020F00400CBF80000A068E8B1FFF76B
:1027000001F98246DBF8000010F0020F07D02BE041
:10271000DBF8000040F00100CBF80000EDE7FFF728
:10272000F1F8A0EB0A0141F2883081423CD8DBF895
:10273000000010F0020FF2D016E0FFF7E3F8824637
:10274000DBF8000010F0020F0ED0FFF7DBF8A0EB73
:102750000A0141F28830814226D8DBF8000000E00F
:102760000AE010F0020FF0D1B8F1000F04D0484891
:10277000016821F080510160A069E8B3414909680E
:1027800001F00C0108294ED00228C7F860900ED045
:10279000FFF7B8F80446286810F0007F2CD0FFF748
:1027A000B1F8001B022839D90320BDE8F88FFFF7E4
:1027B000A9F88046286810F0007F09D0FFF7A2F83A
:1027C000A0EB08000228EFD8286810F0007FF5D1B0
:1027D000D4E907010843A16A304A490802EB0141E4
:1027E000626A41EA8211084394F82C1040EA0160C1
:1027F00030600120386600E052E0FFF783F80446BD
:10280000286810F0007F4BD1FFF77CF8001B0228EE
:10281000CAD8286810F0007FF6D041E0286810F090
:10282000007FBCD13CE0012808BFBDE8F88F3068CC
:10283000E26900F4800191421CD1226A00F03F015C
:10284000914217D147F6C071626A0140B1EB821F15
:1028500010D1A26A4FF0FF3300F4403103EB520273
:10286000B1EB024F06D194F82C1000F07060B0EB81
:10287000016F15D00120BDE8F88F00000438024038
:102880000000474208380240800E47427438024038
:102890004038024000700040703802400000FFFFE6
:1028A0000020E8E7002804BF0120704770B5044607
:1028B000406A002500281CBF2561656104D0A5621F
:1028C00094F8510058B905E06068B0F5827F18BFF0
:1028D000E561F4E784F85050204600F045F8022006
:1028E00084F851002068016821F040010160A0884F
:1028F000218900F4827001F404410843A18901F4A4
:1029000000610843217C01F002010843217D01F0B0
:1029100001010843218B01F400710843217F01F07C
:102920003801084394F8201001F080010843218DFC
:1029300001F40051084321680860A169042000EAFD
:10294000114094F8241001F0100101432068416007
:102950002068C16921F40061C1616565012084F8C6
:102960005100002070BD0000F0B587B00024009435
:10297000019402940394049401683C4A02250326BE
:102980000527A1F18040B0F5983029D0384B39485F
:10299000A1F1804CBCF5605C3BD0A1F1804CBCF552
:1029A000705C1CBF07B0F0BD196841F400411960AC
:1029B000196801F400410591116841F004011160AA
:1029C000116801F0040105914FF4E051CDE90015C3
:1029D0000621CDE903616946FEF770FE07B0F0BD40
:1029E0002548016841F480510160006800F480507E
:1029F0000590106840F0010010601068694600F012
:102A000001000590E020CDE900051C48CDE90367F1
:102A100028E0196841F480411960196801F4804187
:102A20000591116841F004011160116801F0040181
:102A30000591116841F002011160116801F0020175
:102A400005910C21CDE900156946CDE90367FEF734
:102A500035FE4FF40050CDE90005CDE90246694648
:102A600004970748FEF72AFE07B0F0BD3038024051
:102A70004038024000080240443802400000024052
:102A8000000402402DE9F84F044690F851001D461D
:102A900091468A46012836D160680427B0F5827FC6
:102AA00004BFA068002824D0FEF72CFF0646BAF128
:102AB000000F18BFB9F1000F76D094F8500001282C
:102AC00021D04FF0010884F8508084F8517000271D
:102AD0006765C4F838A0A4F83C90A4F83E9027633A
:102AE000A786E78627646764A068B0F5004F0DD01D
:102AF00016E084F85170009313460A46204600F011
:102B000045F9BDE8F88F0220BDE8F88F206801681C
:102B100021F0400101602068016821F480410160DA
:102B20002068016811F0400F03D1016841F04001B5
:102B30000160E0680028E08F0FD058B320688168FA
:102B400011F0010F27D0C068A16B0880A06B801C1A
:102B5000A063E08F401EE08728E0D8B1206881683C
:102B600011F0010F09D0007BA16B0870A06B401C15
:102B7000A063E08F401EE08709E0FEF7C3FE801BE4
:102B8000A84203D3B5F1FF3F28D100E035B3E08F71
:102B90000028E3D10DE0FEF7B5FE801BA84204D368
:102BA000B5F1FF3F1AD101E015E0BDB1E08F00287B
:102BB000C4D132462946204602F0E0F900281CBF65
:102BC0002020606584F8518084F85070606D002882
:102BD00008BFBDE8F88F0120BDE8F88F84F8518068
:102BE00084F850700320BDE8F88F2DE9F84F1D469A
:102BF00016468A460446FEF785FE074694F85100BD
:102C0000012826D1BAF1000F18BF002E71D094F818
:102C1000500001281DD04FF0010984F85090032086
:102C200084F851004FF00008C4F85480C4F830A074
:102C3000A686E686C4F83880A4F83C80A4F83E80D6
:102C4000C4F84480C4F84080A068B0F5004F03D0B9
:102C50000CE00220BDE8F88F2068016821F04001F7
:102C600001602068016841F48041016020680168CA
:102C700011F0400F03D1016841F040010160E068AC
:102C8000B0F5006F606804D0002818BF012E31D065
:102C90003AE0002818BF012E0BD1206B2168008874
:102CA000C860206B00F102002063E08EA0F10100FB
:102CB000E086E08E002845D02068816811F0020F80
:102CC00009D0216B0988C160206B801C2063E08ED5
:102CD000401EE08609E0FEF715FEC01BA84203D3A4
:102CE000B5F1FF3F3BD100E0C5B3E08E0028E3D152
:102CF00028E048E0206B216800780873206B401CB6
:102D00002063E08E401EE086E08ED8B120688168A6
:102D100011F0020F09D0216B09780173206B401C60
:102D20002063E08E401EE08609E0FEF7EBFDC01B4D
:102D3000A84203D3B5F1FF3F11D100E075B1E08E99
:102D40000028E3D13A462946204602F055F90028EA
:102D50001CBF20206065A06860B907E0FFE784F829
:102D6000519084F850800320BDE8F88F2068C16836
:102D70008068009084F8519084F85080606D00283D
:102D800008BFBDE8F88F0120BDE8F88F2DE9F84FA6
:102D90001F4692468B46044601250A9EFEF7B2FD69
:102DA000804694F851006168012806D0B1F5827F11
:102DB00002BFA168002904282BD1BBF1000F1CBF62
:102DC000BAF1000F002F00F0F38094F850000128B2
:102DD0001FD0012084F8500094F8510004281CBF33
:102DE000052084F851004FF00009C4F85490C4F84D
:102DF00038A0E787A787C4F830B0E786A786C4F86D
:102E00004090C4F844902068016811F0400F07D149
:102E100002E00220BDE8F88F016841F04001016046
:102E2000E068B0F5006F606804D0002818BF012F7B
:102E30005AD09BE0002818BF012F41D1206B216898
:102E40000088C860206B00F102002063E08EA0F1D2
:102E50000100E08634E02068816811F0020F1CBF99
:102E6000E18E00290ED0012D0CD1216B0988C160A3
:102E7000206B00F102002063E08EA0F10100E086EB
:102E80004FF000052068816811F0010F1CBFE18F31
:102E900000290CD0C068A16B0880A06B00F1020073
:102EA000A063E08FA0F10100E0874FF00105FEF77D
:102EB00029FDA0EB0800B04202D3B6F1FF3F5CD180
:102EC000E08E002804BFE08F0028C4D1424631467E
:102ED000204602F091F8002859D02020606584F83F
:102EE00050900120BDE8F88F206B216800780873AE
:102EF000206B401C2063E08E401EE08636E0206898
:102F0000816811F0020F1CBFE18E00290ED0012D47
:102F10000CD1216B09780173206B00F10100206353
:102F2000E08EA0F10100E0864FF000052068816886
:102F300011F0010F1CBFE18F00290CD0C068A16BFC
:102F40000870A06B00F10100A063E08FA0F1010008
:102F5000E0874FF00105FEF7D5FCA0EB0800B0427A
:102F600003D3B6F1FF3F01D007E036B1E08E002871
:102F700004BFE08F0028C2D1A8E74FF0010084F819
:102F8000510084F850904FF00300BDE8F88FA0681E
:102F900018B92068C168806800904FF0010084F87B
:102FA000510084F85090606D002808BFBDE8F88F8C
:102FB0004FF00100BDE8F88F7047704790F83C2053
:102FC000012A04BF02207047012280F83C20CA6811
:102FD000D1F808C022F4407242EA0C02D1F804C0D1
:102FE00022F4806242EA0C02D1F800C022F40062AE
:102FF00042EA0C02D1F810C022F4805242EA0C02DC
:10300000D1F814C022F4005242EA0C02C96900232C
:1030100022F4804211430268516480F83C30002061
:10302000704790F83C20012A04BF0220704730B45A
:10303000012480F83C40022280F83D200268D2F84A
:1030400004C093680D682CF0700C45EA0C0CC2F8B3
:1030500004C00268A2F1804CBCF5803C18BFB2F1FC
:10306000804F1DD0A2F1804CBCF5806C1CBFA2F13A
:10307000804CBCF5006C13D0A2F1804CBCF5406CC8
:103080001CBFA2F1804CBCF5823C09D0A2F1804C5F
:10309000BCF5A03C1CBFA2F1804CBCF5C05C04D1C7
:1030A000496823F080031943916080F83D40002176
:1030B00080F83C1030BC0846704710B50446002923
:1030C00008BF94F842000AD0042908BF94F84300CE
:1030D00005D008290CBF94F8440094F84500012855
:1030E0001CBF012010BD0220002908BF84F8420047
:1030F0000AD0042908BF84F8430005D008290CBF72
:1031000084F8440084F845000422206802F021F984
:103110002068416C41F4004141642068A0F1804185
:10312000B1F5803118BFB0F1804F1DD0A0F18041C2
:10313000B1F580611CBFA0F18041B1F5006113D0F1
:10314000A0F18041B1F540611CBFA0F18041B1F513
:10315000823109D0A0F18041B1F5A0311CBFA0F1AE
:103160008041B1F5C05104D1816801F00701062901
:1031700003D0016841F001010160002010BD70B56D
:1031800004460D460068002202F0E3F82068026A57
:1031900041F211110A4240F2444204BF036A134251
:1031A00003D1436C23F4004343642068036A0B4259
:1031B00004BF016A114203D1016821F001010160DD
:1031C0000120002D08BF84F842000AD0042D08BF5A
:1031D00084F8430005D0082D0CBF84F8440084F81F
:1031E0004500002070BD002804BF0120704710B5C5
:1031F000044690F83D0028B9002084F83C002046A1
:1032000000F01EF8022084F83D00211D206802F025
:103210001DF8012084F8460084F83E0084F83F0041
:1032200084F8400084F8410084F8420084F84300A8
:1032300084F8440084F8450084F83D00002010BD67
:1032400000B587B000210091019102910391049192
:103250000068A0F18041B1F580311ED02949A0F16C
:103260008042B2F5806228D0A0F18042B2F580524F
:103270001CBF07B000BD086840F010000860086877
:10328000002200F01000059005213620FEF78CFF8B
:103290003620FEF779FF07B000BD1B48016841F0FA
:1032A000010101600068002200F001000590052185
:1032B0001920FEF779FF192020E0086840F002008D
:1032C0000860086800F0020005901048016841F0AD
:1032D000020101600068694600F0020005900220CA
:1032E000009001900290039004900948FEF7E6F9DF
:1032F000002205211D20FEF757FF1D20FEF744FF89
:1033000007B000BD40380240443802403038024027
:103310000004024090F83D1001291CBF01207047B5
:10332000022180F83D100168CA6842F00102CA60BB
:103330000068A0F18041B1F5803118BFB0F1804F35
:103340001DD0A0F18041B1F580611CBFA0F180418A
:10335000B1F5006113D0A0F18041B1F540611CBF0F
:10336000A0F18041B1F5823109D0A0F18041B1F5E1
:10337000A0311CBFA0F18041B1F5C05104D18168DA
:1033800001F00701062903D0016841F00101016045
:103390000020704790F83C200023012A0DBF022036
:1033A0004FF0010C80F83CC0704770B4022280F8E6
:1033B0003D200268946824F0770424F47F449460EC
:1033C0000A68502A43D00CDC202A75D004DC002A7D
:1033D00018BF102A0FD18BE0302A6DD0402A6DD053
:1033E00009E0602A4DD0702A0ED0B2F5805F03D07C
:1033F000B2F5005F19D0012380F83DC0002180F8AC
:103400003C1070BC18467047D1E901450268C96894
:10341000966844EA012126F47F46294331439160AE
:1034200001688A6842F077020FE0D1E9014502683D
:10343000C968966844EA012126F47F46294331434E
:10344000916001688A6842F480428A60D4E7026829
:10345000CD684C68116A166A26F0010616629669F4
:1034600021F00A0126F0F00646EA05152143956190
:10347000116201688A6822F0700242F057028A6085
:10348000BAE702684C68C968156A166A26F0100621
:103490001662966925F0A00526F4704646EA0131C9
:1034A00045EA04149161146201688A6822F070028E
:1034B00042F067028A609FE71AE0FFE702684C6803
:1034C000C968156A166A26F001061662966925F023
:1034D0000A0526F0F00646EA01112C4391611462B8
:1034E00001688A6822F0700242F047028A6083E72E
:1034F00001688C6824F07004224342F007028A605D
:103500007AE700000E49814218BF704710B50D4C94
:10351000207818B10C210A4800F08AF90C210848DB
:1035200000F090FB00EE100A2078B8EE400A04EBA1
:10353000800080ED040A2078401C207010BD00003F
:103540007C0B0020801300202DE9F041054690F807
:103550003C0000260C46012804BF0220BDE8F08193
:10356000012085F83C007AB14FF47047042A1BD043
:10357000082A45D00C2A18BF012669D0002085F8FA
:103580003C003046BDE8F081D4E90012E3682868C9
:1035900001F05EFF2868816921F00C0181612868D3
:1035A0008169A268114329E02868D4E90032E16802
:1035B000D0F820C0D0F8208028F01008C0F8208073
:1035C000D0F8188007EA013128F4407848EA02224E
:1035D00022F4704211432CF0A0024FF0A00C0CEA30
:1035E00003131A43816102622868816921F44061F2
:1035F000816128688169A26841EA02218161BDE791
:103600002868D4E90013D4F80CC0026A076A27F4CA
:1036100080770762C76922F4206227F003073B43E3
:10362000F02723F0F00307EA0C1C4CEA03034FF4E5
:10363000206C0CEA01211143C36101622868C16951
:1036400021F00C01C1612868C169A268114329E019
:103650002868D4E90021E368D0F820C0D0F82080A1
:1036600028F48058C0F82080D0F81C8007EA033383
:1036700028F4407848EA012121F4704119432CF4E0
:1036800020434FF4204C0CEA02321A43C16102621B
:103690002868C16921F44061C1612868C169A268D4
:1036A00041EA0221C16169E7002804BF0120704797
:1036B00010B5044690F83D0028B9002084F83C007D
:1036C000204600F01EF8022084F83D00211D2068ED
:1036D00001F0BCFD012084F8460084F83E0084F827
:1036E0003F0084F8400084F8410084F8420084F8E8
:1036F000430084F8440084F8450084F83D0000202D
:1037000010BD704730B500250446002908BF94F865
:103710003E000AD0042908BF94F83F0005D00829CC
:103720000CBF94F8400094F84100002908BF94F8B9
:1037300042200AD0042908BF94F8432005D0082964
:103740000CBF94F8442094F8452001280EBF012AAC
:10375000012030BD4FF00200002904BF84F83E0074
:1037600084F8420010D0042904BF84F83F0084F894
:10377000430009D0082907BF84F8400084F84400BA
:1037800084F8410084F8450041B104290BD0082990
:103790000ED00C2918BF01250FD047E02068C26861
:1037A00042F002020DE02068C26842F0040208E024
:1037B0002068C26842F0080203E02068C26842F054
:1037C0001002C2600122206801F0B4FD2068A0F15F
:1037D0008041B1F5803118BFB0F1804F1DD0A0F10C
:1037E0008041B1F580611CBFA0F18041B1F500615D
:1037F00013D0A0F18041B1F540611CBFA0F1804120
:10380000B1F5823109D0A0F18041B1F5A0311CBFE2
:10381000A0F18041B1F5C05104D1816801F00701E8
:10382000062903D0016841F001010160284630BD3E
:1038300070B50D0004464FF0000609D0042D0CD0E1
:10384000082D0FD00C2D18BF012610D0304670BDAA
:103850002068C16821F002010DE02068C16821F0F4
:10386000040108E02068C16821F0080103E0206835
:10387000C16821F01001C16000222946206801F0D2
:1038800059FD2068016A41F21112114207D1016A03
:103890009210114203D1016821F001010160012061
:1038A000002D04BF84F83E0084F84200CED0042DE1
:1038B00004BF84F83F0084F84300C7D0082D07BF39
:1038C00084F8400084F8440084F8410084F84500FE
:1038D000BCE72DE9F04104460068C66805694FF071
:1038E000000715F0020F18BF16F0020F13D06FF08B
:1038F00002010161012020772068806910F0030F28
:10390000204602D0FFF7FEFD04E000F08CF82046D0
:1039100000F07AF9277715F0040F18BF16F0040F9E
:1039200014D021686FF0040008610220207720681D
:10393000806910F4407F204602D0FFF7E3FD04E0E9
:1039400000F071F8204600F05FF9277715F0080FB6
:1039500018BF16F0080F14D021686FF00800086136
:10396000042020772068C06910F0030F204602D0A1
:10397000FFF7C8FD04E000F056F8204600F044F9D7
:10398000277715F0100F18BF16F0100F14D021680C
:103990006FF010000861082020772068C06910F4DB
:1039A000407F204602D0FFF7ADFD04E000F03BF879
:1039B000204600F029F9277715F0010F18BF16F0FF
:1039C000010F06D021686FF001000861204600F069
:1039D0001CF915F0800F18BF16F0800F06D0216873
:1039E0006FF0800008612046FFF7E6FA15F0400FFF
:1039F00018BF16F0400F06D021686FF04000086134
:103A0000204600F035F915F0200F14BF16F0200FF6
:103A1000BDE8F0816FF02000216808612046BDE814
:103A2000F041FFF7CABA70472DE9F041044690F81B
:103A30003C0000260D46012804BF0220BDE8F081AD
:103A4000012084F83C0082B1042A20D0554FDFF8D1
:103A500058C1082A2FD00C2A18BF01266ED000208A
:103A600084F83C003046BDE8F081206801F080FC1D
:103A70002068816941F0080181612068816921F035
:103A800004018161206881692A69114311E020687D
:103A900001F0A6FC2068816941F400618161206821
:103AA000816921F480618161206881692A6941EA24
:103AB00002218161D3E72068016A026A22F48072E0
:103AC00002624268C369D5F8008023F0730348EAB4
:103AD0000303D5F8088021F4007141EA0821B842B7
:103AE00018BF604507D1D5F80C8021F4006141EA88
:103AF000082121F48061B84218BF604509D1D5F88A
:103B000014C022F4405242EA0C12D5F818C042EA1E
:103B10000C124260C3616A68C26301622068C169B5
:103B200041F00801C1612068C16921F00401C1614F
:103B30002068C1692A6941EA020131E02068026A0D
:103B4000016A21F4805101624168C369D5F800809F
:103B500023F4E64343EA0823D5F8088022F4005210
:103B600042EA0832B84218BF604505D1D5F814C002
:103B700021F4804141EA8C114160C36169680164AC
:103B800002622068C16941F40061C1612068C169B5
:103B900021F48061C1612068C1692A6941EA02217A
:103BA000C1615CE70000014000040140002804BF3F
:103BB0000120704710B5044690F83D0028B9002058
:103BC00084F83C00204600F01EF8022084F83D00F6
:103BD000211D206801F03AFB012084F8460084F89A
:103BE0003E0084F83F0084F8400084F8410084F8E7
:103BF000420084F8430084F8440084F8450084F8C7
:103C00003D00002010BD7047704710B504460068A5
:103C1000A0F18041B1F5A05108BFFEF729FA206854
:103C2000A0F18041B1F5806108BF0CF0D3FA2068A3
:103C3000A0F18041B1F5805118BF10BDBDE8104022
:103C40000CF0D0BA02460020002902BF1068406B79
:103C50007047042902BF1068806B7047082902BFB3
:103C60001068C06B70470C2904BF1068006C704767
:103C70007047704770470000F8B50168044608684F
:103C8000CA684B6910F00F0F4FF0000569D003F0C0
:103C9000010C02F490765CEA060677D010F0010F72
:103CA00018BF12F4807F03D0616C41F001016164A0
:103CB00010F0040F18BF13F0010F03D0616C41F036
:103CC0000201616410F0020F18BF13F0010F03D05E
:103CD000616C41F00401616410F0080F1CBF02F038
:103CE000200151EA0C0103D0616C41F008016164CC
:103CF000616C002908BFF8BD10F0200F1EBF12F044
:103D0000200F204601F019FC20684069616CC0F367
:103D1000801011F0080F08BF002832D0204601F0B3
:103D2000E5FB2068406910F0400F25D0206800F1C5
:103D3000140050E8001F21F0400140E80012002A62
:103D4000F4D1E06BC0B17B490165E06BFDF78DFA02
:103D5000002808BFF8BDE06B016D01B0BDE8F04080
:103D6000084710F0200F18BF12F0200F0ED0204689
:103D7000BDE8F84001F0E1BB2046FFF77BFFF8BD4E
:103D800004E02046FFF776FF6564F8BDD4F830C044
:103D90002023BCF1010F7CD110F0100F18BF12F0DE
:103DA000100F76D008684868009048694FF0020606
:103DB00010F0400F45D0E16B086840680004000C2B
:103DC0001CBFA28D824298BFF8BDE085C869B0F5DE
:103DD000807F2DD020680C3050E8001F21F48071C6
:103DE00040E80012002AF5D12068143050E8001F86
:103DF00021F0010140E80012002AF5D120681430BA
:103E000050E8001F21F0400140E80012002AF5D1DF
:103E100084F84230256320680C3050E8001F21F000
:103E2000100140E80012002AF5D1E06BFDF7CAF955
:103E30006663A08DE18D401A81B22046FFF719FF1D
:103E4000F8BDA08DE18D401A81B2E08D002814BF2D
:103E50000029F8BD206800F10C0050E8002F22F482
:103E6000907240E8002CBCF1000FF3D120681430B0
:103E700050E8002F22F0010240E8002CBCF1000FB6
:103E8000F4D184F84230256320680C3050E8002FCC
:103E900000E00AE022F0100240E80023002BF3D1FA
:103EA00066632046FFF7E5FEF8BD10F0800F18BFEF
:103EB00012F0800F2DD094F84100212818BFF8BDD2
:103EC000A068B0F5805F04BF20690028206A18D080
:103ED00000F101012162216800784860E08CA0F1C6
:103EE00001000004000CE08418BFF8BD2068C16820
:103EF00021F08001C1602068C16841F04001C160CB
:103F0000F8BD0088C0F308004860206A801C206269
:103F1000E4E710F0400F14BF12F0400FF8BD204648
:103F2000CA6822F04002CA6084F8413000F048F9C3
:103F3000F8BD0000DD540008002804BF01207047D0
:103F400070B5044690F84100002520B984F840502F
:103F5000204600F023F8242084F841002068C1683E
:103F600021F40051C160204601F04EFB2068016938
:103F700021F4904101612068416921F02A014161E9
:103F80002068C16841F40051C1606564202084F854
:103F9000410084F842006563002070BDF0B587B031
:103FA0000021009101910291039104910168514C0B
:103FB000514A022307265148A1F180454FF0030CD6
:103FC000B5F5883535D0251FA1F18047B7F588476D
:103FD0004FD0A1F18040B0F5904069D0A1F1804070
:103FE000B0F58A301CBF07B0F0BD206840F020005B
:103FF0002060206800F020000590106840F0040068
:1040000010601068694600F004000590C020CDE9FA
:1040100000030820CDE903C03948FDF74FFB00221B
:1040200005214720FEF7C0F84720FEF7ADF807B09E
:10403000F0BD216841F010012160216801F01001FC
:104040000591116841F001011160116801F0010151
:1040500005914FF4C061CDE90013CDE903C669466F
:10406000FDF72CFB002205212520FEF79DF82520D9
:10407000DBE7296841F400312960296801F4003147
:104080000591116841F001011160116801F0010111
:1040900005910C21CDE90013CDE903C66946FDF772
:1040A0000DFB002205212620FEF77EF82620BCE726
:1040B000286840F480202860286800F4802005905B
:1040C000106840F0020010601068694600F00200BD
:1040D00005904FF44060CDE90003CDE903C60948DF
:1040E000FDF7ECFA002205212720FEF75DF82720D6
:1040F0009BE7000044380240303802400000024094
:10410000000802400004024070472DE9F8430446CD
:1041100090F841001F4615460E4620281CBF02207D
:10412000BDE8F883002E12BF002D0120BDE8F88302
:104130004FF0000060644FF0210084F84100FDF76B
:10414000E1FBA5848146E584A068B0F5805F07BFE8
:10415000206900283546002608BF0025E08C4FF076
:104160002008A0B14B464FF000024FF080012046DE
:10417000009701F0C7FAB8B9DDB1216815F8010B55
:104180004860E08C401EE084E08C0028EAD14B4679
:10419000002240212046009701F0B4FA002804BF15
:1041A00084F84180BDE8F88384F841800320BDE8AD
:1041B000F88336F8020B2168C0F308004860E0E796
:1041C0007047FEE72DE9F0470446C1F30748DDF8E4
:1041D000209000681E4617460D46B8F1010F06D024
:1041E000806925EA00000004000C14D005E0406955
:1041F00025EA00000004000C0DD00020B84246D192
:10420000B6F1FF3F2FD0FDF77DFBA0EB0900B042D8
:1042100003D846BB01E00120F0E72068B8F1010FA8
:1042200006D0806925EA00000004000C19D005E0E2
:10423000406925EA00000004000C12D00020B842BA
:1042400011D100202063202184F83D1084F83E0025
:10425000216C41F02001216484F83C000120BDE87C
:10426000F0870120EBE72068B8F1010F06D08069E4
:1042700025EA00000004000C0CD005E0406925EAA6
:1042800000000004000C05D00020B842B8D0002087
:10429000BDE8F0870120F8E72DE9F0470446C1F3B7
:1042A00007470068984616460D46012F26D08069BC
:1042B00025EA00000004000C61D04FF000094FF027
:1042C000200A2068406910F4806F1ED020680168C1
:1042D00041F40071016021686FF480604861C4F8A6
:1042E000309084F83DA084F83E90206C40F00400AB
:1042F000206484F83C900120BDE8F087406925EAFD
:1043000000000004000CD8D139E0B6F1FF3F06D020
:10431000FDF7F8FAA0EB0800B04203D816B1012F60
:104320001ED025E02068012F14D0806925EA000006
:104330000004000C1CD0C4F8309084F83DA084F830
:104340003E90206C40F02000206484F83C900120D6
:10435000BDE8F087406925EA00000004000CEAD1BE
:104360002068406925EA00000004000CA9D106E09D
:104370002068806925EA00000004000CA1D100201B
:10438000BDE8F0872DE9F0410446006816460D4669
:10439000406910F0400F04BF00274FF0200824D1DF
:1043A0002068406910F0100F0FD020686FF01001E6
:1043B0004161276384F83D8084F83E70206C20645E
:1043C00084F83C700120BDE8F081FDF79BFA801B6A
:1043D000A84200D825B92068406910F0400F07D0E6
:1043E0002068406910F0400FDAD00020BDE8F0816D
:1043F000276384F83D8084F83E70206C40F02000F4
:10440000206484F83C700120BDE8F0812DE9F04182
:104410000446006816460D46406910F0800F04BF40
:1044200000274FF0200829D12068406910F4806FE0
:1044300011D020686FF480614161276384F83D806A
:1044400084F83E70206C40F00400206484F83C70D6
:104450000120BDE8F081B5F1FF3F0AD0FDF752FA27
:10446000801BA84200D825B92068406910F0800F51
:1044700007D02068406910F0800FD5D00020BDE83B
:10448000F081276384F83D8084F83E70206C40F012
:104490002000206484F83C700120BDE8F081000019
:1044A00030B585B000241548009401940294124957
:1044B0000394C0E90014012505618460057680F845
:1044C00020400F49C0E90A14C561C46080F830403B
:1044D0004561FCF7A5FB002818BFFCF7E7FACDE91A
:1044E0000045694605480294FCF7E2FA002818BF27
:1044F000FCF7DCFA05B030BD002001401C090020AB
:104500000100000F10B582B00024104900940E483D
:10451000019408600846FCF7B8FD002818BFFCF7B6
:10452000C5FA0220CDE90040002269460748FCF7A1
:1045300044FD002818BFFCF7B9FA00210348FCF736
:1045400009FE02B010BD000000740040C409002044
:10455000094808B5016841F4800101600068002243
:1045600000F48000009005213820FDF71DFEBDE815
:1045700008403820FDF708BE30380240F0B5B9B029
:1045800000203690379036A826F00EFA324D334C84
:1045900032AE686294E80F0086E80F00002132A86E
:1045A00026F0EBF91034286294E8CF108DE8CF1094
:1045B00000216846103C26F059FA2C34686094E8D3
:1045C000CF100DF11C0E2C3C8EE8CF10002107A857
:1045D00026F04CFA4834A86094E8CF100DF1380E5C
:1045E000483C8EE8CF1000210EA826F03FFA643434
:1045F000E86094E8CF100DF1540E643C8EE8CF10C3
:10460000002115A826F032FA8034286194E8CF10F2
:104610000DF1700E803C8EE8CF1000211CA826F012
:1046200025FA9C34686194E8CF100DF18C0E9C3C07
:104630008EE8CF10002123A826F018FAB834A8611C
:1046400094E85F102AAF87E85F1000212AA826F0BF
:104650000DFAE86139B0F0BD00000020843803088D
:104660002DE9F04F87B00024814800940194029412
:1046700003940494016841F010010160016801F0A5
:1046800010010591016841F004010160016801F029
:1046900004010591016841F080010160016801F0A9
:1046A00080010591016841F001010160016801F09C
:1046B00001010591016841F002010160016801F00A
:1046C00002010591016841F0080101600068DFF80E
:1046D000A49100F008000590002240F2BF71484606
:1046E000FDF70AF9DFF890A100224EF211015046C1
:1046F000FDF702F901224FF481715046FDF7FCF8F5
:10470000012291034846FDF7F7F8DFF870B1002267
:104710004FF4A2415846FDF7EFF8594F00224FF2EF
:10472000BB313846FDF7E8F8012240F20441384633
:10473000FDF7E2F8DFF84C8100224FF4C05140460B
:10474000FDF7DAF844F23F0000900125CDE901546D
:10475000694648460394FCF7B1FF4AF213100090F3
:10476000CDE90154694650460394FCF7A7FFA8031E
:104770000226CDE90005CDE9026469465046FCF702
:104780009DFF4FF404100096CDE9010469464046B0
:10479000FCF794FF4FF4F0604FF0030ACDE90005F9
:1047A000CDE9024A69464846FCF788FFE8030090D5
:1047B0004FF48810CDE9010469464846FCF77EFFB6
:1047C0004FF4A2400090CDE9015469465846039445
:1047D000FCF774FF4FF48270CDE90005CDE9025477
:1047E00069463846FCF76AFF4FF402700090CDE945
:1047F0000154694638460394FCF760FFA8024FF065
:104800001109CDE90009CDE9025469463846FCF7A3
:1048100055FFEE02CDE90064694638460294FCF784
:104820004DFF4FF2B300CDE90005CDE9024A6946DC
:104830003846FCF743FF0096CDE9015469464046EF
:104840000394FCF73BFF2803CDE90009CDE90254AE
:1048500069464046FCF732FF002205210720FDF79C
:10486000A3FC0720FDF790FC07B0BDE8F08F000027
:1048700030380240001002400008024000040240AC
:10488000000C0240000002400D4810B50B490160C9
:104890004CF25031416000214FF480428160C0E908
:1048A000031241618161C1610162FDF731F80028A5
:1048B00008BF10BDBDE81040FCF7F8B80054004038
:1048C000D8090020104810B50E4901604FF48271DC
:1048D0004160002181600122C160C0E904125202DE
:1048E00082611022C0E90721416281620A21C1620E
:1048F000FDF7D8FF002808BF10BDBDE81040FCF749
:10490000D5B80000003001402C0A0020104810B536
:104910000E4901604FF482714160002181600122E3
:10492000C160C0E90412520282611822C0E9072165
:10493000416281620A21C162FDF7B4FF002808BF0D
:1049400010BDBDE81040FCF7B1B8000000380040D1
:10495000840A0020104810B50E4901604FF482719E
:104960004160002102228160C0E903121202C0E905
:1049700005122022C0E90721416281620A21C16239
:10498000FDF790FF002808BF10BDBDE81040FCF700
:104990008DB80000003C0040DC0A0020F0B59BB060
:1049A0000024149415941694179418941994089448
:1049B00009940A940B940C943F4D0D940E9400941A
:1049C0000194029403940494059406944AF2FF100F
:1049D0000794C5E9024080202C61C5E90540354FA8
:1049E0000126C5E900762846FEF7FDFB002818BF22
:1049F000FCF75CF84FF48050149014A92E48FEF791
:104A0000C9FC002818BFFCF751F82B48FFF7CEF877
:104A1000002818BFFCF74AF8189418A926481994DA
:104A2000FEF7FFFA002818BFFCF740F86020089056
:104A30004FF4FA70CDE909040420CDE90B40024699
:104A40000D9408A91C480E94FEF7EEFF002818BF2D
:104A5000FCF72CF800944FF40050CDE90440029488
:104A600001940394694614480794FEF7A7FA0028B6
:104A700018BFFCF71BF80F94109411941294139420
:104A80002868B8421CBF1BB0F0BD0C48016841F05B
:104A90000201016000680FA900F002001A900220D4
:104AA000CDE90F60119606481396FCF707FE1BB080
:104AB000F0BD000000000140340B002030380240FF
:104AC0000004024010B58AB00024244800940194E8
:104AD00002940394049405940694079408941E4940
:104AE0000994C0E900144FF6FF71C0E9024180212A
:104AF00004618161FEF777FB002818BFFBF7D6FF42
:104B00004FF48050009069461448FEF743FC00289B
:104B100018BFFBF7CBFF1148FEF7C6FD002818BFF2
:104B2000FBF7C4FF049404A90C480594FEF779FA36
:104B3000002818BFFBF7BAFF0120CDE90640089412
:104B40000C2206A905480994FEF7FEFC002818BFB0
:104B5000FBF7ACFF0AB010BD000400407C0B002046
:104B600010B582B00024104800940E4901940160F1
:104B70000121C0E901144AF2FF11C1608021816165
:104B8000FEF731FB002818BFFBF790FF0094694641
:104B900005480194FEF745FA002818BFFBF786FF89
:104BA00002B010BD00100040C40B002010B5134C23
:104BB00011484FF4C06120604FF4966060604FF47C
:104BC0008050A0600020C4E903010C21C4E9051055
:104BD000E0612046FFF7B0F9002818BFFBF766FF39
:104BE0002068C16841F02001C1602068C16841F0BF
:104BF0001001C16010BD000000100140181200201B
:104C000010B5114C0F480C2120604FF41650606015
:104C10000020A060E060C4E90401A061E0612046DA
:104C2000FFF78AF9002818BFFBF740FF2068C1682A
:104C300041F02001C1602068C16841F01001C160ED
:104C400010BD000000440040601200200C4810B568
:104C50000A4901604FF4E1314160002181600C227A
:104C6000C160C0E904128161C161FFF765F90028E4
:104C700008BF10BDBDE81040FBF718BF004800405A
:104C8000A812002010B5114C0F480C2120604FF4E1
:104C9000E13060600020A060E060C4E90401A06130
:104CA000E0612046FFF748F9002818BFFBF7FEFE39
:104CB0002068C16841F02001C1602068C16841F0EE
:104CC0001001C16010BD000000140140F01200206E
:104CD000FEE7FEE7F8B50446294E00200090294F74
:104CE0000D460122F06011033846FCF705FE022054
:104CF00005F06DFB0022B9143846FCF7FDFD0220DB
:104D000005F065FB002C1CBF602000F0E3F8307854
:104D10002040284314BF032202224FF47A736946CD
:104D20001948FDF7AFFE9DF80000F1689DF80120DD
:104D3000014342EA0121F1603178214029430CD03E
:104D400010445B309DF80210C0B240F081007170D9
:104D500081421CBF4FF0FF30F8BD012211033846DD
:104D6000FCF7CAFD022005F032FB00224FF480510F
:104D70003846FCF7C1FD022005F029FBF068F8BDBC
:104D80009000002000040240840A002010B5642036
:104D9000FCF76AFC00F07CF8642005F018FBDD23CA
:104DA00089222021022000F0A7F8022000F012F84A
:104DB0000649002208614FF480510548FCF79CFD2C
:104DC000BDE81040022005F002BB0000900000206A
:104DD00000040240F0B52B4F0446012283B01103BA
:104DE0003846FCF789FD022005F0F1FA0022B914DB
:104DF0003846FCF781FD022005F0E9FA44F0400056
:104E000000F068F800244FF47A768DF804408DF8AD
:104E10000840012302AA01A91B480096FDF7B6FF2E
:104E20001A4D9DF808000123A8708DF804408DF8F4
:104E3000084002AA01A914480096FDF7A7FF9DF8B3
:104E40000800E8708DF804408DF80840012302AA9C
:104E500001A90D480096FDF799FF9DF808002871FB
:104E6000022005F0B4FA012211033846FCF744FD94
:104E7000A878E978000440EA0120297903B00843C2
:104E8000F0BD000000040240840A002090000020D1
:104E900010B50F4C012211032046FCF72DFD022016
:104EA00005F095FA0022A1142046FCF725FD02200A
:104EB00005F08DFA022000F00DF80A2005F087FABF
:104EC00020460122BDE810401103FCF715BD00008B
:104ED0000004024001B582B000208DF804004FF4B8
:104EE0007A700090012301AA02A90248FDF74EFF43
:104EF00003B000BD840A00202DE9F04190461D4E0C
:104F00000D46044601221F4611033046FCF7F4FC0F
:104F1000022005F05CFA0022B1143046FCF7ECFCEC
:104F2000022005F054FA44F02000FFF7D3FF012CD3
:104F30000CBF05F07F002846FFF7CCFF4046FFF787
:104F4000C9FF3846FFF7C6FF022005F040FA0122EC
:104F500011033046FCF7D0FC012C18BFBDE8F081EE
:104F60000548817811F0400F1CBF01210170BDE898
:104F7000F0810000000402409000002038B5044693
:104F80004068B0F5827F0FD1A068B0F5004F18BF20
:104F9000B0F5806F1AD12068036823F040030360E6
:104FA0006068B0F5827F0DD00B460092002201218F
:104FB000204600F057F8E0B1606D40F020006065D9
:104FC000032038BDA068B0F5806F09D00B46009271
:104FD00000228021204600F045F80028ECD108E0AE
:104FE0000B46009200220121204600F03BF80028E9
:104FF000E2D1002038BD0000F8B515460E460B463C
:10500000009204460122022100F02CF8A0B91348B6
:1050100013490068B0FBF1F04FF47A7148430090F7
:105020006068B0F5827F0DD1334600228021204692
:10503000009500F017F870B1606D40F020006065D9
:105040000320F8BD009830B1401E009020688068B1
:1050500010F0800FF6D10020F8BD0000B000002055
:1050600000366E012DE9F8431F46904689460446F6
:10507000089DFCF747FC401B3D1AFCF743FC064625
:105080002A480068C0F3CB306843009020688068ED
:1050900039EA00000CBF01200020404517D0B7F1CD
:1050A000FF3F0BD0FCF72EFC801BA84212D28DB123
:1050B0000098002808BF0025401E009020688068E6
:1050C00039EA00000CBF012000204045E7D1002054
:1050D000BDE8F8832068416821F0E0014160606824
:1050E000B0F5827F0BD1A068B0F5004F18BFB0F5C6
:1050F000806F04D12068016821F040010160A06A3E
:10510000B0F5005F09D12068016821F40051016009
:105110002068016841F400510160012084F85100C9
:10512000002084F850000320BDE8F883B000002080
:105130004FF4FA7025F014FCFAE7000010B5502087
:1051400080F31188BFF34F8FBFF36F8F2EF0DEF91E
:1051500018B104494FF080500860002080F3118896
:1051600010BD000004ED00E010B592B000200290E8
:105170000390049005900C900D900E900F9010905D
:105180001C48016841F080510160006800F08050C7
:1051900011901948016841F48041016000680224BF
:1051A00000F48040119001200090000401908001E3
:1051B000CDE906400A2008904FF49670CDE9090425
:1051C00004200B906846FDF75FF908B172B6FEE760
:1051D0000F20CDE90C0480200E9040010F9010901C
:1051E00002210CA8FDF724F8002804BF12B010BD5E
:1051F00072B6FEE740380240007000400248016885
:1052000041F470010160704788ED00E00148FEF74D
:1052100060BB0000340B00200148FEF75ABB0000C1
:105220007C0B002010B50448FBF7F7FEBDE81040EA
:105230000248FEF74EBB0000C4090020C40B00204A
:105240000148FEF746BB000038130020F0B40268A6
:10525000334BDFF8D0C0344D344E354C984218BF34
:10526000B0F1804F07D0604518BFA84203D0B042CC
:1052700018BFA04204D14F6822F0700247EA020230
:10528000984218BFB0F1804F25D0604518BFA842A2
:1052900021D0B04218BFA0421DD0A0F1804CBCF577
:1052A000A03C1CBFA0F1804CBCF5A23C13D0A0F1E7
:1052B000804CBCF5A43C1CBFA0F1804CBCF5C05C8C
:1052C00009D0A0F1804CBCF5E05C1CBFA0F1804C83
:1052D000BCF5005C05D1D1F80CC022F440724CEA58
:1052E0000202D1F814C022F0800242EA0C020260ED
:1052F0008A68C2620A688262984212BFA042096943
:1053000001634FF001014161016911F0010F04BF18
:10531000F0BC7047016921F001010161F0BC7047E8
:10532000000001400004004000080040000C004064
:105330000004014001F01F010123D0F820C08B4080
:105340002CEA03030362036A02FA01F119430162C2
:10535000704701F00F010423D0F820C08B402CEAE5
:1053600003030362036A02FA01F119430162704701
:1053700070B4026A036A23F0010303624368D0F841
:1053800018C00C682CF0730C44EA0C0C8C6822F0EA
:1053900002022243104C114DA04218BFA84206D170
:1053A000CE6822F0080246EA020222F00402A0427D
:1053B00018BFA84207D14C6923F4407344EA0303A1
:1053C0008C6944EA03034360C0F818C0496841632C
:1053D000026270BC70470000000001400004014000
:1053E00070B4026A036A23F0100303624368D0F8C2
:1053F00018C00C682CF4E64C4CEA042C8C6822F0A3
:10540000200242EA0412104C104DA04218BFA842DC
:1054100006D1CE6822F0800242EA061222F0400253
:10542000A04218BFA84207D14C6923F4406343EA65
:1054300084038C6943EA84034360C0F818C0496858
:105440008163026270BC70470000014000040140AB
:1054500030B4046AD0F820C02CF0010CC0F820C091
:10546000D0F818C0A0F18045B5F5803518BFB0F16F
:10547000804F1FD0A0F18045B5F580651CBFA0F11D
:105480008045B5F5006515D0A0F18045B5F54065BE
:105490001CBFA0F18045B5F582350BD0A0F1804549
:1054A000B5F5A0351EBFA0F18045B5F5C0554CF04F
:1054B000010203D12CF0030C4CEA02024FF0F00C75
:1054C00022F0F0020CEA03131A4324F00A0301F05D
:1054D0000A0119438261016230BC704710B5806BCC
:1054E0000021C185C184FEF7C5FB10BD01680C31E8
:1054F00051E8002F22F4907241E80023002BF5D1EF
:105500000168143151E8002F22F0010241E8002324
:10551000002BF5D1016B012909D101680C3151E84B
:10552000002F22F0100241E80023002BF5D12021AA
:1055300080F8421000210163704708B590F84210CE
:1055400022291CBF022008BD8168B1F5805F04BF1D
:105550000269002A19D0826AB1F5805F1ED0002945
:1055600004BF0169002919D00168496801F07F0171
:105570001170816A01F101018162C18DA1F1010106
:105580000904090CC1850CD026E00268816A5268C2
:10559000C2F308020A80816A891CEDE70168496844
:1055A000E6E70168CA6822F02002CA600168CA689A
:1055B00022F48072CA6001684A6922F001024A61DD
:1055C000202180F8421000214163026B012A08BFAC
:1055D000016303D0FEF798FD002008BD01680C317F
:1055E00051E8002F22F0100241E80023002BF5D1F2
:1055F00001680A6812F0100F02D00A684968009129
:10560000818DFEF736FBE7E72DE9F041044600689F
:105610000169E26821F44051114301612169A068E8
:10562000E26908436169114301432068C26822F4BA
:10563000037222F414421143C16020684169A269D7
:1056400021F44071114341612068A0F18041B1F51E
:1056500088311CBFA0F18041B1F58A3129D0FCF717
:10566000B9FE8446E16900201927254D3226B1F59F
:10567000004F21D06068830F8200ACFB0701FAF76E
:1056800001FE0146A5FB012040097A42424301EB9D
:10569000820106EB0111A5FB0121490901F0F0028D
:1056A00002EB001001F00F01084421688860BDE89A
:1056B000F081FCF79FFED4E761684A1840EB0003D5
:1056C000ACFB0701FAF7DEFD0346A5FB0310410919
:1056D00018460A016FF01803594300EB810006EBEE
:1056E000C000A5FB0010400900F0F80102EB4101E9
:1056F00000F00700084421688860BDE8F0810000E0
:105700001F85EB512DE9F84304460068089E984632
:10571000006817460D4631EA00000CBF012000204A
:10572000B84256D1B6F1FF3F4AD0FCF7EBF8A0EBF8
:105730000800B0422CD85EB32068C16811F0040F95
:1057400018BF802D3CD0402D1CBF016811F0080F00
:1057500036D001684FF0000240680090206800F1E8
:105760000C0050E8001F21F4907140E80013002B5A
:10577000F4D1206800F1140050E8001F21F001016D
:1057800040E80013002BF4D1206B01280DD102E07A
:105790000320BDE8F88320680C3050E8001F21F09A
:1057A000100140E80013002BF5D1202084F84200BE
:1057B00022630820606484F840200120BDE8F8835B
:1057C0002068006835EA00000CBF01200020B842C4
:1057D000A8D00020BDE8F88310B50448FEF74CFAC5
:1057E000BDE81040014825F07FBB000018120020E2
:1057F00010B50448FEF740FABDE81040014825F016
:1058000073BB0000601200200148FEF735BA0000AB
:10581000A812002010B50448FEF72EFABDE810408B
:10582000014825F061BB0000F0120020FEE70000F7
:105830000FB4084B10B504A902AA039801F0EEFEBC
:10584000044602A9002002F06CFA204610BC5DF864
:1058500014FB0000237D000837B514460846064BAC
:105860006A46214601F0DAFE04466946002002F04D
:1058700058FA20463EBD0000237D00080A684B68A8
:1058800002604360704700B52DED048BB0EE409A86
:10589000F0EE609A83B051EC190BFAF7F4FF41EC8B
:1058A000180B18EE100A18EE901A8DED008B0028D8
:1058B00018BF0120084320F00040C0F17F6000F1D4
:1058C000E040C00F14D019EE101A19EE900A8DEDB9
:1058D000009B002918BF0121084320F00040C0F1BF
:1058E0007F6000F1E040C00F04BF012000F018F815
:1058F000B0EE480A03B0F0EE680ABDEC048B00BDC0
:1059000002E008C8121F08C1002AFAD17047704788
:10591000002001E001C1121F002AFBD170470000E6
:105920000149086070470000D00500202DE9FF5FA5
:1059300082B00021DDE90430020DDDF840B0034300
:1059400018D044F61050A2F2FF32424315141198B9
:1059500001281FD0A5EB0B00401C5FEA000A4FF0A6
:1059600000064E4FDFF83891B046504615D5CAF1C3
:10597000000413E0119801244AA3012801D16FEA21
:105980000B010298119AC0E90031C0E9024206B049
:10599000BDE8F09FCBF10000DFE704460021404A5C
:1059A000491842EB0450CDE9001012E0E00707D09F
:1059B00032463B4640464946FAF77AFD80468946DC
:1059C00032463B4610461946FAF772FD06460F4628
:1059D0006410002CEAD1DDE90401DDE90023BAF10D
:1059E000000F06DAFAF764FD42464B46FAF760FD0F
:1059F00005E0FAF7CFFD42464B46FAF7CBFD0446E9
:105A00000E460022284BFAF7A7FF03D84FF0FF30CD
:105A1000014607E00022254B20463146FAF7A1FC5B
:105A2000FAF782FF102409E0002C0ADB0A22002387
:105A3000FAF728FC039B30321A55641E50EA010223
:105A4000F2D1641C039AC4F111031444119A012A7F
:105A500003D0012208430DD10AE0084304D00020FE
:105A60004FF0110B119072E7A3EB0B056D1E0DE0CB
:105A70005B4504DD4FF0000205F1010504E003DAA7
:105A80004FF00002A5F10105002AECD0029811990F
:105A9000C0E90231C0E9004579E700000000144088
:105AA0000000F03F300000000000F0430000E03F45
:105AB00010B54421074800F085FF00220F21064859
:105AC00023F0B0FA054CA06002F0F4FC0020207036
:105AD00010BD00006C9B0020E184000854020020EF
:105AE0002DE9F04F80460C46B1F90000B2F90410E0
:105AF00083B0154688427CDCB4F90400B5F9001087
:105B0000814276DCB4F90200B5F90610884270DCF7
:105B1000B4F90600B5F9021081426ADC0022294678
:105B2000204600F0C9F800281EBF002003B0BDE8E1
:105B3000F08F0026A088B4F90010E288401A0FFA0E
:105B400080FA60886B88121A181A00B212B2002804
:105B500012DDADF800106188ADF80210A188ADF833
:105B60000410618801260844ADF80600DDE9000153
:105B7000C8F80000C8F80410B5F906106088081AC3
:105B8000101A00B20028C4BFB4F906208A4213DDFF
:105B90002188ADF80010E988ADF80210A188ADF8B1
:105BA0000410E9880844ADF80600DDE9001208EBAE
:105BB000C600761C01604260B5F90270B4F90200BB
:105BC0008742D8BF0746B5F90600B4F906108842E7
:105BD000A8BF0846C01B0FFA80F92888B4F9001046
:105BE000EB46401A00B20028C8BFB9F1000F13DD20
:105BF00000E030E0ADF80010ADF8027021880844F4
:105C0000ADF8040007EB0900ADF8060008EBC6008C
:105C10005946761CFFF732FEB5F904102088081AA1
:105C2000AAEB000000B2002811DDADF80010ADF8BD
:105C30000270A9880844ADF8040007EB0900ADF82C
:105C4000060008EBC6005946761CFFF717FE03B0A6
:105C50003046BDE8F08F03B04FF0FF30BDE8F08F65
:105C600030B4B1F90030B2F900C06345D8BF634623
:105C70000380B1F902C0B2F90240A445D8BFA446DE
:105C8000A0F802C0B1F90440B2F90450AC42A8BF78
:105C90002C468480B1F90610B2F906209142A8BFC3
:105CA0001146C1800120A34203DC6145A4BF30BC82
:105CB0007047002030BC7047F8B50D460446B0F977
:105CC0000000B1F90010164688424BDBB4F902100F
:105CD000B5F90220914245DBB4F90410B5F904206E
:105CE0008A423FDBB4F90610B5F906208A4239DB57
:105CF000B6B3ADF800006088ADF8020032466946E0
:105D0000284600F09DF8002808BFF8BDA088ADF82F
:105D100000006088ADF8020032466946284600F06F
:105D20008FF8002808BFF8BD2088ADF80000E08893
:105D3000ADF8020032466946284600F081F8002896
:105D400008BFF8BDA088ADF80000E088ADF80200FB
:105D500032466946284600F073F8002808BFF8BDAF
:105D60000120F8BD0020F8BDB0F90020B1F90430E1
:105D70009A4213DCB0F90420B1F9003093420DDCF3
:105D8000B0F90220B1F906309A4207DCB0F90600FA
:105D9000B1F902108842A4BF01207047002070476B
:105DA000F8B50D460446B0F90400B1F900101646E6
:105DB000884243DBB4F90600B5F9021088423DDBA6
:105DC000B4F90000B5F90410814237DBB4F90210D0
:105DD000B5F906208A4231DB76B3ADF80000608861
:105DE000ADF8020032466946284600F029F818BB93
:105DF000A088ADF800006088ADF802003246694620
:105E0000284600F01DF8B8B92088ADF80000E088F9
:105E1000ADF8020032466946284600F011F858B93C
:105E2000A088ADF80000E088ADF80200324669466F
:105E3000284600F005F808B10020F8BD0120F8BDA3
:105E400070B50E46B1F90010B0F9003082B01446BA
:105E500005469942A4BFB5F90400884241DBB6F972
:105E60000220B5F902108A42A4BFB5F906C09445D4
:105E700037DB002C72DDC01A401C00B200EBD07082
:105E80004210ACEB0100401C00B200EBD07040109F
:105E90009042C8BF10468442C8BF0446ADF80030E7
:105EA000288800222044ADF804006888ADF802007C
:105EB000688831462044ADF806006846FFF7C0FF09
:105EC00090B1BDF8040031462044ADF80400BDF89F
:105ED00006002044ADF8060068461FF033F902B012
:105EE00070BD02B0002070BDE8880022001BADF834
:105EF0000200E888ADF8060031466846FFF7A0FFCB
:105F000078B1BDF8040031462044ADF80400BDF876
:105F10000200001BADF8020068461FF013F902B042
:105F200070BDA8880022001BADF80000A888ADF85D
:105F3000040031466846FFF783FF80B1BDF80000DA
:105F40003146001BADF80000BDF80200001BADF8A3
:105F5000020068461FF0F6F802B070BD1CE06888C9
:105F6000ADF80200688800222044ADF806003146F2
:105F70006846FFF765FF78B1BDF800003146001BA9
:105F8000ADF80000BDF806002044ADF806006846F4
:105F90001FF0D8F802B070BD02B0012070BDB1F999
:105FA0000030B2F900C06345A8BF63460380B1F971
:105FB0000230B2F902C06345A8BF63464380B1F91D
:105FC0000430B2F904C06345D8BF63468380B1F999
:105FD0000610B2F906209142D8BF1146C180704721
:105FE0002DE9F04F91B0044622F0B8FF4FF0000BBE
:105FF000DFF88885CDF840B00C90002C14BFE06825
:1060000011F07AF9C8F8040000691EF04BFFD8F8C7
:1060100004004069002818BF1EF044FFD8F80400AF
:10602000C0691EF03FFFD8F80400006A1EF03AFF76
:10603000D8F804000169002902BFA0F850B111B0DE
:10604000BDE8F08F0025B0F85001002888BF4FF060
:10605000010961D9D8F80400411991F830110029DB
:1060600053D1B0F85001002400284ED9D8F80400CC
:10607000011991F83011002940D1A5423ED000EB22
:10608000C40100EBC50030303031FFF76DFEA8B31E
:10609000D8F8040000EBC40101F1300200EBC500A8
:1060A00000F130016846FFF77AFF68460EF0DBFA30
:1060B0000646D8F8040000EBC50030300EF0D3FAE5
:1060C0000746D8F8040000EBC40030300EF0CBFADD
:1060D0003844864212D2D8F80410BDF8002001EBF3
:1060E000C5000286BDF802204286BDF804208286E3
:1060F000BDF80620C286081980F83091D8F804004F
:10610000641CB0F85001A042B0D8D8F804006D1C4F
:10611000B0F85001A8429DD8D8F8040001680A7C64
:1061200012F0010F7DD0C9684968002979D000F5C7
:10613000AC7000F0B8FC002873D1D8F804000168F6
:10614000C9688B680D930A68934208BF4A680F922A
:1061500011F0EAF8CDE9030BCDF814B0CDF818B082
:10616000CDF81CB0CDF820B0CDF824B0CDF828B0D3
:10617000CDF82CB0D8F804000026B0F85001002863
:1061800088BF0DF1100949D9D8F80400811991F898
:106190003011E1BB00F5AC7000F0F5FB070036D024
:1061A000D8F80400394600F5AC7000F000FC8246D7
:1061B000D8F80400394600EBC60000F1300204A80C
:1061C000FFF78EFC0546B0F1FF3F1DD00024002DE7
:1061D00010DDD8F80400394600F5AC7000F019FC69
:1061E00009EBC4010A68496802604160601C44B25E
:1061F000A542EEDCD8F80400394600F5AC7000F09A
:106200005DFC384619F092FB5FEA0A07C8D1D8F85E
:106210000400761CB0F85001B042B5D8D8F804009C
:1062200000E023E000F5AC7000F0ADFB040017D0F7
:1062300003980F99CDE900100294D8F80400234682
:10624000039A00680D99C06BD0F838C0E047D8F8C1
:106250000400214600F5AC7000F0A9FB0400E7D172
:10626000D8F8040000F5AC7000F078FB25F086FB50
:10627000D8F80410B1F85001F0B309680A7C12F0A4
:10628000010F20D0C968496800291CBF00240028DC
:1062900019D9D8F80400011991F8301159B900F54D
:1062A000AC7000F0DFFBD8F8041001EBC4010A6BFE
:1062B000496B02604160601C84B2D8F80400B0F8F9
:1062C0005001A042E5D8D8F804004FF48071303076
:1062D00019F0D4FCD8F80400202100F5987019F0CA
:1062E000CDFCD8F80400A0F850B10C9822F028FE9C
:1062F0001090D8F8040000E006E00068436A1BB183
:10630000D8F800201099984719F056FA00F088F94B
:1063100000F058F9DFF868921F263F27D9F814508B
:10632000002D57D110F0E8FF11F012F818F052F8D4
:10633000054600227F211EF08AFCBDF800000022E5
:106340006BF3040080B26BF34A1080B26BF3CF2082
:10635000ADF8000080B20090BDF8001028461EF095
:1063600065FCBDF80000002266F3040080B267F30C
:106370004A1080B266F3CF20ADF8000080B20090E2
:10638000BDF8001028461EF0DEFC0022032128463E
:106390001EF0C5FC0022032128461EF0B1FC00229D
:1063A000032128461EF0B1FC0022032128461EF0DE
:1063B000B1FC0022032128461EF0C0FC71A1284632
:1063C00018F000FF00231A46062128461AF0E9F9C2
:1063D000C9F81450D9F8000022F0B2FDB0F5967F4C
:1063E00011D2D8F8000041F28831814248D2D9F860
:1063F000040010990844C9F80400D9F80800401CAA
:10640000C9F808003CE022F0A9FDC9F80000D8F85E
:106410000400406800281DBF00684FF47A71B1FB8A
:10642000F0F14221D9F80400002804BF0120C9F886
:106430000400D9F80800002808BF0C4606D04FF425
:106440007A725043D9F80420B0FBF2F4C9F804B0D2
:10645000C9F808B08C4288BF0C46D9F81000204417
:10646000C9F81000D9F80C00401CC9F80C0022F043
:10647000F9FDC0F16403224643A1284618F0DDFE71
:10648000454D6C68F4BB10F037FF10F061FF17F05A
:10649000A1FF044600227F211EF0D9FBBDF80000B9
:1064A00000226BF3040080B26BF34A1080B26BF3EE
:1064B000CF20ADF8000080B20090BDF8001020465B
:1064C0001EF0B4FBBDF80000002266F3040080B2A9
:1064D00067F34A1080B266F3CF20ADF8000080B2B7
:1064E0000090BDF8001020461EF02DFC0022032174
:1064F00020461EF014FC0022032120461EF000FC62
:10650000002200E013E0032120461EF0FEFB0022E3
:10651000032120461EF0FEFB1AA1204618F052FE71
:1065200000231A46042120461AF03BF96C602868C3
:1065300022F006FDB0F5967F9CBF11B0BDE8F08F4C
:1065400022F00CFD286002A819F012FA04990298B2
:10655000401A820A514200EB81201049A1FB001031
:1065600083099DF821109DF82000CDE900010CA1C0
:10657000204618F062FE11B0BDE8F08F60010020E7
:10658000D49400203F0000002575204650530A2572
:10659000752525204350550068010020A1A0A0A02A
:1065A00025752E2575206B4220757365642028257E
:1065B00064202525290A2564252520667261672E19
:1065C0000000000070B50A4E0024C4EBC40556F864
:1065D0002500002818BF19F0A9F906EB85001C2139
:1065E00019F04CFB601CC4B2042CEED370BD00004B
:1065F000489C002009494968002908BF70474A683B
:1066000082421CBF0A68824203D10A7E42F0010224
:106610000A7649690029F2D1704700003401002050
:10662000704700000421014800F0CCB9609B0020B5
:106630002021014800F0C6B9789B00202DE9F041E7
:1066400084B00446DDE90A571E004FF0000008BF81
:10665000B5F5807F3DD0039001900290ADF80C100D
:106660000090ADF80410ADF80A20ADF80E203B46BE
:106670002A46314668461EF0B9FC3B462A4631465A
:10668000E84601A81EF0B2FC3B462A46314608F116
:1066900008001EF0ABFC3B462A46314608F10C00D0
:1066A0001EF0A4FCBDF90030BDF904209342B4BF34
:1066B0009C469446BDF90810BDF90C008142B4BF58
:1066C0000D460546AC450ADA9342ACBF1046184663
:1066D00008E020806080481EA080501E57E088425D
:1066E000C8BF0846801E2080BDF90030BDF90410E7
:1066F0008B42CCBF9C468C46BDF90820BDF90C00EE
:106700008242CCBF15460546AC4504DD8B42D4BF62
:106710000846184602E09042B8BF1046801CA08090
:10672000BDF90210BDF906008142B4BF8C46844613
:10673000BDF90A20BDF90E309A42B4BF15461D4678
:10674000AC451BDA8142B8BF0846801E6080BDF9A7
:106750000230BDF906209342CCBF9C469446BDF959
:106760000A10BDF90E008142CCBF0D460546AC456E
:1067700009DD9342D4BF1046184607E09A42B4BFE1
:1067800010461846E1E78842B8BF0846801CE08002
:1067900004B0BDE8F08100002DE9F04116460F4637
:1067A0008046124C22F0DAFB054633463A46414613
:1067B000204616F097FF20B10020A062E06950B19A
:1067C00011E02C21204619F059FA4FF00040A06248
:1067D0000020BDE8F081284622F0B2FBE0610028ED
:1067E00004BF0120E0612046BDE8F0819C9B0020B1
:1067F00010B514210A4800F0E5F8094800F0EAF85D
:1068000004000BD0142119F039FA0648206006481C
:1068100060600648A0600648E06010BDFEE700002A
:10682000849B002069CF010821D001089DD2010876
:1068300031CF010870B584B00D46040005D110F0C9
:106840005BFD040004BF04B070BD10F0CBFD002858
:1068500004BF04B070BD94F8280010F0040F1CBFF2
:1068600004B070BD0026002D02BFA4F8506104B032
:1068700070BDADF80060ADF80260204610F054FD28
:10688000401EADF80400204610F098FD401EADF803
:1068900006006A46294602A8FFF7E2F9002804BF6D
:1068A00004B070BD2068017C11F0020F0CD0DDE94E
:1068B0000001C4E90C010120A4F85001606800281F
:1068C00004BF04B070BD45E08269002A1CBF02A964
:1068D00090470025B4F85001002811D904EBC500F9
:1068E00000F13001002202A8FFF7E6F900281CBFE2
:1068F00004B070BD681C85B2B4F85001A842EDD850
:1069000080B220280ED204EBC000BDF8081001862A
:10691000BDF80A104186BDF80C108186BDF80E1036
:10692000C1860DE0A4F85061BDF800102186BDF8C5
:1069300002106186BDF80410A186BDF80610E1863C
:10694000B4F85001401CA4F850016068002804BF4E
:1069500004B070BD22F04CFC04B070BD70B50600F0
:106960000CBF00247468002C08BF70BD211D306866
:1069700045582146304600F0A1F8204618F0D6FFD1
:106980002C00F3D170BD002818BF4068704702008A
:106990004FF000000CBF00215168002914BF12689D
:1069A0007047091D401C51580029FAD170470068F2
:1069B000091D40587047006840587047002818BFAC
:1069C0008068704700224260C91C21F00301826088
:1069D0000160704738B504460068083018F0D2FEF0
:1069E000002808BF38BD002100912268031D115006
:1069F000616800912268D1506168002918BF009039
:106A000001D0226850506060A168002908BFA060D2
:106A100038BD002812BF00290020704738B5044651
:106A200040680D46A84204D12046BDE83840FFF733
:106A3000D1BF2068083018F0A5FE002808BF38BD77
:106A400021684959009011B123680A1D985000919E
:106A50002268115000902168021D4851009521685C
:106A60008D5038BD38B504460068083018F08AFEED
:106A7000002808BF38BD002100912268031DD150B5
:106A8000A168009122681150A168002918BF0090E8
:106A900003D0226801F104015050A0606168002910
:106AA00008BF606038BD30B14168002907BF806809
:106AB0000028002070474FF00100704781B0002887
:106AC00004BF01B070470022D0F804C00B1D8C45F4
:106AD0000CD10168C9584160002911BF0092826041
:106AE00001B070470068425001B07047D0F808C04C
:106AF0008C450ED1036859588160002911BF00925E
:106B0000426001B07047006801F10401425001B0D9
:106B10007047D0F800C05CF801205CF803100091C9
:106B20002AB1D0F800C002F104034CF8031000921F
:106B30000029D7D101B0704710B5044600688268BB
:106B4000002A1CBF2146904720680068002818BF13
:106B50002060F4D110BD8068002818BFB0F916007D
:106B60007047806800281CBF807E8009704770B520
:106B7000144605460E4651EA040004BF012070BDCC
:106B800028461AF017F8AB6822463146188A304476
:106B90001882AB68588A20445882012328461CF08A
:106BA0000CFC00220B21284615F040FB012818BFE1
:106BB00070BD28461CF03EFB012070BD77B581B04A
:106BC0000E46050019D062221BF05AFE04001CBFBD
:106BD0002068002811D04FF06302314628461BF090
:106BE0004FFE10F0FF0208D0236820460399984713
:106BF0000090BDF80000ADF80C00039804B070BD23
:106C00002DE9F047054692B0408C1A9C40F00800F0
:106C1000688490462A841E468946228928461BF0AD
:106C20002FFE82462E842289494628461BF028FEE4
:106C30000746688CBA4520F00800688407D14FEAFF
:106C40000A41B1EB074F04BF12B0BDE8F087A5F8C9
:106C500020802289494628461BF012FE80462E8459
:106C6000494628460BF04BF921890068424620F03E
:106C700009FD20890B2821D147F6FF7AD04518BF9E
:106C800057451BD128461BF06DFF00EBD070461016
:106C900028461AF0F2FF00EBD0704010D04505D125
:106CA000711C421C9142B4BF88469046574505D19D
:106CB000711C421C9142B4BF0F4617461848FFF79B
:106CC00089FE06002BD03560C6E903872089B08095
:106CD0006846C6F808900CF0A3FE1248FF21CDE9E3
:106CE0000060114802901148039000200890CDE9FF
:106CF000090120880B9060889DF8421040420C905A
:106D0000E0680790002060F300018DF842102069D0
:106D1000069068460CF0FAFE12B0BDE8F087FEE778
:106D2000909B0020B9210308E12303081D230308D9
:106D300014210148FFF746BE909B00202DE9F84F33
:106D40000646408C0024C0F30510174688462546A9
:106D5000002888BF4FF0040940F2ED80F06809EB8D
:106D6000C501405810F0007F40F0DE8080B230EA6C
:106D7000080114BF00230123B8430CBF01200020E9
:106D8000834200F0D180F0686A46102150F835A0A7
:106D9000504620F01DFA00286DD16A461121504658
:106DA00020F016FA002866D16A461221504620F0DB
:106DB0000FFA00285FD16A461321504620F008FAE6
:106DC000002858D16A461521504620F001FA0028C3
:106DD00051D16A461421504620F0FAF900284AD1D0
:106DE0006A460A21504620F0F3F9002843D16A464A
:106DF0006B21504620F0ECF900283CD16A466C210A
:106E0000504620F0E5F9002835D16A460121504668
:106E100020F0DEF978BB6A460421504620F0D8F90C
:106E200048BB6A460221504620F0D2F918BB6A4698
:106E30000321504620F0CCF9E8B96A4605215046B6
:106E400020F0C6F9B8B96A460621504620F0C0F9CC
:106E500088B96A463221504620F0BAF958B96A46D4
:106E60006E21504620F0B4F928B96A466D2150468B
:106E700020F0AEF910B10320BDE8F88F6A46692111
:106E8000504620F0A5F9002849D16A466A215046AB
:106E900020F09EF9F0BB6A466E21504620F098F92A
:106EA000C0BB6A466D21504620F092F990BB6A46FD
:106EB0003721504620F08CF960BB6A463821504695
:106EC00020F086F930BB6A463521504620F080F923
:106ED00000BB6A464021504620F07AF9D0B96A4694
:106EE0004521504620F074F9A0B96A464121504628
:106EF00020F06EF970B96A464221504620F068F9D8
:106F000040B96A464321504620F062F910B96A46FA
:106F1000492100E003E0504620F05AF908B102246C
:106F200002E0002C08BF0124708C6D1CC0F305101A
:106F3000A8423FF613AF2046BDE8F88F01484068ED
:106F40007047000060010020054800214160016198
:106F5000C160816001604161024801604160704729
:106F6000D494002068010020C0F30410072888BFD3
:106F700007207047A0F57F41FF390ABF1F20002876
:106F8000704771283EBF0849085C7047713880B26D
:106F90000649096829B1064A526890423CBF085C1C
:106FA0007047002070470000F87803088002002036
:106FB0009402002010B518210348FFF703FD034990
:106FC0000120087010BD00003C9B00209C020020A6
:106FD000002808BF70472DE9F04117460D460446CA
:106FE000F9F7A1F9DFF8388006462946D8F80820D5
:106FF000204690470546D8F8082060193946904742
:1070000001462846721A824238BFBDE8F081431813
:10701000E35C2354401C8242F9D2BDE8F0810000B9
:10702000B00200202DE9F041084E15460C4672686A
:107030001F46804619469047206020B13868726824
:107040004044002190472860BDE8F081B002002054
:107050002DE9FF4F8DB083461A980026002818BFEF
:107060000680BBF1000F02BF002011B0BDE8F08F19
:107070009BF80000002819BF0E98002811B0BDE849
:10708000F08F4FF0000005901B9810F0060F18BF0E
:10709000002014D01BF800100A2918BF0D2904D0B5
:1070A000002918BF401CF5D100E0401C1A990029A6
:1070B0001CBF4FF0FF320A8011B0BDE8F08F1B9863
:1070C00010F0020F1CBF41F6FF7010900496049858
:1070D0001BF8000000281CBF1098002840F3E38034
:1070E0000498002106910BEB000201920E9A0A927D
:1070F0000F9A0992109A08921B9A0DF1180907929B
:1071000000280CBF012000200B90019800281FBF11
:10711000007800280A98002808BF0F467BD012F09C
:10712000020F1CBF41F6FF7008904FF00007704A35
:1071300002970397009752683C46BA464FF0FF38D3
:1071400002A901989047054602980390019800789B
:10715000002877D0664A03A90198526890470090AA
:1071600007980AF1010A10F0010F14D00020232D16
:1071700004D0F1B201291FD068B15BE016F0FF0026
:1071800008BF012656D0012808BF002603D00228D8
:1071900008BF00264ED02946009A0A9815F0BAF981
:1071A00000B221180CB2002802DD0998204404B274
:1071B000B8F1FF3F0AD103E0202D08BF022639E0D5
:1071C0000998211A08988142C8BFB8460A2D18BFED
:1071D0000D2D18D0A5F59C4145F2A5104FF00002E9
:1071E000814210D943A10020097859B141A10B5C1B
:1071F000AB4201D1012205E0401CC0B23DA1095CB7
:107200000029F3D172B1002F08BFB8F1FF3F06D1BA
:10721000B9F1000F00E027E018BFC9F80040AAF15B
:10722000010A0FE0B9F1000F04D0B8F1FF3F08BF29
:10723000C9F80040DDE9027002900198009DC05D30
:10724000002887D1B8F1FF3F05D00B98002818BF60
:10725000474635D008E0BAF1000F04D00D2D04BF29
:1072600000980A2800D1029F10990698A1EB00010E
:1072700009B210910599084400B205909FB1049895
:1072800000EB070104919BF800000A2818BF0D28A5
:1072900009D01BF801000A2818BF0D287FF417AF8A
:1072A00001F101000490049890B11A98002818BFC9
:1072B000059801D01A990880049811B0BDE8F08FA4
:1072C000B9F1000F1CBF0020C9F800000027CBE770
:1072D000074A04A95846526890471A9A002AEBD0E8
:1072E000014600220E9815F015F900B20590E1E76D
:1072F000B0020020202C2E3B3A2D5F00002814BF46
:10730000002A70472DE9F041164688460746F9F7EE
:107310000AF804463046F9F706F8050008BFBDE84C
:10732000F0812C440D4A4146384692689047014608
:107330002844A04205D8621BBA5C3A55641EA0429C
:10734000F9D97818002D08BFBDE8F08116F8011BA7
:1073500000F8011B6D1EF9D1BDE8F081B0020020DC
:1073600000230278232902D0012A0ED013E0002A3C
:1073700008BF01210DD00021012A08BF01700AD0E9
:10738000022A04BF0170012305E0202908BF022161
:1073900000D101700123184670472DE9F0410B46DA
:1073A0000F46064602460021084622F0E7FA044648
:1073B0004FF00008401C18F0E5F9050009D005F869
:1073C00004803B463246611C22F0D8FA2846BDE8CC
:1073D000F081FEE72DE9F05F1F46DDF828801400FC
:1073E0000D46824618BF4FF0010911D0660806FB12
:1073F000075B59465046C0470028B8BF34460BDDEE
:1074000029EA0400C0EB54040BEB0705002CEDD176
:107410004FF00000BDE8F09FF8DB5846BDE8F09F54
:107420002DE9F04F83B04FF0300ADDE90C64DDE95F
:107430001058DDE90EBC129F17F0020F1ED1B8F1F3
:10744000000F18BF17F0010F06D007F00C0959EA1A
:107450000B0918BFA8F10108AC423EBF202C06F86A
:1074600004A0641CF8D317F0010F18BFA04505D97C
:10747000202C3CBF06F804A0641CF4D317F0100FB6
:1074800036D017F4806F0CD15CB1AC4218BF4445C4
:1074900007D1641E05D0BCF1100F08BF641E07D0D1
:1074A00002E0BCF1100F03D0BCF1020F13D019E0C1
:1074B00017F0200F07D0202C36D24FF0580C06F8CA
:1074C00004C0641C0EE0202C2ED24FF0780C06F87D
:1074D00004C0641C06E0202C26D24FF0620C06F893
:1074E00004C0641C202C3CBF06F804A0641C1BD202
:1074F000202C19D2BBF1000F05D04FF02D0C06F84F
:1075000004C0641C10E017F0040F05D04FF02B0CE2
:1075100006F804C0641C07E017F0080F04D04FF011
:10752000200C06F804C0641CCDE9003115468146E4
:10753000AA4617F0030F0CD1A346444509D22A46A8
:10754000DDE900316D1C2020C8470BF1010BC3455C
:10755000F5D344B12A466D1C641EDDE90031305D6F
:10756000C847002CF6D117F0020F1CBFA5EB0A008C
:10757000804509D92A46DDE900316D1C2020C84725
:10758000A5EB0A008045F5D803B02846BDE8F08F8A
:107590002DE9F04F91B00024DDE91ACADDE91E851E
:1075A000DDE91C69BCF1000F08BF25F0100515F4DA
:1075B000806F0DF1200B02D0BCF1000F1BD0BCFB83
:1075C000F6F706FB17C7FFB20A2F38BF303708D3CC
:1075D00015F0200F14BF4FF0410E4FF0610E7744AD
:1075E0000A3FBCFBF6FC0BF80470641CBCF1000FF6
:1075F00018BF202CE3D3CDF800B0CDE9014ACDE986
:107600000585CDE90369FFF70BFF11B0BDE8F08FE9
:107610009A4238BF88547047704700002DE9FF4FE9
:1076200095B09A46884606460025EEE1252877D192
:1076300000242746F94A0121039400E0044316F888
:10764000013F203B01FA03F01042F7D130782A289D
:1076500011D06FF02F033078A0F13002092A16D82C
:10766000039A44F0020402EB820203EB420210444C
:10767000761C0390EFE758F8042B0392002A03DAF4
:10768000504244F40054039044F00204761C3078D5
:107690002E2816D116F8010F44F004042A280DD024
:1076A0006FF02F023078A0F13003092B09D807EBD7
:1076B000870302EB4303C718761CF3E758F8047BF3
:1076C000761C30786C280FD006DC4C2817D0682840
:1076D0000DD06A2814D104E0742810D07A280FD174
:1076E0000DE044F400140AE044F4801401E044F492
:1076F00040147278824202D104F58014761C761C04
:10770000307866280BD013DC582877D009DC0028A5
:1077100075D04528F6D04628F4D047281AD193E1F1
:1077200018E0632835D0642879D0652812D18BE120
:10773000702873D008DC6728F1D069286FD06E28D4
:107740000DD06F2806D1ACE073282CD0752874D0EA
:10775000782853D05246179990476D1C54E1C4F3D2
:107760000250022809D003280DD0D8F800100428B0
:107770000DD00D6008F1040846E1D8F80010EA17B2
:10778000C1E90052F6E7D8F800100D80F2E70D705D
:10779000F0E718F8041B8DF8001000208DF80100A8
:1077A000EB46012003E058F804BB4FF0FF306107BF
:1077B0004FF0000102D40DE009F101018946B94200
:1077C0000FDA8145F8DB1BF809100029F4D108E035
:1077D00009F1010189468142FADB1BF809100029F1
:1077E000F6D103985346A0EB090721463846179A6D
:1077F00000F080FA284400EB090507E044E008E1C6
:107800000DE01BF8010B524617999047B9F1010999
:10781000F7D2534621463846179AF2E039E00A215A
:10782000C4F302524FF0000B0091022A06D058F820
:10783000040BC117032A09D00AE023E008F107006E
:1078400020F00702F2E80201904605E000B2C117FD
:10785000042A01D140B2C117002906DA0A460021E4
:10786000404261EB02012D2202E0220504D52B22C9
:107870008DF80420012203E0E20701D02022F7E77F
:10788000914657E00A2100E010214FF0000B0091D3
:107890000BE010214FF0000B44F004040827009186
:1078A00003E008204FF0000B0090C4F30252022ABC
:1078B00005D058F8040B0021032A08D008E008F18D
:1078C000070020F00702F2E80201904603E080B2D0
:1078D000042A00D1C0B24FF0000922072AD532781D
:1078E000702A07D0DDF800C08CF0100C5CEA0B0C9D
:1078F00005D00EE040228DF80420012208E050EA75
:10790000010306D030238DF804308DF805200222C3
:107910009146009B83F0080353EA0B030AD150EA17
:10792000010201D1620705D530228DF804204FF005
:1079300001097F1E3278582A04D039A20C920CAA71
:1079400002920BE03BA2F9E75B46009AF8F79AFC3B
:107950000C9B9B5C029A521E0292137050EA010229
:10796000F2D1029804A9081A00F1200B600702D591
:1079700024F4803400E001275F4502DDA7EB0B0013
:1079800000E0002000EB0B01009003984944401AEE
:107990000390E00306D453462146179A039800F05B
:1079A000A9F90544002706E001A85246C05D1799D1
:1079B00090476D1C7F1C4F45F6DBE0030CD553460A
:1079C0002146179A039800F095F9054404E0302009
:1079D0005246179990476D1C0099481E0090002947
:1079E000F5DC08E00298029952460078491C0291A1
:1079F000179990476D1CBBF10001ABF1010BF1DC55
:107A00005BE100F065F90544761C307800287FF4CE
:107A10000DAE19B02846BDE8F08F0000092801001E
:107A200030313233343536373839616263646566F4
:107A300000000000303132333435363738394142B6
:107A40004344454600000000600700D4062708F1C3
:107A5000070020F00700F0E80223804603F0004C06
:107A60005FEA0C0001D097A009E0200501D596A09F
:107A700005E0E00701D095A001E0AFF24C001390C3
:107A8000307823F0004365280CD006DC452809D067
:107A900046281DD047287FD13BE0662818D06728AC
:107AA0007AD136E00021112F01DB112000E0781C93
:107AB000CDE9000104A90CA8FDF738FFDDE90D01AF
:107AC0000C9A4FF0000B07F10109109200914EE063
:107AD0004FF000400097CDE9011004A90CA8FDF774
:107AE00025FFDDE90D020C9B0F994FF0000B91462D
:107AF0001093009211B9791C00EB0109B7EB090052
:107B000003D4C0F1FF3B07F10109A9EB0700019085
:107B100042E0012F00DA01270021112F01DD1120A1
:107B200000E03846CDE9000104A90CA8FDF7FEFEEF
:107B3000DDE90D010C9A00914FF0000BB94610924F
:107B400021070FD4009A4A4503DA914601E0A9F1D2
:107B50000109B9F1010F05DD109AA9F10101515C8C
:107B60003029F4D0B84202DA10F1040F03DA01210F
:107B7000CDE9011010E0002803DC8344A9EB0001EB
:107B800002E0411C494500DD8946A0EB0B00401C8A
:107B900001904FF000400290200705D4019848451D
:107BA00002DB4FF0FF30019000208DF84B0002986F
:107BB0000DF14B07B0F1004F25D002200C902B2087
:107BC0000D90029800280CDA404202902D200D9072
:107BD00007E00A210298F8F77BFD3031029007F8A0
:107BE000011D0C99481E0C900029F2DC0298002817
:107BF000EFD1791E0D980870307800F0200040F029
:107C0000450007F8020D11A8C01BC01D0290139873
:107C1000007800B1012000EB0901019801EBE0714F
:107C2000029801440398401A401E0390E00306D4D2
:107C300053462146179A039800F05CF805441398C0
:107C4000007818B15246179990476D1CE00323D570
:107C500053462146179A039800F04CF805441BE060
:107C6000BBF1000F07DB0098584504DD1098179909
:107C700010F80B0001E01799302052469047019808
:107C80000BF1010B401E05F10105019004D12E20DE
:107C90005246179990476D1CB9F10001A9F10109ED
:107CA000DEDC05E017F8010B5246179990476D1C72
:107CB0000299481E02900029F4DC53462146179A87
:107CC00003989EE62D0000002B000000200000001D
:107CD0002DE9F041044600251E461746880404D4C9
:107CE00005E039462020B0476D1C641EF9D52846B2
:107CF000BDE8F0812DE9F041044600251E4690467E
:107D0000C80301D5302700E02027880404D505E00A
:107D100041463846B0476D1C641EF9D52846BDE87B
:107D2000F0810A68531C0B60107070472DE9FF4FFB
:107D300099B080461A98269E1C464FF0000A0028EB
:107D400008BFDFF870852078002871D0C0B22528E0
:107D500008BF00256DD134E00ADC202808BF45F0BB
:107D600008052ED0232808BF45F0100529D009E0CA
:107D70002D2808BF45F0020523D0302808BF45F064
:107D800001051ED0C0B20027A0F1300109299CBF17
:107D900000276FF02F0102D92A281AD00BE02046C5
:107DA00007EB8702007801EB4202871814F8010FF5
:107DB00030380928F3D920784FF000092E2811D047
:107DC0002DE014F8010F2B2808BF45F00405F8D06A
:107DD000C2E756F8047B002FBCBF45F002057F4286
:107DE000641CE8E714F8010F45F48065A0F1300148
:107DF00009299CBF4FF000096FF02F0102D92A28F2
:107E000018D00CE0204609EB8902007801EB420211
:107E100000EB020914F8010F30380928F2D9207854
:107E20006C281BD00FDC682830D06A281CD01EE0DC
:107E300046E03AE056F8049BB9F1000FD8BF4FF086
:107E40000009641CEBE7742808BF45F480750DD069
:107E50007A2804BF45F48075641C08E014F8010F0B
:107E600045F480756C2802D145F40075641C2078B7
:107E700069283FD031DC62283CD011DC252800F095
:107E80000F82502818BF582834D00EE014F8010F84
:107E900045F08005682808BF45F04005E7D1E5E7D3
:107EA000632800F07A81642824D0DDE91A13524651
:107EB0000AF1010AC047641C207800287FF446AF0D
:107EC0001B98824534BF5246421E034600201A9931
:107ED000C0471DB05046BDE8F08F732800F08D817B
:107EE00004DC6F2818BF7028DFD103E0752818BFA5
:107EF0007828DAD1782814BF58284FF0100B1BD0FF
:107F0000702818BF50280ED06F2808BF4FF0080BFC
:107F10001FD062280EBF4FF0020B4FF00A0B25F066
:107F2000100516D010E060784FF0100B45F48875FE
:107F3000562808BF641C02D12078582802D0207827
:107F4000502801D145F02005C0B2692818BF642827
:107F500001D025F00C0515F4806F18BF25F0010540
:107F60002078692818BF64284CD056287ED015F494
:107F7000007F7CD01A98CDE908A01B980790F01DCF
:107F800020F0070202F10806D2E900010022009267
:107F90009246019250EA010208BF25F0100515F43F
:107FA000806F02D050EA01021CD05A46019BF8F7BC
:107FB00069F90346D0B20A2838BF303006D315F02D
:107FC000200F14BF4122612210440A3810AA02F87F
:107FD0000A0018460AF1010A53EA010202D0BAF176
:107FE000200FE2D3CDE90575CDE903B910A90098BA
:107FF0000091CDE901A0DDE908214046079BFFF78C
:108000000FFABEE015F4007F58D0F01D20F00701F4
:1080100001F10806D1E900021A99CDE910A11B99D6
:10802000079100210B46091A73EB0201B8BF1146F4
:1080300003DB0021404261EB0201002AB4BF0122B0
:108040000022009200229246019250EA010208BFEB
:1080500025F0100515F4806F02D050EA01021FD000
:108060005A46019BF8F70EF9034601E053E063E03E
:10807000D0B20A2838BF303006D315F0200F14BF15
:108080004122612210440A3808AA02F80A00184660
:108090000AF1010A53EA010202D0BAF1200FDFD33C
:1080A000CDE90575CDE903B908A900980091CDE99E
:1080B00001A0DDE910214046079BA0E715F4807F71
:1080C00012D056F8040BCDE90475CDE902B9C10F01
:1080D000002815DDCDE90001DDE91A1352464046BE
:1080E000FFF756FA82464DE015F0400F0AD016F819
:1080F000040BCDE90475CDE902B9C10F0028E9DC14
:108100004042E7E715F0800F1ABF36F8040B00B2C3
:1081100056F8040BEDE756F8040B41680968009126
:1081200003681B98A0EB0A021A9800EB0A0140466C
:10813000FFF7FCFD824425E015F4807F0FD0CDE9E8
:108140000475CDE902B9002156F8040BCDE9000110
:10815000DDE91A1352464046FFF71AFA11E015F00E
:10816000400F11D016F8040B0021CDE90001CDE934
:1081700002B9CDE90475DDE91A1352464046FFF70E
:1081800007FA8246641C97E615F0800F1ABF36F88E
:10819000040B80B256F8040BE6E74FF0010915F026
:1081A000020F0FD14FF00209012F0BD9DDE91A138D
:1081B00052460AF1010A2020C047484609F1010948
:1081C0008742F3D8DDE91A13524616F8040B0AF178
:1081D000010AC04715F0020F1CBF09F101054F4508
:1081E000D0D9DDE91A1352460AF1010A2020C0470E
:1081F00028466D1C8742F4D8C4E756F8042B009239
:10820000B9F1000F14BF49464FF0FF311046037813
:108210001BB1491E40F10000F9D2A0EB020B15F48E
:10822000806F02D0D94598BFCB4615F0020F1AD106
:1082300058460BF1010BB84215D2DDE91A1352462C
:108240000AF1010A2020C04758460BF1010BB84241
:10825000F3D308E000995246491C0091DDE91A1356
:108260000AF1010AC0470098007828B115F4806F20
:10827000F0D0B9F10109EDD215F0020F1CBF0BF1DE
:1082800001055F457FF67EAFDDE91A1352460AF11C
:10829000010A2020C04728466D1C8742F4D871E7A8
:1082A000DDE91A1352460AF1010A2520C047641C71
:1082B00002E60000197600082DE9F04F05467448E3
:1082C0000C462DED028B00260178DFF8C8B187B08F
:1082D000012729BB0770704870490670704801601B
:1082E0004FF48271C0E90116C66079020661C0E9E7
:1082F00005711021C0E907160A214662C0E90A612A
:10830000FAF7D0FA002818BFF8F7D0FB0022202196
:108310005846F9F7F1FA012202216248F9F7ECFA1E
:10832000002220215846F9F7E7FA0A202AF0F8FA45
:1083300006214FF47A704FF040084FF008096FF0B3
:108340007F4AB0EE048ADFED588A022D02D0092D53
:1083500045D08FE08DF804100546009001A9534ADE
:1083600001234F48FAF712FD05202AF0D9FACDE98A
:108370000468069600220396CDE900672023114683
:10838000A020029625F0D2F805202AF0C9FA8DF82F
:10839000049001A9454A3B4641480095FAF7F6FC8E
:1083A0001E202AF0BDFA42A001A9006802AACDE968
:1083B0000050032302963A48FAF7E8FC9DF80800BB
:1083C0009DF80910000400EB01209DF80A100844F4
:1083D00010F4000F44D080EA0A00401C40E08DF801
:1083E00004100546009001A9304A01232C48FAF7F1
:1083F000CDFC05202AF094FACDE904680022069607
:108400000396CDE90067202311461046029625F019
:108410008DF805202AF084FA8DF8049001A9234AEA
:108420003B461F480095FAF7B1FC1E202AF078FA67
:108430001FA001A9006802AACDE9005003230296FB
:108440001748FAF7A3FC9DF808009DF809100004EE
:1084500000EB01209DF80A10084410F4000FBAD177
:1084600000EE100AB8EEC00A20EE080A20EE280A34
:1084700084ED000A012220215846F9F73DFA07B0A1
:108480000520BDEC028BBDE8F04F2AF049BA000090
:1084900084000020001002408F00002000300140C6
:1084A0002C0A002000080240000000348500002053
:1084B000FFFFFF0010B5084C012020700748FEF7B1
:1084C00062FA0028A06803D0BDE8104020F090BEFA
:1084D000BDE8104020F080BE540200206C9B0020BC
:1084E0002DE9F0475B4E706820F02AFD0546707854
:1084F00080F0010070705848FEF745FA040078D00B
:1085000000274FF6FF784FF00109377094F84200CA
:108510007178C0F380028A426CD061F3820084F8E3
:108520004200216B4A1910F0080F1BD1002919DCF9
:10853000002A17DB10F0010F09D1616939B120461B
:108540008847216A01442162A16A0844A062A168A7
:1085500000291CBF2046884794F8420040F00800DC
:1085600084F84200206B4019206361D4E16A88429C
:10857000C8BF21632046E16988470146606A884296
:1085800005D061626268002A1CBF20689047D4E968
:108590000B0181424CDB94F8420010F0020F03D033
:1085A000B4F8400050B126E0B4F8400030B1404586
:1085B0001CBF401EA4F840001DD0F1E7A06B20B105
:1085C00094F8420010F0020F15D021462248FEF721
:1085D00075FAFFF76FFFE1682046002918BF88474A
:1085E00020462169002918BF8847204617F09EF9C8
:1085F0001EE02AE022E0E06B41422163A06BB8B1AB
:1086000094F8420010F0020F02D1606B41422163E6
:1086100094F8420029EA500161F3410084F84200D5
:10862000A26A206A2262A062A26BE06AE262A06390
:10863000307818B10848FEF7A6F903E0214606484D
:10864000FEF7B5F904007FF460AF20F087FC70609E
:10865000BDE8F087540200206C9B002070B50446F2
:1086600040680D46002818BFFFF7F8FF2268002A6F
:1086700008BF70BD29462046BDE87040104789B24A
:108680000BF04FBF89B20BF08EBF000010B5818F89
:1086900092B00446A9B168460BF0C2F90B4801211B
:1086A000CDE90040A08F0B9000200890CDE9090192
:1086B000074807900748039068460BF027FA12B066
:1086C00010BD12B0BDE8104022F0AABED9B4020815
:1086D000E53A0108DBB402082AF013B830B50546C4
:1086E00083B048680C4620F0030001AA694621F0D7
:1086F0007DFCDDE9001205EBC11000EB8203D86BB5
:1087000060B164B1C4E90205C46004F10B0C04F16A
:1087100008002CF0030C604502D0FEE7FEE7FEE700
:10872000DC630123286903FA01FC40EA0C0028619C
:1087300005EB810003FA02F241691143416103B084
:1087400030BDF0B583B04FF0000704460E0001972E
:108750003D4600974DD0084601AB6A46802909D3B3
:10876000B0FA80F1C1F11A014FF0010C0CFA01F1DD
:10877000491E0844194621F039FC01980A2838DAC4
:1087800004EB8002009953694FF0FF3202FA01F1C5
:10879000194013D1401C216902FA00F0084008BFBB
:1087A0003D4618D0C143491C0840B0FA80F0C0F1E2
:1087B0001F0004EB80010190496999B1CA43521C22
:1087C0001140B1FA81F1C1F11F0104EBC01000EBBF
:1087D00081000091C56B65B1686820F00300B0426C
:1087E00001D2FEE7FEE7DDE900322946204623F00C
:1087F0007BFD03B02846F0BD70B5064682B00D463D
:10880000084600F02BF8040025D0606810F0010F36
:108810001ED0696831F003011ED020F003006A46C3
:1088200001A921F0E3FBDDE900322146304623F0C7
:108830005BFD6968284631F003020ED062682C4661
:1088400022F00302121D1144416000F007F8046099
:1088500002B0284670BDFEE7FEE7FEE700F1080221
:10886000406830F00301A1F10400104418BF7047C4
:10887000FEE72DE9F04107460C004FF0000008BF6D
:10888000BDE8F08152B31146606810F0010F26D0A8
:1088900020F0030001F11002824210D8204600F0BF
:1088A0001FF8054626462046FFF7D8FF0660686891
:1088B000294640F0020068603846FFF70FFF204667
:1088C000FFF7CCFF416821F002014160606820F0B1
:1088D0000100606004F10800BDE8F081FEE7FEE7FA
:1088E00070B500F108030A1F9C18426804F10803E0
:1088F00022F0030CACEB0102DD1C25F00305121F76
:10890000AB4200D0FEE753181B1D9C4500D0FEE78C
:10891000237903F003031A43626022F003020C2A56
:1089200000D2FEE7027902F00302114341602046C3
:10893000FFF794FF0460416841F002014160606804
:1089400040F001006060204670BD38B5044615F067
:108950003FFA054615F074FA30B1218F2046E186C2
:108960001AF068FC012038BD0121606A1AF060F934
:1089700090F0010F20461FD013F076F8228FE18E81
:108980008A420DD02187E08E00906A461C21204645
:1089900013F04CFC012818BF38BD20461AF04AFCE1
:1089A000284615F058FA0428DCD1204619F060F961
:1089B000002114F03EFAD5E713F07EFAD2E770B545
:1089C00013F030FC054619F0B1F9044628460CF0C6
:1089D00041FC01462046BDE8704000221FF0ACBBC0
:1089E0002DE9F04F0C4687B08046002119F05DF864
:1089F00040B3DFF800B400214046BBF8062019F070
:108A00003FFF81460146002031F91030A3F5F852AE
:108A1000FF3A18BF401CF7D16061400016F0F2FE2B
:108A200060606069400016F0EDFEE060606900265D
:108A300000284CD939F91610EF4DA1F5F8509A38A5
:108A400007D040E007B02046BDE8F04F1C2117F0EA
:108A500015B90027404619F03BF800282FD93946B0
:108A6000404619F022F88246E4491AF0E8F8D0B9F5
:108A700050460021BBF8122019F002FFC0B20128B5
:108A800011D150460021BBF8102019F0F9FEC0B2F8
:108A9000B04208D1504619F0F0F8A84203DB504626
:108AA00019F0EBF8054640467F1C19F011F8B84262
:108AB000D5D8002DA4BFE06820F8165003DAE1688D
:108AC000002021F816006069761CB042B2D800255B
:108AD00061692E462846002984BF41F69A735A1CC4
:108AE00019D939F910109142A2BF2944A1F5F855BE
:108AF0009B3D0CDA994203BFE16831F81010314414
:108B0000D4F80CC01CBF2CF8101031440EB26169AF
:108B1000401C8142E5D840460021142219F0B0FEE5
:108B200007B2404619F039F86369C3F1010107FB48
:108B30000100801B01B20029B8BF00214FF0FF3CAB
:108B400000221046002B88BF41F69B761FD939F9C9
:108B50001030B3420CDBA3F5F8529B3A12B211FB72
:108B600002F3B3FBF5F3D4F80CC02CF810308446B4
:108B70006369401C8342EAD8BCF1000F07DBA81AE6
:108B80004843B0FBF5F0081AE16821F81C00002109
:108B9000BBF80220404619F073FE8146404619F0AA
:108BA00019F800904946002041F6FF7231F9103063
:108BB000934218BF401CF9D12061400016F022FEFC
:108BC00020602069400016F01DFEA060206900268C
:108BD000002844D939F91610874DA1F5F8509A3874
:108BE00039D10027404618F073FF00282FD93946A5
:108BF000404618F05AFF824680491AF020F8D0B952
:108C000050460021BBF80C2019F03AFEC0B20128F2
:108C100011D150460021BBF80A2019F031FEC0B234
:108C2000B04208D1504619F09DFFA84203DB5046E0
:108C300019F098FF054640467F1C18F049FFB842DE
:108C4000D5D8002DA4BFA06820F8165003DAA1687B
:108C5000002021F816002069761CB042BAD8002501
:108C600021692E462846002984BF41F69A72531C7A
:108C700019D939F910109942A2BF2944A1F5F85524
:108C80009B3D0CDA914203BFA16831F810103144CA
:108C9000D4F808C01CBF2CF8101031440EB2216962
:108CA000401C8142E5D840460021152219F0E8FD1C
:108CB0002369009900B2C3F1010200FB0210801B7E
:108CC00001B20029B8BF00214FF0FF3C002210463E
:108CD000002B88BF41F69B761FD939F91030B3427B
:108CE0000CDBA3F5F8529B3A12B211FB02F3B3FB73
:108CF000F5F3D4F808C02CF8103084462369401CE2
:108D00008342EAD8BCF1000F07DBA81A4843B0FB46
:108D1000F5F0081AA16821F81C0000211522404630
:108D200019F0AEFD0FFA80F900211422404619F027
:108D3000A7FD00B2049000211622404619F0A0FDC4
:108D4000C0B201280CBF01260026002101224046A6
:108D500019F096FD0FFA80FA00210422404619F01E
:108D60008FFD42F2D17705B2BA4505BFB8F82200AF
:108D700010F4006F4FF0000A4FF0010A404618F05F
:108D800029FF059040460021BBF8042019F078FD2A
:108D9000C2B22369A1682068CDE90031CDE902069D
:108DA0004B465146059809F04BF92083BD4205BF5B
:108DB000B8F8220010F4806F00250125404618F015
:108DC000ECFE064640460021BBF8082019F058FD8D
:108DD000C2B260694FF0000C6368E1688DE80B1067
:108DE00029463046049B09F02BF9608307B0BDE8A3
:108DF000F08F00009001002001E0FFFF010006005D
:108E00002DE9F84F0022054611461BF0ADFB00216D
:108E10003222284619F034FD044600211322284648
:108E200019F02EFD20440FFA80F900211222284665
:108E300019F026FD744920440FFA80F80968009162
:108E40006A462C21284613F0F1F9BDF800006F4C5A
:108E5000404448440FFA80FA284618F039FE074685
:108E600000211622284619F00BFDC0B201284FF050
:108E7000000B0CD0002F70D9A8686549006850F825
:108E80002B60304619F0DBFE00287CD168E0002F13
:108E900063D9A8685E49006850F82B60304619F025
:108EA000CEFE002844D15B49304619F0C8FE98B97F
:108EB000304618F03BFF78B100210A2219F0E0FC9F
:108EC0000004000C08D0B5F91800B6F91410401AC7
:108ED000411C8C4220DD2AE000210922304619F095
:108EE000CFFC10F0FF0018BF03280DD0062818BFD4
:108EF000082809D04FF000014FF00702304619F062
:108F0000BFFC00B250B113E0B5F91800B6F9141067
:108F1000401A411CA1420ADB0C4608E0308BB18AA2
:108F2000401A401C00B24844A042A8BF044624B2E4
:108F30000BF1010BBB45ACD341F6FF70C44218BF27
:108F400004EB080000D004B241F6FF70C44218BF21
:108F50005445C4BF2046BDE8F88F5046BDE8F88FA1
:108F60002C49304619F06BFEA8B9304618F0DEFEE9
:108F700088B100210A2219F083FC0004000C0AD0F9
:108F8000B6F9180000E032E0B5F91410401A411C9F
:108F90008C4220DD2AE000210922304619F070FCC5
:108FA00010F0FF0018BF01280DD0042818BF0728B3
:108FB00009D04FF000014FF00802304619F060FC74
:108FC00000B250B113E0B6F91800B5F91410401A08
:108FD000411CA1420ADB0C4608E0308BB18A401AE2
:108FE000401C00B24044A042A8BF044624B20BF18A
:108FF000010BBB45FFF440AF41F6FF70C44218BF00
:1090000004EB09009FD19FE79439030801E0FFFFBB
:10901000010004000100060000B50B88B0F808C08C
:1090200083B06344ADF800304B88B0F80AC06344A5
:10903000ADF802308B88B0F808C06344ADF8043056
:10904000C98843891944ADF80610436969469847B1
:1090500003B000BD2DE9F05F4FF0010E4FF0090A9B
:10906000FE4F0026002897F824B097F82D2097F897
:10907000339097F8328097F8315097F8304097F84E
:109080002FC097F82E3000F01D81012818BFBDE8D1
:10909000F09FBBF1070F80F0C780DFE80BF00410F2
:1090A00025415D7D9F00092A2CBF09205018C2B2BE
:1090B00087F82D200021012023F0DEFCB4E0092BED
:1090C0003CBF581887F82E0007D3092A1ABF87F823
:1090D0002E6087F83DE087F82EA097F82E2001211A
:1090E000084623F0C9FC9FE0BCF1090F3CBF0CEB24
:1090F000010087F82F000AD3092A0FBF092B87F830
:109100002F60022087F83D0008BF87F82FA097F84E
:109110002F204FF002014FF0010023F0ADFC83E05F
:10912000092C3CBF601887F830000ED3092A08BF0D
:10913000092B05D1BCF1090F08BF87F830A004D076
:1091400087F83060032087F83D0097F8302003212E
:10915000012023F091FC67E0092D3CBF681887F8D7
:10916000310010D3092A08BF092B06D1BCF1090F21
:1091700004BF092C87F831A005D087F831604FF083
:10918000040087F83D0097F831204FF004014FF0BC
:10919000010023F071FC47E0B8F1090F3CBF08EB78
:1091A000010087F8320012D3092A08BF092B09D120
:1091B000BCF1090F08BF092C04D1092D08BF87F89D
:1091C00032A004D087F83260052087F83D0097F878
:1091D00032200521012023F04FFC25E0B9F1090FD1
:1091E0003CBF09EB010087F8330015D3092A08BFFB
:1091F000092B0BD1BCF1090F08BF092C06D1092D91
:1092000004BFB8F1090F87F833A005D087F83360A1
:109210004FF0060087F83D0097F833204FF0060125
:109220004FF0010023F028FC97F83D10002908BFFB
:10923000BDE8F09F97F82D00894A40F6354350432A
:1092400097F82E2012FB03F200EB421097F82F2024
:1092500040F2712312FB03F200EB021297F8300088
:10926000C1F1070100EB4003C3EBC01002EBC002E9
:1092700097F8310000EBC00303EB001002EB800213
:1092800097F8320000EB800002EB400097F83320A3
:1092900083180A2021F0B0F900EE903A63210120F2
:1092A000F8EEE00A30EE200ABDEEC00A10EE104AD9
:1092B000224623F0E1FB204623F020FE87F83D60A4
:1092C000BDE8F09FBBF1070F50D2DFE80BF00412AE
:1092D0002843607FA200002A0EBF87F82D60501A35
:1092E00087F82D0097F82D200021012023F0C4FBE2
:1092F0009DE0002B1CBF581A87F82E0006D00121D4
:1093000097F82E20084623F0B7FB90E0002A1ABFFA
:1093100087F82EA087F83EE087F82E60EFE7BCF1D3
:10932000000F1CBFACEB010087F82F0006D097F8A8
:109330002F200221012023F09FFB78E0002A0FBF9D
:10934000002B87F82FA0022087F83E0008BF87F87F
:109350002F60ECE7002C1CBF601A87F8300006D0A5
:1093600097F830200321012023F086FB5FE0002ADC
:1093700008BF002B05D1BCF1000F08BF87F8306093
:10938000EED087F830A0032087F83E00E8E7002DF4
:109390001CBF681A87F8310006D097F831200421E5
:1093A000012023F069FB42E0002A08BF002B06D110
:1093B000BCF1000F04BF002C87F83160EDD087F8B6
:1093C00031A04FF0040087F83E00E6E7B8F1000F47
:1093D0001CBFA8EB010087F8320006D097F83220B6
:1093E0000521012023F048FB21E0002A08BF002BC3
:1093F00009D1BCF1000F08BF002C04D1002D08BF1B
:1094000087F83260EAD087F832A0052087F83E005E
:10941000E4E7B9F1000F1CBFA9EB010087F83300A6
:1094200058D097F833200621012023F025FB97F828
:109430003E10002908BFBDE8F09F97F82D00084AAC
:1094400040F63543504397F82E2012FB03F200EB11
:10945000421097F82F2040F2712303E0385D01207D
:1094600040420F0012FB03F200EB021297F83000AB
:10947000C1F1070100EB4003C3EBC01002EBC002D7
:1094800097F8310000EBC00303EB001002EB800201
:1094900097F8320000EB800002EB400097F8332091
:1094A00083180A2021F0A8F800EE903A63210120E9
:1094B000F8EEE00A30EEC00ABDEEC00A10EE104A27
:1094C000224623F0D9FA204623F018FD87F83E60A3
:1094D000BDE8F09F002A08BF002B0BD1BCF1000FA4
:1094E00008BF002C06D1002D04BFB8F1000F87F88B
:1094F000336096D087F833A04FF0060087F83E001F
:109500008FE700002DE9FF4F074689B0C8781A9C05
:1095100000F0010015460E46002814BFFD48FE4825
:10952000079014BFFD48FE4805900CBFFB48FC485F
:1095300006906188A2884FF0000EA1EB0201D4F8DA
:1095400010900AB270467146B9F1000F17D9E3685E
:109550004FF010084FF0080A01EB810C08EB8C0B60
:1095600013F80BB01BF0010F1CD00AEB8C0C33F876
:109570000CC0A2EB0C0212B2491C8945ECD84FF08A
:109580000008B9F1000F55D908EB88031021D4F871
:109590000CC001EB830101911CF8011011F0010FC7
:1095A00009D042E04FF00C0B0BEB8C0C33F80CC0E5
:1095B000604400B2E0E700286ED092FBF0F90C2185
:1095C00001EB830100913CF801104FF0060A01FB0A
:1095D00009F14FF004090AEB830A09EB83093CF90E
:1095E0000AA009B23CF909908A45D4BFD3468B46FC
:1095F000D94503DC8A45CCBF8946D146894505D08B
:10960000DDF804A001218E464CF80A10D4F80CC0F5
:10961000082101EB83012CF80190E3680099595A65
:10962000401AA2EB090100B20AB2216908F101084F
:109630004145A9D8BEF1000F7FF47BAF002116226F
:10964000384619F01DF9C0B2012818BF0020049057
:109650000020ADF80800ADF80C0003A902A8CDE980
:1096600000012089B4F9022003B23078189921F062
:10967000C9FAF1780498014207D0384618F0AAFADE
:10968000BDF808100844ADF808002946384618F01F
:109690000CFA804600F06FB9FEE7A249404619F087
:1096A000CEFA80B1F078C0F3800020B16D1E40F199
:1096B000528100F055B9B8686D1C41688D42C0F206
:1096C000578100F04DB9984800214289404619F071
:1096D000D7F810F0FF0F56D022694FF00009484626
:1096E000002A88BFE16810D900EB800351F82330CD
:1096F000434507D100EB8002082000EB820031F9DE
:10970000009002E0401C8242EED8F07810F0010F89
:10971000B8F8220019BF40F4006020F4806040F4E3
:10972000806020F40060A8F82200059908F1140078
:10973000884748452DD0404619F07CFDB8F8140004
:10974000ADF80000B8F81600ADF80200B8F818003F
:10975000ADF80400B8F81A00ADF80600079A4946BB
:1097600008F1140090476A462921404612F05EFD38
:10977000404618F0DBFA4246222112F057FD4046DF
:1097800019F058FD05E0B8F8220020F44060A8F870
:10979000220070784FF0000B01280FD0022815D15D
:1097A000069908F114008847B4F90010491C21F00B
:1097B0000101081A00EBD070401005E0069908F18D
:1097C000140088472188081A0FFA80FBF178049862
:1097D000014208D0059908F114008847BDF8081027
:1097E000081AADF8080000216B22404619F048F82D
:1097F0000FFA80FA00216C22404619F041F80FFA66
:1098000080F9404619F0AEF90090404618F035FA5C
:1098100001460AF4C040B0F5005F13D12AF4C040FD
:10982000B0F5FA6F0EDCB0F57A7FC8BFC0F57A707C
:10983000009A42433D4880FB02204211A2EBE070B7
:109840000FFA80FA09F4C040B0F5005F12D129F494
:10985000C040B0F5FA6F0DDCB0F57A7FC8BFC0F537
:109860007A704143314880FB01104111A1EBE07057
:109870000FFA80F9B8F814101698401A504402B242
:10988000B8F816101798401A484401B2F07800F062
:109890000100002814BFBDF90800584610440FFA13
:1098A00080F908BFBDF908B00BEB01000FFA80FA90
:1098B00059EA0A001FD0404619F0BCFCB8F8140061
:1098C0004844A8F81400B8F818004844A8F818004C
:1098D000B8F816005044A8F81600B8F81A0050441A
:1098E000A8F81A00404619F0A5FC00235246494644
:1098F000404619F062FDF178049801421CD10599A7
:1099000008F11400884719990844BDF80C10084460
:109910000EE00000E9460108DF4601088346010821
:109920004F46010801000600840100201F85EB510D
:10993000BDF80810084406E0BDF80C10199808445A
:10994000BDF80810081AADF80800F078C0F38000E0
:1099500048B16D1E04D4B868006850F825800AE04C
:109960004FF0000807E0B8686D1C41688D42F7DAD7
:10997000006850F82580B8F1000F1CBF0C98854294
:109980007FF48BAE0DB0BDE8F08F002908BF7047A3
:109990002DE9F04F8BB00446018300680F46002884
:1099A00018BF15F0C3FF07EB4700062101EB40008D
:1099B00015F0E8FE206000283DD0022101EB4701B0
:1099C0000144E160042101EB87010144C4E9010184
:1099D00001210026012F2FD0F800083015F012FFCA
:1099E00000EB87010B1DB90009B20025C1F101028E
:1099F000ADF804208E10ADF80010ADF802502A46E4
:109A0000069602950029C0F2E8804FF003084FF057
:109A100005090DF1180A0DF1080B4FF0000CBDF906
:109A20000460002E13DCBDF8021008EB4101314444
:109A3000ADF8041019E0FEE7B4220270E068068079
:109A4000E0684180A06806800BB0BDE8F08FBDF8EB
:109A500002E0BDF80010AEEB010E09EB4E0E7644AD
:109A6000491EADF80460ADF80010BDF80210491CA5
:109A70000EB2ADF80260BDF900108E420BDC8E1004
:109A80004AF82C6001F003014BF82C100CF1010C8A
:109A9000BCF1040FC3DBBCF1040F74D1DDF824C0AA
:109AA0000699614515D120F8121023F81250DDE90E
:109AB000021C6144DDE904C6B4446144D4F804C026
:109AC0000CF80210D4F804C009010CF80210511C63
:109AD0007AE0DDF81CC0614529D020F8121023F887
:109AE0001250D4F804C002990CF80210D4F804C043
:109AF00009010CF80210511C069A09B2521E20F8F6
:109B0000112023F81150DDE9032C6244DDF814C064
:109B10000CF1040C6244D4F804C00CF80120D4F811
:109B200004C012010CF80120491C0AB24DE0DDF816
:109B300020C020F81210614523F81250DDE9021C04
:109B4000614421D0D4F804C00CF80210D4F804C049
:109B500009010CF80210511C069A09B2521E20F895
:109B6000112023F81150DDE9042C6244D4F804C01C
:109B700008320CF80120D4F804C012010CF80120BE
:109B8000491C0AB221E028E0DDF810C06144D4F895
:109B900004C00CF80210D4F804C009010CF802103B
:109BA000511C069A09B2521E20F8112023F81150B8
:109BB000059AD4F804C00C320CF80120D4F804C083
:109BC00012010CF80120491C0AB2BDF90210BDF9BE
:109BD00000C06D1C61457FF720AF40F2D32117FB19
:109BE00001FC00EB42054FEAAC2135F9025C8D42E5
:109BF00005D103EB420535F9025C8D421FD0ACEB79
:109C0000812CBCF5007F04DC0CFB0CFC4CF3CF3C3E
:109C100007E0CCF5806C0CFB0CFC4CF3CF3CCCF19A
:109C20000F0C20F8121023F81210616801F802C01E
:109C300061684FEA0C1C01F802C0511C0AB2911E67
:109C400011D433F811C020F812C030F811C023F835
:109C500012C0D4F804C01CF801500CF80250521C79
:109C600012B2491EEDD5E6684FF0000C6146A6F829
:109C700000C0002A1FDDE56825F81C10A66830F832
:109C8000115026F81C5033F9115065450DD1914201
:109C90000BDAA76830F9116037F81C50B542A8BF3D
:109CA000354627F81C50491CEDE70CF1010C0FFA62
:109CB0008CFC9142DFDB15F027FE0BB0BDE8F08F86
:109CC00007B582B0022A9EBFBDF80C0005B000BDEA
:109CD000BDF80C30BDF80800D90A01EBD0211F29CE
:109CE00028BF1F2161F3CF20C3F34511C0F3451CEA
:109CF0006144ADF808003F2928BF3F2161F34A10B5
:109D000003F01F0100F01F031944ADF808001F29DC
:109D100028BF1F2161F30400ADF80800FF2A02BF2D
:109D200080B205B000BDDDE902010CF093FE0090A9
:109D3000BDF8000005B000BD07B582B0022A9EBF85
:109D4000BDF80C0005B000BDBDF80810BDF80C0052
:109D5000CB0A4FEAD02C13FB0CF35B0963F3CF2142
:109D600001F01F0300F01F0C13FB0CF35B0963F3FE
:109D70000401C1F34513C0F3451013FB00F0800943
:109D800060F34A11ADF80810FF2A02BF88B205B08F
:109D900000BDDDE902010CF05DFE0090BDF80000A1
:109DA00005B000BD07B582B0022A9EBFBDF80C0009
:109DB00005B000BDBDF80C30BDF80800D90AA1EB14
:109DC000D0210029D8BF002161F3CF20C3F3451172
:109DD000C0F3451CA1EB0C01ADF808000029D8BF69
:109DE000002161F34A1003F01F0100F01F03C91A9C
:109DF000ADF808000029D8BF002161F30400ADF8D8
:109E00000800FF2A02BF80B205B000BDDDE90201F3
:109E10000CF020FE0090BDF8000005B000BDF8B5C4
:109E2000044612F0FFF90646204612F0BFF9054637
:109E3000304617F07BFF04462B2D2CD00A2D18BF7F
:109E4000F8BD13F0C5FF18B10079012808BFF8BDAF
:109E50006946304617F0D8FF94F82C0010F00C0F2C
:109E6000304634D017F0B6FE0546002116222046B3
:109E700018F006FDC0B20128BDF9000005EBD57150
:109E80000CBFC0EB610000EB610090FBF5F018BF68
:109E900001B206D006E0618DBDE8F84000221EF058
:109EA0004BB901B20029B8BF00210025608D88425E
:109EB00018BF0125012220461EF03EF9002D08BFE3
:109EC000F8BD00221C21204612F0B0F9F8BD17F0B1
:109ED00064FEBDF9021000EBD07201EB620191FB50
:109EE000F0F0DEE730B590F8542083B002F00102C4
:109EF0008A4204BF03B030BD002990F854100CBF53
:109F000021F0010141F0010180F85410B0F84840FF
:109F1000B0F84A10ADF80210B0F84C20ADF80420AB
:109F2000B0F84E30ADF80630D0F824C0BCF814506C
:109F30002C44ADF80040BCF816C06144ADF80210E6
:109F4000416A898A1144ADF80410416AC98A1944EA
:109F5000ADF80610694619F0A7F903B030BD00004E
:109F60000100054803D001220421F7F7C5BC0022F7
:109F70000421F7F7C1BC0000000C024030B50C46CC
:109F80004249444B424A0D462DED028B81B0C1E956
:109F900001239FED418A002836D0404A0168914252
:109FA000C8BFB3EE040A07DCB1F1814FB4BFB1EE14
:109FB000000A90ED000A01DA80ED000ADFED380AB0
:109FC00020EE200ADFED370A20EE080A80EE201A84
:109FD000BCEEC10A10EE100A80B240F41010010C61
:109FE0008DF80010010A8DF801108DF80200A968A3
:109FF000002088470A2028F093FC6A6803216846FD
:10A000009047A96801208847002C02BF01B0BDEC31
:10A01000028B30BD24492068F0EE040A884284BFD8
:10A02000B8EE040A84ED000A04D820498842C8BF6B
:10A03000C4ED000A94ED001AF6EE001AB7EE040A19
:10A0400001EE210A20EE080A80EE201ABCEEC10AB9
:10A0500010EE100A80B240F48010010C8DF8001050
:10A06000010A8DF801108DF80200A96800208847C8
:10A070000A2028F055FC6A68032168469047A968C1
:10A080000120884701B0BDEC028B30BD9C1300203D
:10A09000B1A00008619F000800FF7F470000A041B9
:10A0A0000000C84200401C45000020C000002040C5
:10A0B0000A4601464FF47A730148F8F796BD00004E
:10A0C000DC0A0020002808BF704790ED000A10EE5F
:10A0D000101A174A9142C8BFF3EE0E0A09DCF0EEDF
:10A0E000400AF5EEC00AF1EE10FA38BFDFED110AB2
:10A0F00001D2C0ED000AB2EE041AC0EE010A9FEDD3
:10A100000E0AB0EE081A60EE800A80EE810A10EEA8
:10A11000100AB0F18B4FA8BF9FED080ABCEEC00A31
:10A120000022114610EE103A0548F6F7FDBF000078
:10A130000000F041000000000000804500F07F4575
:10A14000C409002008B5084611460CF077FB0090C2
:10A15000BDF8000008BD2DE9F04F0546C87A89B06A
:10A1600014460E4602289EBF012009B0BDE8F08FBC
:10A1700018463269B168FCF70FFB070004BF09B04D
:10A18000BDE8F08F786900F01F01032914BF06298C
:10A190004FF0060824D000F01F010E2912D0142918
:10A1A0000CBF4FF0140800F01F0019D0801E0D28BE
:10A1B00021D2DFE800F01D20201D201D1D1D1D1DCA
:10A1C0001D1D1D0030884FF00E08002804BF708848
:10A1D000B0F5807F04D04FF000004FF00508B86163
:10A1E0003A6A5AB12146284625F0E1FB00F0E7B86B
:10A1F0004FF00508F4E74FF00408F1E7B8690028CC
:10A200005BD02088ADF808006088ADF80A00A0880F
:10A21000ADF80C00E088ADF80E00B6F90030002B68
:10A2200004BF7088B0F5807F2DD0A0882188628817
:10A23000A0EB010000F1010001B2E08806F1040C7E
:10A24000A0EB020000F1010002B27088CDE9000C21
:10A2500002A8FCF7F3F9BDF8080021880844ADF81E
:10A260000800BDF80A0061880844ADF80A00BDF88E
:10A270000C0021880844ADF80C00BDF80E00618880
:10A280000844ADF80E0002AA04A8A968FBF7E8FC90
:10A2900000287ED004A8D5F80890A860D5F818C08A
:10A2A000BB692846BCF1000F04D022463146CDF8E8
:10A2B0000080E047C5F8089081E0224604A8A9681C
:10A2C000FBF7CEFC00287AD0BDF81400BDF81010C2
:10A2D000401A401C0FFA80FB0BEB4B0015F092FA72
:10A2E0008246A8680190BDF81000ADF80800BDF8DE
:10A2F0001200ADF80A00BDF81400ADF80C00BDF86E
:10A300001600ADF80E00012102A80AF0E8F9BDF927
:10A310001000B4F90010BDF91290401AB4F90210FF
:10A32000A9EB0104BDF916104945A4BF00B208907D
:10A3300040DB02AA06A80199FBF792FC50B35B46EA
:10A3400022B2CDF800A03846089913F037FA012858
:10A350000ED0384613F080F9504615F0D5FA38463D
:10A3600013F07AF90198A86009B00020BDE8F08FD9
:10A3700006A8A860D5F818C02846314602AA534658
:10A38000BCF1000F1CBFCDF80080E047BDF80A000B
:10A3900001E014E008E0401CADF80A00BDF80E0032
:10A3A000401CADF80E00641CBDF9160009F101094E
:10A3B0004845BEDA0198A860504615F0A5FA38461F
:10A3C00013F04AF909B00120BDE8F08F704782B060
:10A3D00000220092002804BF02B070470192019948
:10A3E000491C01910429FADB0099491C0091814222
:10A3F000F4D102B0704700002DE9F0411646254A1D
:10A4000080460C46107800283FD0B4F90400B4F917
:10A410000010B4F902C0411A4B1CB4F90610A1EBAC
:10A420000C0C0CF1010C03FB0CF35361B4F900307C
:10A430005360B4F902309360C2E90301B4F902C079
:10A44000B4F90050A1EB0C01401B4B1C421C6146AF
:10A45000284609F067F8B4F90270B4F90600B8426A
:10A4600013DBB4F90050B4F90400854208DC3088ED
:10A4700028F0B0F8B4F904006D1CB61C8542F6DD76
:10A48000B4F906007F1CB842EBDA4046BDE8F04163
:10A490000CF02BBF1C0100202DE9F74FC87898B0B5
:10A4A0000C4602289CBF1BB0BDE8F08FB2F900300B
:10A4B000ADF82830B2F902C0ADF82AC0B2F90400F4
:10A4C000ADF82C00B2F90620ADF82E20B4F920101A
:10A4D00001291FDD94F82210FD291BD32188C9B161
:10A4E00094F82310C1F3C0052B44C1F38001ADF8EB
:10A4F00028306144ADF82A1094F82310C1F30011FC
:10A50000401AADF82C0094F82300C0F34000101A54
:10A51000ADF82E0018980AA982680CA8FBF7A0FBDA
:10A52000002804BF1BB0BDE8F08FE07B10F00705EA
:10A5300007BF60680290E088ADF80800BDF8080029
:10A540006189884208BF00250AA80DF0B1FF5FEAC3
:10A55000000B4FF0000003900490059006900790C8
:10A5600008900990A0788DF82500BDF80800ADF896
:10A57000140002BF20880028002D5CD094F80380CE
:10A58000B8F1FD0F28BF4FF0FF08BDF82C10BDF843
:10A590002800081A401C0FFA80FABDF82E00BDF8FA
:10A5A0002A10401A401C0FFA80F9CA45B4BF504621
:10A5B0004846B4F90060B6EB600FA8BF4610BDF87E
:10A5C0003400BDF83010401A401C07B24FF0FF3085
:10A5D000169000200290002ED8BFBBF1000F0ED0C5
:10A5E000384615F00FF90290002332460AA90EA84A
:10A5F0000EF0A8FA00210EA80DF00CFD1690BDF883
:10A600003000ADF80000BDF83400ADF80400029849
:10A610000690FF20CDF80CD08DF82400CDF820D086
:10A620004A465146A01D12F0FDF95FEA000919D013
:10A63000022D0CD016E00AA80390E0788DF82400D3
:10A6400003A918980FF05AF91BB0BDE8F08FBDF9B7
:10A650003010D9F8080000EB4100BDF92810A0EB3C
:10A66000410004904FF0020ABBF1000F33D0BDF956
:10A670003240BDF93600A042C0F2ED8026B2ADF8FE
:10A680000260ADF806603A464146029815F0BDFA00
:10A69000BDF930103B46324602980DF0C1FE8DF8F0
:10A6A0001C00012808BF8DF81CA0012D09D1BDF99F
:10A6B0002A10D9F80800611A00EB41000088ADF8B3
:10A6C000140003A918980FF019F9BDF93600641C9D
:10A6D000A042D3DABFE04FF0000B002E59DDBDF8E9
:10A6E0002A00584404B2BDF82E00A0EB0B000FFA6C
:10A6F00080FABDF93200A042C4BFBDF936008245E0
:10A7000043DC3A464146029815F07FFABDF9001045
:10A710003B46224602980DF083FE8DF81C0001286E
:10A7200004BF02208DF81C00BDF93200A04213DCEA
:10A73000ADF80240ADF80640012D09D1BDF92A104F
:10A74000D9F80800611A00EB41000088ADF8140048
:10A7500003A918980FF0D2F8BDF93600824514DC31
:10A76000ADF802A0ADF806A0012D0AD1BDF92A105E
:10A77000D9F80800AAEB010100EB41000088ADF810
:10A78000140003A918980FF0B9F80BF1010BB345A9
:10A79000A5DBBDF82800ADF85000BDF82C00ADF8E1
:10A7A0005400BDF82A003044ADF85200BDF82E0028
:10A7B000801BADF8560014A80DF07AFE834628439E
:10A7C00025D001208DF81C00BDF92E008DF82480C5
:10A7D000A0EB060ABDF92A00841954453BDCBBF105
:10A7E000000F0DD03A464146029815F00EFABDF919
:10A7F00030103B4622B202980DF012FE8DF81C007C
:10A80000ADF80240ADF80640012D1DD112E0BDF8B3
:10A810002A008DF824803044ADF80200BDF82E00E7
:10A8200003A9801BADF806000020069018980FF0D1
:10A8300065F810E0BDF92A10D9F80800611A00EB9C
:10A8400041000088ADF8140003A918980FF056F8DD
:10A85000641C5445C3DD0298002818BF15F054F855
:10A860001698B0F1FF3F05D016980EF021FA0EA809
:10A870000DF0FEFDB9F1000F1CBF484612F0CBF8F9
:10A880001BB0BDE8F08F2DE9F0410646086990B095
:10A8900015460C4600281CBFA07E02289CBF10B0A5
:10A8A000BDE8F08129460EA8B268FBF7D9F9002867
:10A8B00004BF10B0BDE8F0810EA8B768B060206991
:10A8C00013F074FA022806D008A9206912F0DAFE03
:10A8D00001284CD0A6E04FF0000841F6FF70CDE90A
:10A8E0000080CDF80880D4E90412434603A81EF086
:10A8F00035FEA8882A88801A401C01B2BDF90C00D8
:10A9000001EBD17102EB610100EBD072A1EB6201AE
:10A910000844401EADF83010ADF83400E8886A886D
:10A92000801A401C01B2BDF90E0001EBD17102EB9F
:10A93000610100EBD072A1EB62010844401EADF84A
:10A940003600ADF8321004A80DF0B4FA6069049036
:10A95000208BADF81C00A07E8DF82A00CDF8008079
:10A960000CAA04A9304623690CF0C0FF5AE06846DF
:10A970000CF09AFFA0788DF80C00208BADF8080041
:10A98000E07E8DF80A00A07E8DF80B00207F4FF04E
:10A99000FF3C00284AD00899B5F902000CEB515150
:10A9A0000144ADF81A00ADF81E10B5F90610884242
:10A9B00038DC0899B5F90000C1F38A21491E014429
:10A9C000ADF81800ADF81C10B5F90410884217DC7A
:10A9D00006AA6946304623690CF034FF0899BDF891
:10A9E0001800C1F38A22104401B2BDF81C00ADF872
:10A9F00018101044ADF81C00B5F904008142E7DDE1
:10AA0000BDF81A000899BDF81E2000EB515000B2A5
:10AA100002EB5151ADF81A00ADF81E10B5F9061051
:10AA20008842C6DDB76010B0BDE8F081A8882988EB
:10AA3000401A401C00B200EBD07001EB6001089896
:10AA4000C0F38A23A1EB5301ADF81810EA886D8892
:10AA50005B1E521B521C12B202EBD27205EB620259
:10AA6000A2EB905219440CEB5050ADF81C1010445E
:10AA7000ADF81A20ADF81E0006AA694630462369D3
:10AA80000CF0E0FECEE72DE9FF4FA3B09B46DDE9D9
:10AA90003279DDF8C08015460C46FF2F28BFFF270E
:10AAA00008460DF005FD0C9040EA0B0050EA080046
:10AAB0007DD023982146826802A8FBF7D1F80028B0
:10AAC00004BF27B0BDE8F08FBDF80C00BDF808103A
:10AAD000401A401C00B204901C2105A815F0CEF8C5
:10AAE000049814F08FFE08904FF0FF300F90BBF1E8
:10AAF000000F0ADD00235A46214614A80EF022F862
:10AB0000002114A80DF086FA0F9001234246294631
:10AB10001AA80EF017F800211AA80DF07BFA119070
:10AB2000CDF814D0BDF8C4008DF82C70CDF828D025
:10AB3000ADF81C008DF82D90B4F900E0B5F90000D7
:10AB40000EEB0B018142D8BF014609B261F30F063B
:10AB50000D91B4F904101091A1EB0B02B5F904109A
:10AB60008A42A8BF0A460FFA82FAB4F90290B5F9F0
:10AB7000023009EB0B029A42D8BF1A4617B267F3AC
:10AB80001F461296B4F90680B5F90620A8EB0B0C07
:10AB90009445A8BF94460FFA8CF6DDF834C0994569
:10ABA000AAEB0C0C0CF1010C0FFA8CFC00E023E07A
:10ABB000D4BF4FF001094FF000099045ACBF4FF0F2
:10ABC00001084FF000080C9A002A00F0D480BDF86C
:10ABD0000800ADF80000BDF80C00ADF80400BDF9A8
:10ABE0000A40BDF90E00A042A8BFDDF810A07CDB32
:10ABF000B9F1000F7AD185E031980490DDF88C909E
:10AC00001C210CA815F03AF820A80C90BDF81000F3
:10AC1000ADF838008DF84870B4F90200B5F90210AB
:10AC20008842D4BF01270027B4F90600B5F9061001
:10AC30008842ACBF01260026B4F90000B5F9001027
:10AC40008842D4BF4FF0010A4FF0000AB4F9041053
:10AC5000B5F904209142ACBF4FF001084FF0000855
:10AC6000ADF88000A088ADF884006088ADF882005F
:10AC70006888401EADF886001FB10CA948460EF04A
:10AC80003DFEE888401CADF88200E088ADF8860003
:10AC90001EB10CA948460EF031FE2088ADF88000A8
:10ACA0002888401EADF88400002F14BFB5F90200BB
:10ACB000B4F90200ADF88200002E14BFB5F9060009
:10ACC000B4F90600ADF88600BAF1000F03D00CA964
:10ACD00048460EF013FEA888401CADF88000A088FE
:10ACE000ADF88400B8F1000F01E02EE00CE004BFE5
:10ACF00027B0BDE8F08F0CA948460EF0FFFD27B045
:10AD0000BDE8F08FA7421ADCB8F1000F01D1A642CE
:10AD10001BDB25B2ADF80250ADF806500499089837
:10AD200014F0E1FFBDF9081053462A4608980DF0CB
:10AD300077FB8DF8240005A923980EF0DFFDBDF9FF
:10AD40000E00641C84427FF753AF1AA80DF090FBED
:10AD500011980DF0ADFF0F98B0F1FF3F05D014A88A
:10AD60000DF086FB0F980DF0A3FF089814F0CCFDB2
:10AD700027B0BDE8F08F8645D4BF012000200E909B
:10AD800010988842ACBF012000200C900120109048
:10AD90000E990C98084000EA090010EA080F04D048
:10ADA000BCF1320FBCBF0020109001208DF82400B0
:10ADB000109819EA000F0FD00D98ADF80000ADF80B
:10ADC00004A06088ADF80200688805A9401EADF8AF
:10ADD000060023980EF092FD109818EA000F0FD08D
:10ADE0000D98ADF80000ADF804A0E88805A9401C56
:10ADF000ADF80200E088ADF8060023980EF07EFD65
:10AE00000E9870B12088ADF800002888ADF8027067
:10AE1000401EADF80400ADF8066005A923980EF0B9
:10AE20006DFD0C9870B1A88805A9401CADF8000014
:10AE3000A088ADF80400ADF80270ADF80660239864
:10AE40000EF05CFD109800287DD00D9ABDF90C0025
:10AE5000BDF90810521EADF800109042A4BF0D9825
:10AE6000401EADF80400401A401C05B2002D48DD1C
:10AE70000E9850EA09001CBFBDF90A40A7421BDD2D
:10AE80000FFA84FBADF802B0ADF806B02946089879
:10AE900014F029FFBDF900102B465A4608980DF012
:10AEA000BFFA8DF8240005A923980EF027FD12980B
:10AEB000641C0014A042E3DC0E9850EA080020D085
:10AEC000BDF90E00741C84421BDC0FFA84FBADF844
:10AED00002B0ADF806B02946089814F004FFBDF999
:10AEE00000102B465A4608980DF09AFA8DF8240067
:10AEF00005A923980EF002FDBDF90E00641C8442E2
:10AF0000E3DDBDF908000AF101018842D8BF084617
:10AF1000ADF80000BDF80C10ADF80410081A401C84
:10AF20000FFA80FABAF1000F48DD0C9850EA0900D8
:10AF30001CBFBDF90A40A7421CDD25B2ADF8025086
:10AF4000ADF8065000E04BE05146089814F0CBFEF7
:10AF5000BDF9001053462A4608980DF061FA8DF8A5
:10AF6000240005A923980EF0C9FC1298641C001453
:10AF7000A042E2DC0C9850EA08001FD0BDF90E0098
:10AF8000741C84421ADC25B2ADF80250ADF80650AC
:10AF90005146089814F0A7FEBDF9001053462A4602
:10AFA00008980DF03DFA8DF8240005A923980EF0BD
:10AFB000A5FCBDF90E00641C8442E4DD1AA80DF066
:10AFC00057FA11980DF074FE14A80DF051FA0F986D
:10AFD0000DF06EFE089814F097FC27B0BDE8F08FD6
:10AFE000BDF80800ADF80000BDF80C00ADF8040095
:10AFF000B5F90200B4F90210401A5845A8BF8346BB
:10B000000FFA8BF80025B8F1000FC8BFDDF81090DB
:10B01000D4DD6088284406B2E088401B07B2BDF941
:10B020000A00B042C4BFBDF90E00874224DC049977
:10B03000089814F058FEBDF900104B4632460898A7
:10B040000DF0EEF98DF82400BDF90A00B04207DCDE
:10B05000ADF80260ADF8066005A923980EF04EFC2D
:10B06000BDF90E00B84207DBADF80270ADF806700E
:10B0700005A923980EF042FC6D1C4545C9DB9DE7F0
:10B080002DE9F0470646A2F57F4090B092468946EA
:10B09000FF3804BF10B0BDE8F087746AB4F82080B0
:10B0A000984504D02384608C40F0080060844FF4FD
:10B0B00080215722204617F0E3FB07464FF48021FA
:10B0C0005922204617F0DCFB05B2706AB7F9087008
:10B0D00000281CBF002116F0E8FCB0F91600791911
:10B0E0000AFB010005EBD571A0EB6100ADF83A0059
:10B0F0003844691E0844ADF83E00706A818AADF894
:10B100003810008BADF83C0068460DF0F9FD6A463A
:10B110004FF48021204617F002FF0EAA69464846E8
:10B120000DF0D8FDA4F82080608C20F00800608429
:10B1300010B0BDE8F0872DE9F0430646A2F57F4048
:10B140008FB017460D46FF3804BF0FB0BDE8F0833F
:10B15000746AB4F82080984504D02384608C40F051
:10B160000800608402A80CF0A5FE02AA4FF480211A
:10B17000204617F017FE4FF480215922204617F081
:10B180007FFBADF81A00706A4FF00009002808BF75
:10B190004E4603D0002116F088FC0646002E04BF60
:10B1A0000FB0BDE8F0830298B6F91620B0F9081088
:10B1B000BDF91A00431807FB032200EBD073A2EB82
:10B1C00063021044491EADF82A200844ADF82E0051
:10B1D000A08AADF82800208BADF82C000AAA0CA894
:10B1E000A968FAF73DFD78B10CA8AF68A8603046B1
:10B1F00013F0AFFB034606F1140202A92846CDF86E
:10B2000000900CF073FBAF60A4F82080608C20F0FD
:10B21000080060840FB0BDE8F08300002DE9F34F13
:10B220000546F5488DB041680E68306910F0020F90
:10B230001EBF10F0040F0FB0BDE8F08FC0F3011077
:10B2400002284BD001281EBF03280FB0BDE8F08FA5
:10B250004FF00000009008460CF062F80746A988FD
:10B26000B5F900004FF4A053091A491C0CB2E98843
:10B27000B5F90220B3FBF4FC891A491C09B201910B
:10B280008C45B8BFB3FBF4F104920691317CC1F355
:10B290000111012971D06880611E0844E8800020F6
:10B2A000029001980028DCBF0FB0BDE8F08F049831
:10B2B0002044401E00B20790601E0590DDE90101A8
:10B2C000401A06998842C8BF084600B20390012080
:10B2D00038610298002840F0E28056E0A88829886A
:10B2E0006A88401A411CE888801A401C11FB00F053
:10B2F00000210E9C401E0FD004EB400204EB4103E2
:10B30000B2F800C0ADF800C01F881780401E491C6D
:10B31000A3F800C08842EFD872886988E888511A7B
:10B32000491EE9807188081A401E68803288298881
:10B33000A888511A491EA9803188081A401E288001
:10B340002988338930461944ADF80010698873891B
:10B350000E9A1944ADF80210A98833891944ADF842
:10B360000410E98873891944ADF8061043696946E9
:10B3700098470FB0BDE8F08FFFE77188081A401EAC
:10B38000E880001B401C688089E70198A0427DDBB3
:10B390000394307CC0F30110032814BF4FF0000E5B
:10B3A0004FF0010E0023601C00EBD0700A900E9A43
:10B3B00004EBD47009905BE00021E01A401E00B25B
:10B3C00008904EE0601A401EDDF820C000B2BEF1C9
:10B3D000000F22D013FB041802EB480910FB0438BD
:10B3E0000CFB040002EB480802EB400011FB04CC0C
:10B3F000B9F800A0ADF82CA0B8F800B0A9F800B0DA
:10B4000002EB4C0CB0F80090A8F80090BCF800805B
:10B41000A0F80080ACF800A021E013FB041802EBB8
:10B42000480911FB04C80CFB040C02EB480802EBB2
:10B430004C0C10FB0430B9F800A0ADF82CA0B8F803
:10B4400000B0A9F800B002EB4000BCF80090A8F8EA
:10B450000090B0F80080ACF80080A0F800A0481C74
:10B4600001B20A98B1EB600FACDB581C03B209982B
:10B47000B3EB600FA0DB307CC0F3011001280AD0D1
:10B4800031880498081A401EA88000E007E0001BDD
:10B49000401C288053E004982880079867E00098B3
:10B4A00020B94FF4205014F0ADF90090307CC0F377
:10B4B000011003280CBF4FF0010A4FF0000A039956
:10B4C00014FB01F0A0F1010E0598DDF800B048432F
:10B4D0000E9B4FF0000C0890002920DD0898BAF16F
:10B4E000000F604418BFAEEB00000022002C10DDFE
:10B4F00098460BEB40099B1CB8F80080A9F8008027
:10B50000BAF1000F14BF0844401A521C12B2A242F2
:10B51000EEDB0CF101000FFA80FC8C45DEDB307CA9
:10B52000C0F3011001281BD031880498091A029831
:10B53000081A401EA8800399401A401C2880DDE9A3
:10B54000020100EB01080198804512DBB86910F098
:10B55000010F1EBFB86910F0020F01200AD108E0E8
:10B56000029904980844288003990844401EA88042
:10B57000E5E7002078610099304600290CBF0E9A5B
:10B580000A46298803891944ADF82010698843893F
:10B590001944ADF82210A98803891944ADF8241084
:10B5A000E98843891944ADF82610436908A99847EA
:10B5B000386938B1B16A00291CBF304688473869FC
:10B5C0000028F7D1039814FB00F10E9800EB41001E
:10B5D0000E900FFA88F0019902908842FFF66EAE45
:10B5E0000098002804BF0FB0BDE8F08F0FB0BDE891
:10B5F000F04F14F089B90000600100202DE9F04FF0
:10B600009BB0054610F00EFE0446284610F0D4FD0F
:10B610001990204617F0A6FA0546204616F02DFB95
:10B62000A28A05EBD57102EB61020FFA82FAE28A77
:10B6300000EBD07002EB60000FFA80F94FEA610B6B
:10B640000EA80CF0C8FC0EAA0021204617F004FC3E
:10B650004FF41D701BFB00F042F2341190FBF1F02F
:10B66000801CADF83A00002631465022204617F0E3
:10B6700007F907B2002347F6FF7204F1140102A88C
:10B680000DF060FA002102A80CF0C4FC1890A28A08
:10B69000E08AADF84A00218BADF84C10638B3A4438
:10B6A000ADF848203844C91BADF84A00ADF84C103D
:10B6B000D81BADF84E00012347F6FF7212A908A867
:10B6C0000DF040FA002108A80CF0A4FC1A90BDF976
:10B6D0003A00ABEB07010025A1EB00080BEB0007DC
:10B6E00000208DF844008DF858008DF85C007048FB
:10B6F000C188A9421CBFFF218170C58094F83C100D
:10B7000001F0030101292AD0827802294BD091420D
:10B7100016D094F8262040F6CD4302EB021202EB3D
:10B72000420212FB03F2120C027094F8272002EB83
:10B73000021202EB420212FB03F2120C4270817001
:10B7400017AA16A9CDE9001205EB45024FF6FF71C5
:10B7500001EA420C4278017811AB604643E08278FE
:10B76000914215D0A28C02EB420253024FF4B47204
:10B77000B3FBF2F2828094F8272040F6CD4302EB2F
:10B78000021202EB420212FB03F2120C42708170B1
:10B7900017AA16A9CDE900124278E9B211AB808848
:10B7A00004F02EFE21E0914215D0A28C02EB420261
:10B7B00053024FF4B472B3FBF2F2828094F8262065
:10B7C00040F6CD4302EB021202EB420212FB03F2FF
:10B7D000120C0270817017AA16A9CDE90012017827
:10B7E000EAB211AB808804F00BFE9DF85C009DF876
:10B7F0005810C308BDF80000890863F3040080B244
:10B800009DF8442061F34A10D10880B261F3CF2043
:10B81000ADF8000080B20090BDF800000090BDF8C7
:10B820000000ADF83800300A00B283461DF066FE15
:10B8300078430AEBE030ADF850000BF15A0000B24B
:10B8400000901DF05BFE784309EBE030ADF852004C
:10B8500058461DF053FE00FB08F00AEBE030ADF84F
:10B86000540000981DF04AFE00FB08F009EBE030A0
:10B87000ADF8560014AA15AB0EA919980CF09DFB53
:10B88000E81C85B206F58766B5F5807F7FF628AFA0
:10B8900002A80CF0EDFD08A80CF0EAFD18980DF0D8
:10B8A00007FA1A980DF004FA1BB0BDE8F08F0000FB
:10B8B000C80100202DE9F04F88468A689FB00446F1
:10B8C00000F1140118A8FAF7CBF9002804BF1FB043
:10B8D000BDE8F08FD8F808001C9018A8C8F8080038
:10B8E00020460021322216F0CBFF054620460021DB
:10B8F000122216F0C5FF284400B21B9020460021FA
:10B90000102216F0BDFF284406B2204616F062F958
:10B91000B4F88410484340F30F201A90204616F0E4
:10B920003CF9B4F88610484340F30F20179012A852
:10B930000CF051FB12AA0021204617F08DFA414667
:10B94000684615F06EFE00257B480D95CDE9010592
:10B9500012A80690681E09950E906A461A210A954B
:10B96000204610F063FC20463122294616F088FF5D
:10B9700000F0FF0A20463222294616F081FF0FFA16
:10B9800080F920463322294616F07AFFC7B22046B6
:10B9900016F060FA1D90204616F036FBB4F87E10C3
:10B9A000002957D0E18A3144081A0FFA80FBA08A97
:10B9B000ADF85400208BADF85800B4F97E60BAF1B0
:10B9C000020F1BD9B9F1000F18DD17F0020F08D0D4
:10B9D00020460021102216F053FF00B2002808BFB5
:10B9E000012517F0010F09D020460021112216F081
:10B9F00047FF00B2002804BF701E06B2B54229DA24
:10BA000017986A4600FB05F1B4F87E00401E91FBD2
:10BA1000F0F05844ADF85600ADF85A004648019091
:10BA20000120029015A8099016A80A901A210E95D7
:10BA3000204610F0FBFB16AB15AA12A940460CF0ED
:10BA4000BCFA6A461B21204610F0F0FB681C05B2C8
:10BA5000B542D5DBB4F8800000285CD0A18A1B98E1
:10BA6000002601441D98081A0FFA80FBE08AADF801
:10BA70005600608BADF85A00B4F98050BAF1020F4D
:10BA80001BD9B9F1000F18DD17F0040F08D02046BC
:10BA90000021122216F0F4FE00B2002808BF012691
:10BAA00017F0080F09D020460021132216F0E8FEF7
:10BAB00000B2002804BF681E05B2AE422BDADFF8E0
:10BAC00078A015AF0DF158091A986A4600FB06F1E7
:10BAD000B4F880000E96401E91FBF0F05844ADF88B
:10BAE0005400ADF858000220CDE901A0CDE9097954
:10BAF0001A21204610F09AFB16AB15AA12A940464F
:10BB00000CF05BFA6A461B21204610F08FFB701C7C
:10BB100006B2AE42D8DB4FF0FF300E900020099005
:10BB20000A906A461B21204610F080FB1C98C8F83A
:10BB300008001FB0BDE8F08F103B03082DE9F14F5E
:10BB400092B0129810F032FB0546129810F06AFB82
:10BB50000446122D00F01181152D1EBF182D13B0B3
:10BB6000BDE8F08F16F0FEFF8246204616F085F8FD
:10BB7000814620460021322216F082FE06462046EB
:10BB80000021122216F07CFE30440FFA80F8204685
:10BB90000021132216F074FE304400B202902046B9
:10BBA0000021102216F06CFE304407B2204600211E
:10BBB000112216F065FE304400B20390608E4044BE
:10BBC000ADF84000A08E3844ADF8420094F839003A
:10BBD00000F00300012800F0488110A9E08ECDE9B3
:10BBE0000001B4F930304A46514606A8FAF726FD5E
:10BBF000BDF81810A08A0844ADF81800BDF81A1056
:10BC0000E08A0844ADF81A00BDF81C10A08A084468
:10BC1000ADF81C00BDF81E10E08A0844ADF81E0007
:10BC2000B4F914B0B4F916A0B4F91890B4F91A60C4
:10BC3000BDF81810A182BDF81A10E182BDF81C10E1
:10BC40002183BDF81E106183F548129915F013FF8A
:10BC500001281CBF13B0BDE8F08FA4F814B0A4F8FD
:10BC600016A0A4F818906683152D1CBF13B0BDE86C
:10BC7000F08FE08D00281FBFA08D0028E08E0028E7
:10BC800004BF13B0BDE8F08F129810F095FA834608
:10BC9000B4F914A0B4F916006AF30F0960F31F4950
:10BCA0000490B4F918000A9060F30F06B4F91A0072
:10BCB000059004F13202E18ECDE9001260F31F46D7
:10BCC000B4F93030B4F92E20B4F92C1008A8FAF7E2
:10BCD000B5FCBDF82400BDF82010401A401C60F3EC
:10BCE0000F05BDF82600BDF82210401A401C60F375
:10BCF0001F4594F8390000F0030001287ED0BDF8FC
:10BD00001C00BDF81810401A504460F30F06BDF82F
:10BD10001E00BDF81A10411A0498084460F31F462B
:10BD200009EB08000FFA80FA6AF30F0907EB2940C4
:10BD300000B20E900298301A00B260F30F060F9016
:10BD40000398C0EB26400FFA80F994F8380069F3A5
:10BD50001F4600F00301012918BF10F0030F77D030
:10BD6000022900F04881002304F1140219465846C4
:10BD70000BF068FD13B0BDE8F08F129810F050FA88
:10BD800005460078022804BF13B0BDE8F08F94F890
:10BD900038004FF0030181434FF001061CBF00F053
:10BDA0000301022950D0C0F38400042818BF0128E1
:10BDB0004AD120464FF000014FF0460216F060FDD8
:10BDC000C0B2FF2804BF208E00283DD1129810F089
:10BDD00027FA0746E08EB0F5807F3AD0204615F06E
:10BDE0004CFF8046204616F0BDFE04F1320CE28E78
:10BDF000CDE9002C00234246014600E03AE002A8CB
:10BE0000FAF71CFCBDF80800A18A00220844ADF82E
:10BE10000800BDF80A00E18A0844ADF80A00BDF840
:10BE20000C00A18A0844ADF80C00BDF80E00E18AB0
:10BE30000844ADF80E0002A93846F9F73DFF002886
:10BE40001CBF13B0BDE8F08F2E7013B0BDE8F08FAB
:10BE500030E0002204F114013846F9F72DFF0028E4
:10BE60001CBF13B0BDE8F08FEEE706A9204615F021
:10BE7000CEFED5E6B4F92C0029B2401A401C00EBE6
:10BE8000D070AAEB600161F30F090A99A1EB600081
:10BE900060F30F06B4F92E000499A0EB2540401C76
:10BEA00000EBD070A1EB600161F31F490599A1EB94
:10BEB000600033E708A80BF0F7FC08AA0021204631
:10BEC00016F019FFE08EADF82200208EADF82000AC
:10BED000608EADF82400A08EADF8260094F83800EE
:10BEE000BDF81C10C0098DF83400BDF8180004AA74
:10BEF0004044ADF81000BDF81A003844ADF8120007
:10BF00000298081AADF81400BDF81E100398081A1C
:10BF1000ADF81600DBF8081010460291F9F7A0FE04
:10BF2000002804BF13B0BDE8F08F04A8CBF80800C8
:10BF3000B4F92800B4F92C1090FBF1F201FB1202C5
:10BF4000B4F92A00B4F92E1090FBF1F301FB1300B1
:10BF50000E99084400B2ADF80200884203DDE18D7D
:10BF6000401AADF80200BDF90200E18D0144491EFE
:10BF7000ADF80610484538DA0AEB02000FFA80F8EF
:10BF80002F14ADF80080D04504DDA18DA8EB010091
:10BF9000ADF80000BDF90000A18D0144491EADF8C7
:10BFA00004100F99884213DA6A4608A95846636A52
:10BFB0000BF048FCBDF80000BDF8041028442944EB
:10BFC00000B2ADF8041031B2ADF800008842EBDBEE
:10BFD000BDF80200BDF80610384400B23944ADF88F
:10BFE0000200ADF806104845CBDB0298CBF80800FC
:10BFF00013B0BDE8F08F08A80BF05CFF08AA002181
:10C00000204616F0CFFE0020009004F1140208A98B
:10C010005846636A0BF06AFC13B0BDE8F08F00006D
:10C02000307A03082DE9F04FC7B0054610F0FAF852
:10C030000446284610F0C0F8039036A9204615F0B3
:10C04000E6FD00216922204616F01AFC0546002173
:10C050006A22204616F014FCBDF8D8104A1BBDF821
:10C06000DC10ADF8D8204B19BDF8DA10ADF8DC3093
:10C07000091ABDF8DEC0ADF8DA106044ADF8DE0094
:10C08000401A401C0FFA80FA9A1AD4E90A01521C8D
:10C090000FFA82FBA1EB0008D345ACBF4FF00109BA
:10C0A0004FF0000900222C9294F85C2002F0030269
:10C0B000012A08D1002806DA002904DD216B81421B
:10C0C00004BF01202C9020460021122216F0D8FB3C
:10C0D00001B22A9120460021132216F0D1FB00B2B2
:10C0E000299020460021102216F0CAFB00B22890A9
:10C0F00020460021112216F0C3FB00B22790BDF8A4
:10C10000D800A086BDF8DA20E286BDF8DC202287C0
:10C11000BDF8DE2062872A990844A086218F2998DD
:10C12000081A2087E18E28980844E086279891B263
:10C13000081A00B26087B9F1000F11D0E18E401AE1
:10C14000401C00B204281DDAE18A0AEBDA726FF0B3
:10C15000010000EB62000844E086001D608711E0EA
:10C16000218FA08E081A401C00B204280ADAA18A86
:10C170000BEBDB726FF0010000EB62000844A0865D
:10C18000001D2087218FA08E081A401C00B2269027
:10C19000618FE08E081A401C00B20290B9F1000FC6
:10C1A00017BF269F074604F13406351D11BFE4482A
:10C1B00004F13606351DE3482B90A06DB0F1FF3F2A
:10C1C00016D0236DA26A991A636D79439A1A7A433D
:10C1D00091FBF8F192FBF8F209B212B2521A5043F5
:10C1E000C21700EB126001EB202000B2249007E0A0
:10C1F000216BA06A081A784390FBF8F000B22490F3
:10C20000A06CB0F1FF3F16D0236CA26A991A636C40
:10C2100079439A1A7A4391FBF8F192FBF8F209B24A
:10C2200012B2521A5043C21700EB126001EB2020E9
:10C2300000B2259007E0D4E90910081A784390FB72
:10C24000F8F000B2259020460021162216F018FBC7
:10C25000C0B2B9F1000F15D001280AD130462E46E0
:10C2600005462598404200B225902498404200B2ED
:10C2700024903188259808442880318824980844DF
:10C28000308008E029882598081A401C30802988C9
:10C290002498081A28802C9838B3A06A4042784322
:10C2A00090FBF8F000B2B9F1000F0AD031880844D1
:10C2B000B5F9001000B28142DABF318028803080A9
:10C2C00034E02988081A401CB6F9001000B28142F7
:10C2D000CEBF288029803080B5F90000B6F9001063
:10C2E0008842BCBF3080298020E02B9904F13400C3
:10C2F000884701281ADC24A8039915F092F94FF415
:10C3000000303190904825900020269004F13400B0
:10C31000279024AA1A2120460FF088FF24AA1B2167
:10C3200020460FF083FF47B0BDE8F08F04A80CF063
:10C33000E7FC04AA4FF40031204616F0F0FD12A8E5
:10C34000039915F06EF94FF400301F907E484FF0BE
:10C350000008CDE9130804A8169004F134001590E4
:10C3600012AA1A2120460FF061FF20460B224146F7
:10C3700016F086FA05B2D345B4BF58465046B5EB21
:10C38000600FC8BF4510BDF91000029A269991426E
:10C39000A8BF1146B0EB610FC8BF4810B9F1000F3C
:10C3A00008D0228FA18E511A491C09B2B1EB400F5F
:10C3B00022DD07E0628FE18E511A491C09B2B1EB10
:10C3C000400F19DD9DF8130002909DF82A709DF82A
:10C3D00032608DF813808DF82A808DF8328004F158
:10C3E000340204A903980CF075FC02988DF8130030
:10C3F0008DF82A708DF83260A18A2A9800230844AB
:10C40000ADF81001218B29982A46081AADF81401BD
:10C41000E18A28980844ADF81201618B2798081A20
:10C42000ADF8160144A938A80CF08CFB002138A8FF
:10C430000BF0F0FD9DF832508DF832808DF846807B
:10C44000BDF8D810DDF8A8C0BDF8DC206144BDF807
:10C45000DE3009B20646ADF80010BDF8DA00DDF8AE
:10C46000A0C0B9F1000F6044DDF8A4C000B2A2EB97
:10C470000C02DDF89CC012B2A3EB0C03ADF8042053
:10C480001BB2ADF80200ADF8063012D0181A401CED
:10C4900000B204281FDAE18A0AEBDA726FF00100B9
:10C4A00000EB62000844ADF80200001DADF8060084
:10C4B00011E0501A401C00B204280CDAA18A0BEBE0
:10C4C000DB726FF0010000EB62000844ADF8000081
:10C4D000001DADF80400BDF91020002304F1340163
:10C4E0003EA80CF02FFB00213EA80BF093FD074661
:10C4F0006A4604A903980CF0EDFB8DF832508DF8D4
:10C5000013808DF82A808DF8468004F1340204A946
:10C5100003980CF0DFFB3EA80BF0AAFF38A80BF045
:10C52000A7FF38460CF0C4FB30460CF0C1FB12AA42
:10C530001B2120460FF07AFE47B0BDE8F08F0000C7
:10C540008F4601085B460108887903082DE9FF4FF3
:10C5500095B0987B0D4600F00F06897E229C032E35
:10C5600008BF0426012E00F01381022E00F0168170
:10C57000042E00F01981082E1CBF19B0BDE8F08F01
:10C58000DFF894824FF0FF0A4FF48072FD2924D225
:10C59000DFF8889299F80000884204BFD9F80400B7
:10C5A000B04214D04FF00000002A88BF9C4F0ED933
:10C5B00018F800C0BCF1FF0F0EBF8C461CFB01FC3D
:10C5C0004FEA1C2C07F800C0401C9042F0D3DFF863
:10C5D000508289F80010C9F80460D8880A90B3F82E
:10C5E000089000FB06F31798B0F9001015988068C2
:10C5F000B0F900209142ACBF0022521A0B920A9A65
:10C6000001EB020CB0F904209445D2BFDDF828B04C
:10C61000511A01F1010B1799B0F90220B1F902107A
:10C620009142ACBF0022521A0E92B0F9060001EB03
:10C6300009028242D2BF4846401A401C07900E9819
:10C6400000FB03F10B9800FB061004EBD00700F091
:10C6500007041C21684613F011FBA889ADF80800F7
:10C66000A87E8DF81800A87FC0F3C2008DF81900CD
:10C67000FAF764FC0AF058FE0A9901FB09F18142BD
:10C68000D8BF0846109013F0BDF881460390179864
:10C69000002501880B980A18ADF820201798ABF1F7
:10C6A0000101008801441798ADF8241043880E98C2
:10C6B000ADF8302018448B1AADF82200ADF83200E6
:10C6C000ADF834100799ADF826005B1C08441BB286
:10C6D000ADF836000F930CA80BF0EAFE129008A8F4
:10C6E00000900590C6F108001190DDE90A010844A8
:10C6F000A0EB0B00704313900E9807990A908842A4
:10C7000073DA0B98ABEB000014900B992AFA04F043
:10C710002B465945B8BF4FF0000E1ADA3A7802EAB4
:10C72000000C119A121B3CFA02F21ABF18F80220F0
:10C7300009F8052009F805E0119A944239BF3444FC
:10C74000F0400024504628BF7F1C491C6D1C5945F1
:10C75000E4DB129888B109EB0300BDF92620BDF98E
:10C7600020100E900F9B0BF05BFE8DF81000002840
:10C7700004BFDDE90E0113F081FA149841191098F5
:10C78000814217D2BDF82600401CADF8260020E0FB
:10C79000DFF890804FF0800A0222F7E6DFF8888009
:10C7A0004FF0C00A0422F1E6DFF880804FF0F00A73
:10C7B0001022EBE602208DF81000694615980DF066
:10C7C0009DF8BDF82600401CADF82200ADF826000B
:10C7D000002513980799204407EBD00700F00704C1
:10C7E0000A98401C0A9088428FDBBDF92210BDF9DF
:10C7F0002600814209D0401EADF8260002208DF8A7
:10C800001000694615980DF079F8484613F07CF849
:10C8100019B0BDE8F08F0000B23903087C01002098
:10C82000EC9400209C3903089E390308A2390308C0
:10C830002DE9FF4FB2F90240B3F902C0BBB0644525
:10C840000BDA128864F31F4062F30F001A886CF34E
:10C850001F4162F30F0137910AE0128864F31F4110
:10C860001B886CF31F4062F30F0163F30F003791D5
:10C870000FFA81FB06B20714ABEB06044FEA214A1C
:10C88000AAEB0705002CCCBF20466042002DCCBF90
:10C89000294669428842CCBF0120002000903C9884
:10C8A000B0F90210009800285FD0002DD4BF684274
:10C8B00028464201002CCCBF2046604292FBF0F09B
:10C8C000B44A105C10FB01F03F30C0114FEA600821
:10C8D00000F0010101EB08095E45B4BF314659463D
:10C8E000A1EB0001ADF86010CCBF314659460144C0
:10C8F000ADF864105745B4BF39465146A1EB00016D
:10C90000ADF86210CCBF394651460844ADF8660018
:10C910003B9818A982680846F9F7A2F9002804BFD5
:10C920003FB0BDE8F08F00200099002943D0002CD3
:10C9300025DDAAEB080109B2CDE90010A7EB08003C
:10C9400002B25B46314602A80BF008FF0AEB090170
:10C95000012009B2CDE9001007EB090002B25B46E5
:10C9600031460DA80BF0FAFE3EE0002CCCBF20466D
:10C9700060424201002DCCBF284668429EE70AEB88
:10C98000090109B2CDE9001007EB090002B25B46CC
:10C99000314602A80BF0E2FEAAEB0801012009B221
:10C9A000CDE90010A7EB080002B25B4631460DA8A6
:10C9B0000BF0D4FE18E0CDE900A00BEB090003B2A8
:10C9C00006EB090001B23A4602A80BF0C7FE0120AF
:10C9D000CDE900A0ABEB080003B2A6EB080001B262
:10C9E0003A460DA80BF0BAFE002102A80BF012FB8C
:10C9F000399000210DA80BF00DFB38904FF0FF305F
:10CA0000804600903C98407A10F0100F23D13819DE
:10CA1000032100B2CDE90001701B03B23A46314652
:10CA200021A80BF09BFE379902200A14111909B2B4
:10CA3000CDE90010379801B2481B03B22CA80BF0C7
:10CA40008DFE002121A80BF0E5FA009000212CA812
:10CA50000BF0E0FA8046BDF86400BDF86010401AA3
:10CA6000401C06B2FAF76AFA0AF05EFC824618A881
:10CA700007F0F9FD504503D218A807F0F4FD8246EF
:10CA8000504612F0BFFE8346BDF96690BDF86200C5
:10CA9000ADF8660000245146584613F024F91C21D5
:10CAA0001AA813F0EBF83C9818A91A910088ADF871
:10CAB00070003C98007ACDF874B0BDF962508DF8E2
:10CAC00080001F914D452FDC0BEB0407BDF9601072
:10CAD00033462AB238460BF0A3FC8DF8780018B91B
:10CAE0003146384613F0CAF83444A019504505D2EF
:10CAF000BDF86600401CADF8660012E002208DF81B
:10CB000078001AA93B980CF0F9FEBDF866000024E5
:10CB1000401CADF86200ADF866005146584613F06F
:10CB2000E2F86D1C4D45CFDDBDF96210BDF9660020
:10CB3000814209D0401EADF8660002208DF87800D1
:10CB40001AA93B980CF0DAFE584612F0DDFE02A856
:10CB50000BF08EFC0DA80BF08BFC0098B0F1FF3FA2
:10CB60001CBF21A80BF084FCB8F1FF3F1CBF2CA810
:10CB70000BF07EFC39980CF09BF838980CF098F884
:10CB800000980CF095F840460CF092F83FB0BDE8E4
:10CB9000F08F0000B23A03082DE9F04FCBB0054604
:10CBA0000FF040FB0446008E002804BF4BB0BDE8E8
:10CBB000F08F28460FF000FB0390608C40F00801D6
:10CBC0006184204644A915F022F80026B4F820809C
:10CBD0002684608C374640F00801354661842EA8D3
:10CBE0000CF08EF83CA80BF065F92EAA4FF4A021AA
:10CBF000204616F094F93CAA4FF4A021204616F0E6
:10CC0000D1F8608C102220F0080161842046A4F83D
:10CC10002080294615F034FE00B2499020461122AA
:10CC2000294615F02DFE00B24890204612222946D2
:10CC300015F026FE0FFA80FB20461322294615F038
:10CC40001FFE0FFA80FA12A8039914F0EAFC4FF4C1
:10CC5000A0201F90BA48CDE9130504A8169024A877
:10CC60001790208E002840F25981606AB54950F82B
:10CC70002700F3F75FFB48B9781C87B2606AB149B7
:10CC800050F82700F3F756FB0028F5D0E06A30F89B
:10CC90001600C0F30011002940F038810025C0F3D0
:10CCA0000021002918BF0125C0F3801000280ABF09
:10CCB000A08E45F08005B04213D118F0200F18BFA8
:10CCC00045F0200518F0020F18BF45F0020518F0D6
:10CCD000040F18BF45F0040518F0080F18BF45F001
:10CCE0000805A06A002D00EBC601B1F800C0ADF840
:10CCF000B0C04A88ADF8B2208888ADF8B400CB88BF
:10CD0000BDF810118C44ADF8B0C0BDF812C1084494
:10CD1000ADF8B400624403EB0C00ADF8B220ADF8FE
:10CD2000B60000F002812584608C40F00801618427
:10CD300004A80BF0E5FF24A80BF0BCF804AA4FF4FC
:10CD4000A021204616F0EBF824AA4FF4A02120469B
:10CD500016F028F8A4F82080608C20F00801618487
:10CD6000E06A30F81600C0F3C02000289DF8AD003E
:10CD700014BF40F0010020F001008DF8AD002CA898
:10CD8000159012AA1A21209620460FF04FFA9DF80E
:10CD9000330010F0200F3BD020F03E001E308DF805
:10CDA0003300B4F91410BDF9B02059448A4204BFCD
:10CDB00020F008008DF83300BDF9B410B4F9180064
:10CDC000A0EB0A00814205D19DF8330020F010004D
:10CDD0008DF83300B4F916204998BDF9B21010440B
:10CDE000814205D19DF8330020F004008DF8330016
:10CDF000B4F91A204898BDF9B610101A814207D12B
:10CE00009DF833008108490061F345008DF8330037
:10CE1000BDF8B610BDF9B200091A491C0FFA81F924
:10CE200015F0200F09D0E16A31F8161011F4806F67
:10CE30001CBFA0EB0900ADF8B2002CAA04A903980E
:10CE40000BF048FF606ABDF9A430249A50F827001F
:10CE50004790BDF81401BDF810C1BDF9A210A0EBB8
:10CE60000C00401C00B2CDE900109DF8ADC0CDF81B
:10CE700008C046A847991CF071FBBDF8B410BDF876
:10CE8000B000BDF91831091A491C09B2C91A01EBE1
:10CE9000D17100EB6101ADF8B010BDF8B600BDF87E
:10CEA000B2C0BDF91A21A0EB0C00401C00B2801AE0
:10CEB00000EBD0700CEB600000B21944ADF8B41078
:10CEC000811809B2ADF8B200ADF8B61015F0200F18
:10CED0000FD0E26A32F8162012F4806F09D009EB05
:10CEE000D972A0EB6200ADF8B200A1EB6200ADF820
:10CEF000B600002000902CAA24A9479B03980AF0B2
:10CF0000F5FC12AA1B2120460FF090F9701C86B286
:10CF1000781C87B2208EB0423FF6A7AE608C20F01E
:10CF2000080060844BB0BDE8F08F38222EA904A819
:10CF300012F086FD20223CA924A812F081FD0FE703
:10CF4000C0790308285501082DE9F04F9FB0054628
:10CF50000FF068F9044628460FF02EF91E900021C4
:10CF60003222204615F08CFC054600211222204674
:10CF700015F086FC28440FFA80FA0021132220467F
:10CF800015F07EFC28440FFA80F90021102220467B
:10CF900015F076FC28440FFA80F80CA80AF08AFFF6
:10CFA0000CAA4FF40031204615F0FCFED4F828B04E
:10CFB000BBF1000F08D1802012F024FC834601460B
:10CFC000802220460EF05AFE94F83C00002700F024
:10CFD0000F00012808BF012720460021162215F066
:10CFE0004FFCC0B2012808BF0127E06A00286ED0BC
:10CFF00010F0DCFE1490022817D06946E06A10F0A9
:10D0000041FB012803BF0098C0F38A26450D4FF06D
:10D01000FF3618BF3546EFB1A08A711E5044ADF8F7
:10D0200068000844ADF86C001EE09DF84D2041F604
:10D03000FF71BDF942000292CDE90001BDF9443013
:10D040000C9A15A8E16A1CF089FABDF95460BDF983
:10D050005650E0E7208BA0EB0900801BADF868007C
:10D06000711E0844ADF86C00149802285FD0204669
:10D0700014F003FE401BE18A00EBD07001EB60006E
:10D08000ADF86A00691E0844ADF86E0014A80AF0F5
:10D090000BFC14AA4FF40031204615F02CFE06EBD1
:10D0A000D6704010ADF8540005EBD5704010ADF8C7
:10D0B000560020464FF400316E2215F0E1FBADF82A
:10D0C00050001AAA14A9E36A1E980AF0BBFB04A830
:10D0D0000AF0F0FE04AA0021204615F063FE9DF838
:10D0E0002D2041F6FF71BDF92200CDE90001029229
:10D0F000BDF92430594603A8049A1CF02FFAE08A9F
:10D100004044ADF87200BDF80E100844ADF876004A
:10D11000E06AE8B16FB3208BBDF80C10A0EB0900FA
:10D12000401AADF870000844ADF874002AE0E08AB7
:10D13000691E4044ADF86A000844ADF86E00002056
:10D1400000901AAA0CA9E36A1E980AF0CFFBBEE76A
:10D15000204615F007FDBDF90C10A28A401A00EB1D
:10D16000D07002EB6000ADF870000844ADF87400B8
:10D1700008E0A08A5044ADF87000BDF80C100844D7
:10D18000ADF87400002000905B461CAA04A91E980C
:10D190000AF0ACFBA06A002804BF584612F0B4FBAA
:10D1A0001FB0BDE8F08F2DE9F04790B005460FF0B5
:10D1B00039F8044628460EF0FFFF06460CA9204623
:10D1C00014F0B5FC94F84800002510F0100F18BFBB
:10D1D000012510F0200F18BF45F002052046002160
:10D1E000012215F04DFB00B2A0F51C51D13902BF50
:10D1F000608C10F4006F45F0040504A80AF05AFE94
:10D20000B4F84400ADF82600B4F84600ADF82800A4
:10D210008DF82D5004AA0021204615F0C3FD9DF87D
:10D220002C000127002808BF8DF82C70E06B0590BA
:10D23000206C069005994FF6FF7081421CBF06993D
:10D2400081421CD04FF48029A0464FF05502494638
:10D25000204615F015FB024649464046F9F7AEFC5C
:10D260000090BDF80000ADF81E002046494620227F
:10D2700015F006FB0090BDF80000ADF8200094F812
:10D28000480041F6FF7800F00700022818BF032885
:10D290001ED19DF82C00022818BF032818D1BDF913
:10D2A0002200CDE900080295BDF92430049A03A8B4
:10D2B000616A1CF053F9BDF83400BDF83010401A13
:10D2C000401CBDF90C1000B28842B8BF8DF82C701C
:10D2D00004F1300794F8480000F00700032809D053
:10D2E000BDF83600BDF83210401A401C00B2B0F54F
:10D2F000806F00DA00270CA90EA8B268F8F7B0FC1E
:10D30000002804BF10B0BDE8F08794F8480010F082
:10D31000070F0BD1204614F077FE404202B20021E5
:10D320000CA807F0C7F9608BADF8360094F84800F8
:10D330000DF1380A00F00700022818BF032811D0A9
:10D3400000970CAA04A93046636A0AF0CFFAD6F80F
:10D350000890C6F808A094F8480000F007000328D9
:10D360000ED05CE0D6F80890C6F808A000970CAA8A
:10D3700004A93046636A0AF0B9FAC6F80890E8E7EB
:10D38000BDF92200CDE900080295BDF92430049AC8
:10D3900003A8616A1CF0E2F8BDF83400BDF8301053
:10D3A000401A401CBDF90C1000B2884219DA202244
:10D3B000114604980FF0AEF8B4F84410BDF80C20F4
:10D3C00000EB400011440844ADF82600B4F84600D4
:10D3D000ADF8280000970CAA04A93046636A0AF049
:10D3E00085FABDF83600BDF83210401A401C01B273
:10D3F000BDF90E00814212DAB4F84410ADF82610DF
:10D400000499B4F84620098910440844ADF828006E
:10D4100000970CAA04A93046636A0AF067FAC6F8B6
:10D42000089010B0BDE8F0872DE9F04FD7B0054661
:10D430000EF0F8FE044628460EF0BEFE82468268D4
:10D4400004F1140146A8F8F70BFC002804BF57B0FC
:10D45000BDE8F08FDAF80800549046AE204600216F
:10D460003222CAF8086015F00BFA00B20390204689
:10D470000021102215F004FA00B24E90204600213F
:10D48000112215F0FDF900B253902046002112221E
:10D4900015F0F6F900B24D9020460021132215F048
:10D4A000EFF900B24C90208C00254B902584608CC5
:10D4B00040F00801618424A80BF022FC24AA4FF458
:10D4C000A021204615F02BFD3CA80AF0F3FC3CAA55
:10D4D0004FF4A021204615F065FC4B982084608C09
:10D4E000002720F008012046618414F09DFD0146CC
:10D4F000E28A4E981044411A03980844401EADF841
:10D50000CE00204614F088FD4A9020461622294677
:10D5100015F0B6F9C0B201280CBF4FF001094FF069
:10D520000009514612A814F07CF84FF4A0201F9077
:10D53000F948CDE9130504A8169034A81790E08C9B
:10D540004FF0000800287DD9E06ABDF8CE1030F910
:10D550001800491C09B2421E0A44ADF8CE20BDF99C
:10D560001E21ADF8CA1091426CDCB9F1000F0AD04F
:10D57000228B4C99521A4A99521A0399511A491EF0
:10D58000ADF8C81009E0A28A4D990A444A99521A86
:10D5900003991144491EADF8CC10A18C0026002936
:10D5A00067D900EBD0705290401055900020009049
:10D5B000A06A50F8270000281CBF00780090B9F13D
:10D5C000000F0CD0BDF8C800401EADF8CC00216B98
:10D5D00031F81610401A401CADF8C8000BE0BDF839
:10D5E000CC00401CADF8C800216B31F8161008447F
:10D5F000401EADF8CC00A08C0025401E8642B8BF6E
:10D60000022126DAA06A7A1950F8220000281CBFED
:10D61000007810F0010F1CD0206B06EB050201EB27
:10D620004202805EB9F1000F1DBFBDF8C820101A7C
:10D63000ADF8C800BDF8CC2004BF1044ADF8CC0054
:10D64000681C00E01DE085B2A08CAA19401E824231
:10D65000D8DBBDF9CE10BDF91A01814217DA78196D
:10D66000401C87B2701980B2401C86B2A08CB042B8
:10D670009CD808F101001FFA80F8E08C8045FFF487
:10D6800063AF5498CAF8080057B0BDE8F08FBDF9F1
:10D69000CCE0ADF814E1ADF81611BDF9C8309DF835
:10D6A000B300ADF81031BDF9CA20ADF8122110F069
:10D6B000080F0ED0B4F914B0DDF834C1DC44634572
:10D6C00007DDBDF9B0C00CEBDC7CA3EB6C03ADF85F
:10D6D000103110F0040F0DD0B4F916C04E9B634406
:10D6E0009A4207DDBDF9B03003EBD373A2EB6302BE
:10D6F000ADF8122110F0100F11D0B4F918304C9A77
:10D700009A1A521E72450ADDBDF9B02002F00103DB
:10D7100002EBD27203EB62027244ADF8142110F0F6
:10D72000020F11D0B4F91A205398101A401E8842E3
:10D730000ADDBDF9B00000F0010200EBD07002EB91
:10D7400060000844ADF81601E18E0020414504BF99
:10D75000A18EB1427DD1218C11F0400F03D111F087
:10D76000200F18BF202011F0020F18BF40F0020058
:10D7700011F0040F18BF40F0040011F0080F18BF9B
:10D7800040F00800002864D02084608C40F008013C
:10D79000618404A80BF0B4FA34A80AF08BFB04AA45
:10D7A0004FF4A021204615F0BAFB34AA4FF4A02173
:10D7B000204615F0F7FA4B982084608C20F0080181
:10D7C000618444A81590A08C12AA08FB00602090E8
:10D7D0001A2120460EF02AFD44AA04A950460BF057
:10D7E00079FAA06A50F8270000287DD020464FF42F
:10D7F000A021122215F044F8834620464FF4A021C0
:10D80000132215F03DF8029020464FF4A02110227B
:10D8100015F036F8019020464FF4A021112215F0A2
:10D820002FF8BDF8C810BDF8CCC0594409B2ADF806
:10D830002011029ABDF8CAB0ACEB0202DDF804C0B8
:10D84000034612B2DC440020ADF82421ADF822C119
:10D8500000E023E0BDF8CEC0ACEB0303ADF8263109
:10D86000009BC3F3400BBBF1000F18BF0220511AFD
:10D87000491CBDF9E22009B20092CDE90110A06A6D
:10D88000BDF9E4303C9A50F8270000F108014FA898
:10D890001BF064FEBBF1000F1ED10AE0382224A960
:10D8A00004A812F0CDF820223CA934A812F0C8F840
:10D8B00087E7BDF93E11BDF8CA00529A01EBD1715C
:10D8C00000EB6202A2EB6102ADF82221559A02EB55
:10D8D00061010844ADF8260132AA46A950A8F8F71C
:10D8E000BFF908B150A800E010E0CAF80800002015
:10D8F0000090A06A48AA34A950F8270000F1080354
:10D90000504609F0F3FF46A8CAF8080012AA1B21E6
:10D9100020460EF08BFCA2E6F47A030870B50446AC
:10D92000806982B061898668A0896D4669B10028E6
:10D930007ED0814203D12289E3889A4279D3022999
:10D9400078D0032977D000F0DFB8002847D1E088ED
:10D950002189884243D2B4F906001BF0CFFDB4F907
:10D960000410B4F90E20891A48432168498801EB54
:10D97000E030ADF80200E0885A3000B21BF0BEFD86
:10D98000A18810FB01F02168098801EBE030ADF8B7
:10D990000400B4F908001BF0B1FDA18810FB01F0F0
:10D9A0002168498801EBE030ADF8060020895A3043
:10D9B00000B21BF0A3FDB4F90410B4F90E20891ACB
:10D9C000484321683246098801EBE030ADF8000099
:10D9D00069460846F8F744F900286FD08DE02068C2
:10D9E0000088ADF800002068A18840880844ADF8A0
:10D9F0000600B4F906001BF081FDB4F90410B4F977
:10DA00000E20891A48432168498801EBE030ADF8BF
:10DA10000200E0885A3000B21BF070FDA18810FBB4
:10DA200001F02168098801EBE030ADF8040003E063
:10DA300012E048E03FE042E0694632460846F8F727
:10DA40000FF930B1A0698560D4E9052021690BF098
:10DA500041F9A089002857D12068A188008808448E
:10DA6000ADF8040020684088ADF80200B4F9080061
:10DA70001BF044FDA18810FB01F02168498801EBEF
:10DA8000E030ADF8060020895A3000B21BF036FDB8
:10DA9000B4F90410B4F90E20891A484321683246BB
:10DAA000098801EBE030ADF8000069460846F8F758
:10DAB000D7F818B121E0012826D104E024E002289B
:10DAC00018BF012820D1206832460088ADF8000038
:10DAD00020684088ADF802002068A18800880844CA
:10DAE000ADF804002068A18840880844ADF806001D
:10DAF00029460846F8F7B4F830B1A0698560D4E942
:10DB0000052021690BF0E6F8A069866002B070BDBF
:10DB100070B504468069618982B08668A0896D46C7
:10DB200001290FD001287CD0814203D12289E388CA
:10DB30009A4277D3002976D0032908BF022871D0F2
:10DB400000F0E0B8012847D1E0882189884243D21B
:10DB5000B4F906001BF0D2FCA18810FB01F021688B
:10DB6000498801EBE030ADF80600E0885A3000B299
:10DB70001BF0C4FCB4F90410B4F90E20891A484310
:10DB80002168098801EBE030ADF80400B4F9080021
:10DB90001BF0B4FCB4F90410B4F90E20891A484300
:10DBA0002168498801EBE030ADF8020020895A3045
:10DBB00000B21BF0A3FCA18810FB01F021683246E3
:10DBC000098801EBE030ADF8000069460846F8F737
:10DBD00047F800287ED08EE02068A1880088401A8F
:10DBE000ADF8000020684088ADF80200B4F90600E6
:10DBF0001BF084FCA18810FB01F02168498801EB2F
:10DC0000E030ADF80600E0885A3000B21BF076FC38
:10DC1000B4F90410B4F90E20891A48432168098820
:10DC200002E015E048E043E001EBE030ADF804002D
:10DC3000694632460846F8F713F830B1A0698560A6
:10DC4000D4E9052021690BF045F8A089012859D1B4
:10DC500020680088401EADF804002068A188408834
:10DC60000844ADF80600B4F908001BF047FCB4F90D
:10DC70000410B4F90E20891A48432168498801EB41
:10DC8000E030ADF8020020895A3000B21BF036FCBB
:10DC9000A18810FB01F021683246098801EBE030D1
:10DCA000ADF8000069460846F7F7DAFF90B122E0C8
:10DCB000022818BF032825D12068A1880088A0EB7E
:10DCC0000100ADF8000020684088ADF8020020682F
:10DCD000008800E016E0A0F10100ADF80400206823
:10DCE000A188324640880844ADF806002946084617
:10DCF000F7F7B6FF30B1A0698560D4E90520216946
:10DD00000AF0E8FFA069866002B070BD70B50446F5
:10DD10008069618982B08668A0896D4602290DD02C
:10DD200002287CD0814203D12289E3889A4277D3AA
:10DD3000002976D0012975D000F0E6B8022846D136
:10DD4000E0882189884242D25A3000B21BF0D6FBCB
:10DD5000A18810FB01F02168098801EBE030ADF8E3
:10DD60000000B4F906001BF0C9FBB4F90410B4F9C3
:10DD70000E20891A48432168498801EBE030ADF84C
:10DD80000600B4F908001BF0B9FBA18810FB01F0F4
:10DD90002168498801EBE030ADF8020020895A3053
:10DDA00000B21BF0ABFBB4F90410B4F90E20891AD1
:10DDB000484321683246098801EBE030ADF80400A1
:10DDC00069460846F7F74CFF00286ED095E02068BA
:10DDD0000088401EADF804002068A1884088401AE1
:10DDE000ADF80200E0885A3000B21BF087FBA18832
:10DDF00010FB01F02168098801EBE030ADF800006C
:10DE0000B4F906001BF07AFBB4F90410B4F90E2043
:10DE1000891A48432168498801EBE03003E014E0A7
:10DE20004BE043E045E0ADF806006946324608465F
:10DE3000F7F716FF30B1A0698560D4E905202169A4
:10DE40000AF048FFA08902285ED12068A1880088D6
:10DE5000401AADF8000020684088401EADF806006A
:10DE600020895A3000B21BF049FBB4F90410B4F910
:10DE70000E20891A48432168098801EBE030ADF88B
:10DE80000400B4F908001BF039FBA18810FB01F075
:10DE900021683246498801EBE030ADF8020069465E
:10DEA0000846F7F7DDFE00B127E02DE003282BD16F
:10DEB00003E0032818BF002826D12068A188324635
:10DEC0000088A0EB0100ADF800002068A188408820
:10DED000A0EB0100ADF80200206829460088A0F1FF
:10DEE0000100ADF8040020684088A0F10100ADF801
:10DEF00006000846F7F7B4FE30B1A0698560D4E9A2
:10DF0000052021690AF0E6FEA069866002B070BDB6
:10DF100070B504468069618982B08668A0896D46C3
:10DF200003290FD003287CD0814203D12289E388C2
:10DF30009A4277D3022976D0012975D0022974D06C
:10DF400000F0DFB8032846D1E0882189884242D218
:10DF50005A3000B21BF0D2FAB4F90410B4F90E2012
:10DF6000891A48432168098801EBE030ADF80000C8
:10DF7000B4F906001BF0C2FAA18810FB01F0216879
:10DF8000498801EBE030ADF8020020895A3000B238
:10DF90001BF0B4FAA18810FB01F02168098801EB9D
:10DFA000E030ADF80400B4F908001BF0A7FAB4F9AA
:10DFB0000410B4F90E20891A484321683246498872
:10DFC00001EBE030ADF8060069460846F7F748FE79
:10DFD00000286ED08EE02068A18800880844ADF843
:10DFE000040020684088401EADF80600E0885A30E2
:10DFF00000B21BF083FAB4F90410B4F90E20891AA8
:10E0000048432168098801EBE030ADF80000B4F91D
:10E0100006001BF073FAA18810FB01F02168498803
:10E0200004E017E04BE045E048E044E001EBE0307D
:10E03000ADF80200694632460846F7F711FE30B1E6
:10E04000A0698560D4E9052021690AF043FEA08912
:10E05000032856D120680088ADF800002068A18808
:10E060004088401AADF8020020895A3000B21BF0F7
:10E0700045FAA18810FB01F02168098801EBE03026
:10E08000ADF80400B4F908001BF038FAB4F9041034
:10E09000B4F90E20891A484321683246498801EBB9
:10E0A000E030ADF8060069460846F7F7D9FD00B143
:10E0B00020E026E018B1012823D100E008BB206849
:10E0C00032460088ADF800002068A1884088401AD8
:10E0D000ADF802002068A18800880844ADF804006B
:10E0E000206829464088401EADF806000846F7F72C
:10E0F000B7FD30B1A0698560D4E9052021690AF037
:10E10000E9FDA069866002B070BD00002DE9F34F03
:10E11000B7B08046389808F11401826830A8F7F744
:10E120009FFD002804BF39B0BDE8F08F389830A9B2
:10E1300080682C9038988160B8F8820002283CBF33
:10E1400039B0BDE8F08F40460021322214F098FB30
:10E15000044640460021122214F092FB0519404665
:10E160000021102214F08CFB0444404613F032FDD1
:10E170000146B8F88400484340F30F202E904046F3
:10E1800013F00BFDB8F88610484340F30F202A9097
:10E19000404613F05FFEB8F814102944081A00B284
:10E1A0002B90404613F030FFB8F816102144081A9F
:10E1B00000B22D90389808F11401826834A8F7F75E
:10E1C0004FFD002804BF39B0BDE8F08F13A809F057
:10E1D00002FF13AA4FF4A021404614F03DFE16A8FA
:10E1E0000AF08EFD16AA4FF40031404614F097FE57
:10E1F00040464FF40031012214F042FB00B200EB24
:10E20000D0704FEA600940464FF40031042214F008
:10E2100037FB00B200EBD0704110BDF94E202591C4
:10E220008945B8BF494602EBD270B1EB600F05DDFE
:10E230009DF8550040F010008DF85500012A05D1D9
:10E240009DF8550040F010008DF85500B8F8821088
:10E250002E988142ACBF012000202F9008F12400AD
:10E26000F8F7ACFB04001CBF09F10100329000F08C
:10E270007981207B10F0010F40F06C812089ADF88E
:10E280004C002089ADF85C00002C00F0BE8098F8AE
:10E29000880010F0080F0CBF6089002005B22B9891
:10E2A0002895ADF89000ADF8480060682F4630F929
:10E2B0001520207BC0F3001108EB4101B1F96C007F
:10E2C000B1F97010131A2A9A081A5A4392FBF0F007
:10E2D0002A99091A2D980844ADF84A0068463899D9
:10E2E00013F09FF9A2480190032002904FF4A02060
:10E2F0000D9013A8069016A811940490BDF94AB089
:10E30000B8F882000026DA46002840F2E880BDF91D
:10E310004810ADF89010BDF84A00ADF892002C9866
:10E32000B0F9042032981044814200F3D8802E982E
:10E33000B8F8822000FB06F3501E93FBF0F32B98F5
:10E340001844289B00B2334493FBF2FC02FB1C32BE
:10E35000ADF84800237B15B26268C3F3001308EBE5
:10E36000430E32F91520BEF96C30A2EB030C2A9A49
:10E370000CFB02F2BEF970C0ACEB030392FBF3F2AC
:10E380002A9B9B1A2D9A1A442C9B12B2ADF84A2054
:10E39000B3F90030A3EB09035B1E83427DDC002E42
:10E3A0007BD02F9B83B3636847F6FF7C33F91770EC
:10E3B00067451CBF33F9153063456ED05245A8BF81
:10E3C00092465A45D8BF9346814266D0401EADF86A
:10E3D0004800ADF890001746ADF892B0ADF84AA0ED
:10E3E000D34504BF0AF10100ADF84A0012AB24AADC
:10E3F00013A9389809F0E1FDBDF84800BB46401C60
:10E40000ADF84800DA4662E000E0FEE7BDF89000B3
:10E41000A0EB09014844ADF89810ADF89C00BDF898
:10E4200092002599411AADF89A1025990844ADF843
:10E430009E00701E0E90606830F91700A0F5FE4136
:10E44000FF3914BF24A800200990606830F9152016
:10E45000A2F5FE40FF3814BF12A800200A9026A89B
:10E46000039060686A461A2130F917001090404600
:10E470000DF0DCFE606830F91720A2F5FE41FF398F
:10E480001EBF30F91510A1F5FE40B0F1FF0007D016
:10E4900012AB24AA13A9389800E018E009F08DFD0A
:10E4A000B9F1000F1CBF259800280BD0606830F927
:10E4B0001710A1F5FE40FF3804D026AA16A93898F7
:10E4C0000AF008FC6A461B2140460DF0AFFE701CA6
:10E4D00086B2B8F882002F46B0423FF618AF2F98A8
:10E4E000002804BFB8F88200B04233D1606830F928
:10E4F0001510A1F5FE40FF382CD0BDF848006A4643
:10E50000A0EB09014844ADF8A010ADF8A400BDF897
:10E510004A002599411AADF8A21025990844ADF892
:10E52000A600701E0E90002009900A9028A8039063
:10E5300060681A2130F91500109040460DF076FE03
:10E5400028AA16A938980AF0C5FB6A461B2140463E
:10E550000DF06CFE214608F12400F8F72CFA0400B7
:10E560007FF487AE38992C98886039B0BDE8F08F79
:10E57000103B03082DE9F34FB1B00646329806F17F
:10E58000140182682EA8F7F76BFB002804BF33B094
:10E59000BDE8F08F32982EA9322280682D903298F3
:10E5A00081600021304614F06BF9044600211222EC
:10E5B000304614F065F9074600211022304614F069
:10E5C0005FF90546304613F005FBB6F88410484362
:10E5D00040F30F202C90304613F0DFFAB6F8861087
:10E5E000484340F30F2B304613F034FC0146B28A07
:10E5F00038191044401A00B22A90304613F004FD36
:10E600000146F28A28191044401A00B22B9022A821
:10E6100009F0E1FC22AA4FF4A021304614F01CFCC2
:10E6200014A80AF06DFB14AA4FF40031304614F020
:10E6300076FC4FF400310122304614F021F900B28B
:10E6400000EBD0704FEA600A4FF4003104223046EC
:10E6500014F016F900B200EBD0704FEA6009BDF972
:10E660008A20CA45ACBF4946514602EBD270B1EB95
:10E67000600F05DD9DF8910040F010008DF89100CD
:10E68000012A05D19DF8910040F010008DF891000D
:10E6900006F12400F8F792F9040000F04A81207B8B
:10E6A00010F0010F40F03D812089ADF888002089ED
:10E6B000ADF85400002C00F0428196F8880010F06C
:10E6C000080F0CBF6089002005B22A982895ADF884
:10E6D0009400ADF804006068A84630F815000A28D8
:10E6E00004BF9748ADF804002BD02C980090206808
:10E6F000002330F915C0207BC0F3C00106EB4100B8
:10E70000B0F97820B0F97410604611F01BF82A991E
:10E71000CDF800B00844ADF804006068002330F97B
:10E7200015C0207BC0F3001106EB4100B0F970204A
:10E73000B0F96C10604611F005F82B99ABEB0000B6
:10E740000844ADF8060002A8329912F06AFF4FF4AF
:10E75000A0200F907B4803900320049022A80890EB
:10E7600014A813940690B6F88200002700287CD9DC
:10E77000BDF80400ADF89400BDF80600ADF89600B1
:10E780002898B6F88210384490FBF1F201FB120091
:10E7900005B2606830F91500A0F5FE41FF3965D07B
:10E7A000CDF800B0217B0023C1F3001206EB42013B
:10E7B000B1F97020B1F96C1010F0C4FF2B99ABEBDC
:10E7C00000000844ADF806002C9800902068002353
:10E7D00030F915C0207BC0F3C00106EB4100B0F951
:10E7E0007820B0F97410604610F0ACFF2A99002F21
:10E7F0000844ADF8040055D0BDF89400A0EB0A0120
:10E800005044ADF89C00BDF89600ADF89810A0EB10
:10E8100009014844ADF89E00781EADF89A1010909A
:10E82000606830F91800A0F5FE40FF3818BF25A831
:10E830000B90606830F91520A2F5FE40FF3814BF38
:10E8400001A800200C9026A80590606802AA1A2151
:10E8500030F91800129030460DF0E8FC606847F679
:10E86000FF7130F918208A4201E023E01AE01CBF52
:10E8700030F91500884210D001AB25AA22A93298A0
:10E8800009F09BFBBAF1000F18BFB9F1000F04D0DB
:10E8900026AA14A932980AF01DFA02AA1B213046B2
:10E8A0000DF0C4FC781C87B2B6F88200A846B842C6
:10E8B0003FF65EAFB6F88200B84232D1606830F9F8
:10E8C0001510A1F5FE40FF382BD0BDF8040002AAB8
:10E8D000A0EB0A015044ADF8A400BDF80600ADF865
:10E8E000A010A0EB09014844ADF8A600781E1090D6
:10E8F00000200B900C90ADF8A21028A8059060683D
:10E900001A2130F91500129030460DF08FFC28AA1C
:10E9100014A932980AF0DEF902AA1B2130460DF044
:10E9200085FC214606F12400F8F745F804007FF441
:10E93000B6AE32992D98886033B0BDE8F08FFEE70F
:10E9400001E0FFFF103B03082DE9F74F0D46B1F939
:10E950002E10A6B0904600291CBF95F8360002285C
:10E960009CBF29B0BDE8F08F01290BD1B5F9340067
:10E970000028DCBF288E002801BF688E002829B03F
:10E98000BDE8F08FB8F800002B8E00EB030CA88ECA
:10E99000ACEB000C0FFA8CFAB8F804C06AF30F065F
:10E9A000634403440FFA83F9B8F802C06B8E69F32D
:10E9B0000F029C44ACEB000C0FFA8CF7B8F806C0C1
:10E9C00067F31F466344184404B201EBD170AAEB0D
:10E9D0006001A1F10101ADF820104FF0010164F3D5
:10E9E0001F4201EB600018924844ADF82400B5F9CD
:10E9F0002E0000EBD070A7EB6000A0F10100ADF895
:10EA00002200B5F92E0000EBD07001EB600020442D
:10EA1000ADF8260095F836001A90FD2884BFFF2037
:10EA20001A90269808A9826824A8F7F719F90028EF
:10EA300004BF29B0BDE8F08FB8F80000ADF81000B1
:10EA4000B8F80200ADF81200B8F80400ADF81400F0
:10EA5000B8F80600ADF816004FF0FF32114604A8D2
:10EA600005F01BFEBDF81400BDF81010BDF8122013
:10EA7000401ABDF81610B5F90080891A401C491CCF
:10EA800000B209B2C3468842A8BF0846B8EB600F7F
:10EA9000C8BF4FEA6008A9EB0A00E11B401C491CF3
:10EAA00000B209B28842A8BF0846BBEB600FC8BFDE
:10EAB0004FEA600BB5F92E0000EB0B0404FB04F0E9
:10EAC000400010F09FFE0190B5F92EA081465A46F5
:10EAD0000AEBDA733014CDF864A00BEB630C0090F2
:10EAE0004FF0010B18982BEA0A0E0114ACEB0E0C38
:10EAF000801BACF1010C0BEB6303401CADF82A301A
:10EB0000ACEB0000ADF828000098ADF82CC0081A56
:10EB1000401C1844ADF82E000AEB020700230AA996
:10EB20000CA80AF00FF8DDF864A0BAF1010F18BFC5
:10EB30004FEA6A0A384610F065FE834600204E46CA
:10EB40001890002F3BDD7800239038B22290394690
:10EB5000584611F0C8F80CA800901898DDF830C09D
:10EB600002B200215846229BE047E8B19BF8000022
:10EB7000800190FBFAF030800120012F18DD0BEBB3
:10EB800000021BF8001012F8012C914207BF06EB9F
:10EB9000400131F8021C890191FBFAF126F81010AE
:10EBA000401CB842EBDB03E03046239911F066F8D5
:10EBB000189806EB4706401C1890B842C7DB584629
:10EBC00010F0A2FE0CA809F053FCBAF1010F3FD0DF
:10EBD00038B24A465146064620F047FE199800F0E2
:10EBE0000100504403B2012B20DD4FF47F5090FB15
:10EBF000F3F1002007FB07FCBCF1000F88BF8AB2CD
:10EC00000FD939F8101049B1FF2908BF29F8102091
:10EC100004D0890191FBF3F129F81010401C8445C0
:10EC2000EFD84A461946304620F01FFE002007FB69
:10EC300007F24946002A05DD19F810300B54401C34
:10EC40008242F9DC08A809F033FC0126A0B90DE0E6
:10EC5000002007FB07F24946002AF3DD39F810309F
:10EC60009B090B54401C8242F8DCEBE7E878FF2854
:10EC700024BFA878002801D04FF000064FF0FF30E5
:10EC80000E905EB94FF00103424604A912A809F0A4
:10EC900059FF002112A809F0BDF90E90BDF824001B
:10ECA000BDF82010401A401C00B210F0ABFD8246A7
:10ECB0001C211BA810F0E2FF02A81B90CDF878A041
:10ECC0002090A88DADF8740095F836008DF884007A
:10ECD000A8788DF88500BDF82410BDF82020881A8A
:10ECE000401C00B200EBD07002EB60000FFA80FB1A
:10ECF000BDF82200BDF82620ADF80C10121A521CE7
:10ED000012B202EBD272091B00EB6202491C17B26D
:10ED100009B2621EADF80810ADF80A00104400B246
:10ED20000092ADF80E005945D8BF5946ADF808100D
:10ED3000B842A8BF3846ADF80E00269802A98268EE
:10ED400006A8F6F78DFF002859D0424604A906A868
:10ED5000F6F7B2FFF0BBBDF81C10BDF91800BDF905
:10ED60001A20091A491C09B20A91BDF922300199E9
:10ED7000D21A02FB0411BDF92420121B801A084488
:10ED8000401E0C904EB1424604A906A8F7F708F8B9
:10ED900000281CBF01200D9000D10D960A98002874
:10EDA0002DDDBDF81800ADF80800BDF81C00ADF869
:10EDB0000C0002208DF87C00BDF91A90BDF91E10E0
:10EDC000CDF878A089451ADCADF80E90ADF80A9020
:10EDD0000D9800E013E000281CBF0C981E903BD05B
:10EDE0001BA926980AF08AFD0C9820440C9009F182
:10EDF00001000FFA80F9BDF91E004845E4DABDF8BC
:10EE00002400ADF80C00BDF82620001B401C111B8F
:10EE100000B2491CADF8080009B2ADF80A10ADF80F
:10EE20000E205845D8BF5846ADF80800781C0A9007
:10EE30008142D8BF791CADF80A10269802A98268D1
:10EE400006A8F6F70DFF00286CD0424604A906A8D4
:10EE5000F6F732FFA0B165E0224650460C9910F05B
:10EE6000EFFDBDF918104A4650460A9B09F0D8FA42
:10EE70008DF87C00012804BF02208DF87C00AFE7EC
:10EE8000BDF81C10BDF91800BDF90E20091A491C67
:10EE900009B21991BDF91E300199D21A02FB041171
:10EEA000BDF92420121B801A0844401E0C904EB15C
:10EEB000424604A906A8F6F773FF00281CBF0120EC
:10EEC0000D9000D10D96199800282BDDBDF8180083
:10EED000ADF80800BDF81C00ADF80C0002208DF85C
:10EEE0007C00BDF91E90BDF91A10CDF878A04945F7
:10EEF00018DCADF80E900D98ADF80A9000281CBFF4
:10EF00000C981E9035D01BA926980AF0F7FC0C9897
:10EF100020440C90A9F101000FFA80F9BDF91A0004
:10EF20004845E6DDBDF8200000992044ADF8080012
:10EF3000BDF82400001BADF80C00BDF82200ADF8B0
:10EF40000A00084400B2ADF80E00B842A8BF384627
:10EF5000ADF80E00269802A9826806A8F6F780FE92
:10EF600000287DD0424604A906A8F6F7A5FEA0B168
:10EF700080E0224650460C9910F062FDBDF9181051
:10EF80004A465046199B09F04BFA8DF87C0001283F
:10EF900004BF02208DF87C00B5E7BDF81C00BDF869
:10EFA0001810BDF90A20401A401C00B20B90BDF9A0
:10EFB0001A100198891A01FB04000C904EB14246C8
:10EFC00004A906A8F6F7ECFE00281CBF01200D904E
:10EFD00000D10D960B9800284CDD0D9800280EBF2F
:10EFE000CDF878A000201E90BDF81800ADF80800FC
:10EFF000BDF81C00ADF80C00BDF91A90BDF91E005B
:10F00000484537DBADF80E900D98ADF80A9060B129
:10F010001A98FF280C98007804D095F8361010FB49
:10F0200001F0000A8DF8840013E00C980B9A017827
:10F03000504610F0EAFDBDF918104A4650460B9BA9
:10F0400009F0EEF98DF87C00012804BF02208DF84C
:10F050007C001BA926980AF051FC0C98204400E083
:10F0600008E00C9009F101000FFA80F9BDF91E00CB
:10F070004845C7DA95F836008DF88400BDF82000C1
:10F08000BDF826102044ADF80800BDF82400001B90
:10F09000ADF80C00081B401CADF80E1000B20A9928
:10F0A000ADF80A008842D8BF781CADF80A0026984F
:10F0B00002A9826806A8F6F7D3FDE8B3424604A980
:10F0C00006A8F6F7F9FDB8BBBDF81C00BDF818108E
:10F0D000BDF91E20401A401C00B20B90BDF90E1065
:10F0E0000198891A01FB04000C900B98002859DD47
:10F0F0002EB1424604A906A8F6F752FE20B9002E0A
:10F1000008BFCDF878A001D000201E90BDF81800EF
:10F11000ADF80800BDF81C00ADF80C00BDF91E905C
:10F12000BDF91A0048453DDCADF80A90ADF80E90E7
:10F130003EB1424604A900E034E006A8F6F730FEEE
:10F1400000B966B11A98FF280C98007804D095F899
:10F15000361010FB01F0000A8DF8840013E00C98C3
:10F160000B9A0178504610F050FDBDF918104A4630
:10F1700050460B9B09F054F98DF87C00012804BF20
:10F1800002208DF87C001BA926980AF0B7FB0C988A
:10F1900020440C90A9F101000FFA80F9BDF91A0082
:10F1A0004845C1DD95F836008DF88400BDF824008F
:10F1B000ADF80C00011B491C0AB2BDF82200BDF8D5
:10F1C00026102044091B00B20A9BADF8082009B2A2
:10F1D000ADF80A00ADF80E108342D8BF781CADF828
:10F1E0000A00B942D8BF3946ADF80E105A45D8BF0B
:10F1F0005A46ADF80820269802A9826806A8F6F7B4
:10F200002FFDE8B3424604A906A8F6F755FDB8BBA2
:10F21000BDF81C10BDF91800091A491C09B20B9160
:10F22000DDE9002102FB0411BDF92420121B801A24
:10F230000844401E0C9046B1424604A906A8F6F7C1
:10F24000AFFD002818BF012503D1350008BF504687
:10F2500000D00C981E900B98002836DDBDF81800E1
:10F26000ADF80800BDF81C00ADF80C0002208DF8C8
:10F270007C00BDF91A90BDF91E10894525DC00E01F
:10F2800023E0ADF80A90ADF80E9095B9DDE90B21B9
:10F29000504610F0D5FBBDF918104A4650460B9B5E
:10F2A00009F0BEF88DF87C00012804BF02208DF81B
:10F2B0007C001BA926980AF021FB09F101000FFA36
:10F2C00080F9BDF91E004845D9DA01984FF0000CCD
:10F2D000002CC8BF04EBD47517DD00EB0409A9F1BD
:10F2E0000101002207E0037891F800E000F801EB4B
:10F2F00001F80139521CB2EB650FF4DB0CF101018E
:10F300000FFA81FC4846A445E7DBBDF820000099D0
:10F31000ADF80800084402B2ADF80C20BDF8220098
:10F32000BDF826102044091B00B20A9B09B2ADF8B3
:10F330000A00ADF80E109842A8BF781CADF80A007C
:10F34000B942D8BF3946ADF80E10ABF101000F90AD
:10F350008242A8BFABF10102ADF80C20269802A9A9
:10F36000826806A8F6F77CFCE8B3424604A906A822
:10F37000F6F7A2FCB8BBBDF81C10BDF91800091ABD
:10F38000491C09B20B91DDE9002102FB0411BDF912
:10F390000820801A08440C9046B1424604A906A8E9
:10F3A000F6F7FEFC002818BF012503D1350008BF81
:10F3B000504600D00C981E900B98002836DDBDF802
:10F3C0001800ADF80800BDF81C00ADF80C000220D4
:10F3D0008DF87C00BDF91A90BDF91E10894525DC19
:10F3E000ADF80A9000E021E0ADF80E9095B9DDE9A6
:10F3F0000B21504610F024FBBDF918104A46504628
:10F400000B9B09F00DF88DF87C00012804BF022049
:10F410008DF87C001BA926980AF070FA09F101000A
:10F420000FFA80F9BDF91E004845D9DABDF8200071
:10F430000099ADF80800084400B2ADF80C00BDF822
:10F440002210009AADF80A1011440F9A09B2ADF8D3
:10F450000E109042A8BFABF10100ADF80C00B9420C
:10F46000A8BF3946ADF80E10269802A9826806A8F2
:10F47000F6F7F6FBE8B3424604A906A8F6F71CFC2B
:10F48000B8BBBDF81C10BDF91800BDF90A30091A47
:10F49000491C09B20B91BDF91A200199D21A02FB3D
:10F4A0000411BDF90820801A00EB01094EB1424653
:10F4B00004A906A8F6F774FC00281CBF01200D90D3
:10F4C00000D10D960B98CDF878A0002827DDBDF867
:10F4D0001800ADF80800BDF81C00ADF80C000220C3
:10F4E0008DF87C00BDF91A50BDF91E108D4216DC56
:10F4F00000E014E0ADF80E500D98ADF80A50002869
:10F5000018BFCDF8789037D01BA926980AF0F6F9E5
:10F51000681C05B2BDF91E00A144A842E8DABDF896
:10F5200020000099ADF80800084401B2BDF826207B
:10F53000ADF80C10101B401CADF80E2000B20A9A5A
:10F54000ADF80A009042D8BF781CADF80A000F98B9
:10F550008142A8BFABF10101ADF80C10269802A9B9
:10F56000826806A8F6F77CFBE8B3424604A906A821
:10F57000F6F7A2FBA0B15FE022464946504610F0E4
:10F580005FFABDF918102A4650460B9B08F048FF59
:10F590008DF87C00012804BF02208DF87C00B3E7C1
:10F5A000BDF81C10BDF91800BDF90E20091A491C40
:10F5B0000FFA81FBBDF91E300199D21A02FB04112A
:10F5C000BDF90820801A47184EB1424604A906A882
:10F5D000F6F7E6FB002818BF4FF0010900D1B1464D
:10F5E000CDF878A000E027E0BBF1000F24DDBDF8E6
:10F5F0001800ADF80800BDF81C00ADF80C000220A2
:10F600008DF87C00BDF91E50BDF91A10A94213DC1B
:10F61000ADF80A50ADF80E50B9F1000F18BF1E97A3
:10F620002ED01BA926980AF069F9681E05B2BDF90B
:10F630001A002744A842EBDDBDF82000CDF878A0E1
:10F640002044ADF80800BDF8240002A9001BADF865
:10F650000C00BDF822002044ADF80A00BDF82600D9
:10F66000001BADF80E002698826806A8F6F7F8FA97
:10F67000E8B3424604A906A8F6F71EFBA0B143E092
:10F6800022463946504610F0DBF9BDF918105B46AA
:10F690002A46504608F0C4FE8DF87C00012804BFBD
:10F6A00002208DF87C00BCE7BDF91C00BDF91810E4
:10F6B000421A521C15B2002D26DDADF80810ADF827
:10F6C0000C00BDF91A40BDF91E0084421CDCADF8E7
:10F6D0000A40ADF80E402946504610F004FBBDF933
:10F6E00018102B462246504608F09AFE00E00BE028
:10F6F0008DF87C001BA926980AF000F9601C04B262
:10F70000BDF91E008442E2DD2EB912A808F0B0FE59
:10F710000E9809F0CDFA019810F0F6F8504610F066
:10F72000F3F829B0BDE8F08F2DE9F74FD0B050982D
:10F7300005909088B2F90030B2F802C0C01A401C9F
:10F7400001B2D08801EBD171A0EB0C00401C00B2DB
:10F750004FEA610800EBD070B8EB600FA8BF4FEA2A
:10F76000600803EB0800ADF80C0050884044ADF889
:10F770000E0020A808F02FFC20AA4FF4C0215098BA
:10F7800013F06AFB9DF8890040F010008DF88900A5
:10F7900018A808F08FFB18AA4FF4C021509813F056
:10F7A00001FB06A8519911F03CFFE44807904FF483
:10F7B000C02013900320089020A80C9005982430B6
:10F7C000F7F7FCF8050019BFA8F101004E9053B0FF
:10F7D000BDE8F08F1795A989A888A8EB01010AB2A6
:10F7E000BDF80C10A8EB000023920A1AADF8002116
:10F7F000BDF80E200144131AADF804111044ADF801
:10F800000231ADF80601012347F6FF7240A932A884
:10F8100009F098F9BDF80C00239A0123811AADF87C
:10F820000811BDF80E108A1AADF80A21239A521E4B
:10F830001044ADF80C018818ADF80E0147F6FF72C0
:10F8400042A938A809F07EF9BDF80C100023A1EBFD
:10F850000800ADF81001BDF80E20A2EB0800ADF8CD
:10F8600012014E980144ADF814111044ADF8160180
:10F8700047F6FF7244A924A809F064F9002124A8DE
:10F8800008F0C8FB01906889002814BFA0F1010BA3
:10F890004FF6FF7B4FF000096888002840F2368160
:10F8A00068890BF1010B4FF0000A584504BF4FF077
:10F8B000000B4FF0010AA869009068880021421EE1
:10F8C00048466B690FF03EFF07461690BAF1000FED
:10F8D00014BFA868286800904D9014BFE889E88894
:10F8E00006B20598049600F13000F7F767F80400B7
:10F8F00048D0207902283ED1A168B942DCBFE26835
:10F90000974238DC208AA38A304406B2608A984243
:10F9100004BF608AADF800002DD0A07D4FF0000339
:10F9200010F0010F4FF0FF000090384603D00FF0A9
:10F9300009FFC0B204E0D5E905120FF003FFC0B221
:10F94000A18A628AADF80020001DC208BDF800003F
:10F950007B4B89B240EA004041EA0141184019401E
:10F96000091A514300EB5110184040EA1040ADF81D
:10F97000000080B20090059821463030F7F71BF860
:10F980000400B6D1E88B09EB890149004843698836
:10F99000BDF90C20491E90FBF1F1B5F92000B8F13A
:10F9A000A70F00EB800001EB4004BDF80000ADF8AC
:10F9B0008000ADF882604046B8BFA72040441044A4
:10F9C000ADF81C01BDF80E00ADF81E0103AB4FF4FD
:10F9D0008072214647A815F009FB03A80F9047A89D
:10F9E000109018A8CDF850900B90BAF1000F5FD08E
:10F9F000019809F05DF9298A239803AB401ABDF8F4
:10FA00000C104FF480720844ADF81801BDF80E00D8
:10FA1000ADF81A01214646A815F0E8FA202218A9E7
:10FA20002AA810F00DF82AA80B903B4645A21021F9
:10FA300048A816F0C9FD48A8119006AA1A215098A6
:10FA40000CF0F4FB41F6FF70BDF9BA100024CDE9CB
:10FA500000100294BDF9BC304CA82A9A119919F0F3
:10FA60007DFDBDF93011BDF8180101EBD172A0EB9D
:10FA70006202BDF93201BDF81A3100EBD07CA3EB74
:10FA80006C031144ADF8F820ADF8FC101844ADF843
:10FA9000FA30ADF8FE0000943EAA119B0B995198E4
:10FAA00007F024FF002124A808F0B4FA019007E031
:10FAB00000200B90119006AA1A2150980CF0B6FB6A
:10FAC000BAF1000F14BF38A832A8002108F0A2FA3A
:10FAD000044603AB47AA20A9519808F06EFA2046C5
:10FAE00009F0E6F806AA162150980CF09FFBBDF825
:10FAF0003401ADF880000498ADF8820009F10100EE
:10FB00001FFA80F9688848453FF6CAAE32A808F067
:10FB1000AFFC38A808F0ACFC24A808F0A9FC0198B8
:10FB200009F0C6F8059829462430F6F744FF050089
:10FB30007FF450AE53B0BDE8F08F0000484003089A
:10FB40001FF8E007256400002DE9F74FACB017005F
:10FB500005464FF0000B08BF05F13C040ED0012F05
:10FB600008BF05F1540409D0022F08BF05F148046D
:10FB700004D0042F14BF5C4605F16004A068C0F3F4
:10FB80000E0101299CBF2FB0BDE8F08F10F4004F8B
:10FB900001BF208800286088002804BF2FB0BDE87E
:10FBA000F08FA1F101006168C1F30E4100FB01FA81
:10FBB000BAF1000F04BF2FB0BDE8F08F2846002136
:10FBC000122212F05DFE064628460021322212F073
:10FBD00057FE0644284611F0FDFFB5F8841048434F
:10FBE00040F30F2918A808F065F918AA4FF4C021AE
:10FBF000284613F0D7F8284612F02CF9A98A314488
:10FC0000081A00B223902089022F00F4004010D07F
:10FC1000002808BF4FF0000807D028464FF4C02145
:10FC2000102212F02DFE0FFA80F8E88A401E06B26C
:10FC300028E0002808BF4FF0000807D028464FF4FE
:10FC4000C021112212F01CFE0FFA80F8688B401CB4
:10FC500006B22D988068B0F90610B142BCBF2FB033
:10FC6000BDE8F08F1899B4F90020B0F90200B1F99D
:10FC70000810114406EB080211448142BCBF2FB0AA
:10FC8000BDE8F08F20A808F0A6F920AA4FF4C02103
:10FC9000284613F0E1F80020ADF88600ADF88400A6
:10FCA00006A82D9911F0BDFC894807900620089000
:10FCB000022014904FF4C020139018A80B9020A895
:10FCC0000C90022F14BF4FF0010B4FF0000B95F872
:10FCD000880000F0070002281CD1284600211522C8
:10FCE00012F0CEFDB5F8841000B248430012B5F80A
:10FCF000821009EB000292FBF1F109B2081A00EB45
:10FD0000D0722399A9EB000001EB620109B20FFA4E
:10FD100080F92391ADF8126005EB4B0000262A9084
:10FD200060680027C0F30E40B6FBF0F100FB1160E5
:10FD3000002808BF0127BDF98200A9EB000070432D
:10FD4000B0FBFAF12398BBF1000F0844ADF81000A6
:10FD5000BDF91210ADF814005DD0002F0CBFB4F93E
:10FD60000200B4F90000081AADF8160004A80F90BC
:10FD700005A8109095F8880000F00700032852D0DD
:10FD80006068C0F30E40B6FBF0F31693002F1CBF63
:10FD9000208910F4004F6CD04EA24FF0100126A81D
:10FDA00016F012FC18A80B9026A8119010201290A3
:10FDB00006AA1A2128460CF039FA41F6FF70BDF95F
:10FDC0007210CDE9001000270297BDF9743003A826
:10FDD000189A119919F0C2FBBDF90C10BDF8140066
:10FDE00001EBD171A0EB610200EB610001B212B234
:10FDF000BDF81600ADF89020ADF89410BBF1000FDF
:10FE00001FD0A0EB0800BDF80E30ADF89600C01A68
:10FE1000ADF892001DE0002F14BFB4F90000B4F952
:10FE200002000844A0E72A9852460021B0F9780061
:10FE300000902A98B0F9743030460FF083FC0346E6
:10FE4000A3E74044BDF80E30ADF892001844ADF879
:10FE50009600B5F914008142A4BFB5F9180090428C
:10FE600010DB009724AA18A9119B2D9807F03EFDDE
:10FE700008E000200B901190129006AA1A21284643
:10FE80000CF0D4F9BDF98200BDF9101000EBD07070
:10FE900001EB6002B5F914108A420DDBBDF91410B4
:10FEA000A1EB6001B5F91800884205DB05AB04AA97
:10FEB00020A92D9808F081F806AA1B2128460CF0ED
:10FEC000B5F9761C56457FF62BAF2FB0BDE8F08F05
:10FED000103B0308256400002DE9F74FB0B05FEA3E
:10FEE000020904464FF0000B08BF04F13C0611D094
:10FEF000B9F1010F08BF04F154060BD0B9F1020F9C
:10FF000008BF04F1480605D0B9F1040F14BF5E46DE
:10FF100004F16006B06810F4004F01BF3188002979
:10FF2000718800291CBFC0F30E0001289CBF33B0AC
:10FF3000BDE8F08F7168401EC1F30E4100FB01F86F
:10FF4000B8F1000F04BF33B0BDE8F08F19F1000025
:10FF500018BF01202B9020460021322212F090FC85
:10FF6000074620460021102212F08AFC0546204652
:10FF700011F013FEB4F88610484340F30F202D9083
:10FF8000204612F041F8E18AEA191144081A00B239
:10FF90002E90B9F1000F20464FF4C0210FD013224C
:10FFA00012F06EFC07B2B4F918002A90B6F90000FE
:10FFB0002990B6F902A0B9F1010F0ED106E0122284
:10FFC00012F05EFC07B2B4F91400EEE7404200B252
:10FFD0002990CAF100000FFA80FA03A807F0FBFF8E
:10FFE00003AA4FF4C021204612F036FF18A807F0EC
:10FFF00061FF18AA4FF4C021204612F0D3FE06A8D4
:020000040801F1
:10000000319911F00EFB714807900620089000040A
:10001000CDE9130903A80C9018A80B902B98002584
:1000200004EB40002C90BDF90E102D98401A684347
:10003000B0FBF8F12E98B9F1000F0844ADF8860036
:10004000ADF882002A98ADF884000CBF401E401C19
:10005000ADF8840070684FF0000BC0F30E40B5FBA4
:10006000F0F100FB115000281CBFBDF88400A0EB8C
:100070000A006CD0ADF8800021A80F9020A8109045
:100080002C9842460021B0F9700000902C98B0F9ED
:100090006C30A8EB05000FF055FB03461690BBF142
:1000A000000F1CBF308910F4004F5FD048A24FF002
:1000B000100124A816F088FA18A80B9024A8119013
:1000C0001020129006AA1A2120460CF0AFF841F633
:1000D000FF70BDF97210CDE900104FF0000BCDF8A4
:1000E00008B0BDF9743028A8189A119919F036FA99
:1000F000BDF9A210BDF8820001EBD172A0EB620144
:1001000000EB62002B9A09B2002A00B2BDF88020F1
:10011000ADF88A10ADF88E0020D0D319ADF8883034
:10012000BDF8A0301A443A44ADF88C20B4F916203A
:100130009042A4BFB4F91A00884220DBCDF800B089
:1001400022AA18A9119B319807F0D0FB17E0BDF83F
:10015000841029984FF0010B081A8BE7BDF8A030E6
:10016000D31ADB1BADF88830D21BDDE700200B90E3
:100170001190129006AA1A2120460CF057F8BDF9EA
:100180000E00BDF9861000EBD070B4F9162001EB1B
:10019000600191420DDBBDF98210A1EB6000B4F962
:1001A0001A10814205DB20AB21AA03A9319807F080
:1001B00004FF06AA1B2120460CF038F86D1C4545AB
:1001C0007FF631AF33B0BDE8F08F0000103B03087D
:1001D0002564000002484178491C417070470000C6
:1001E0008013002010B5012018F0C2FE164B00212C
:1001F00001225868401C5860B0F57A7FA8BFC3E957
:100200000021D86840F6B83C401CD8606045A8BFC3
:10021000C3E90221586940F2DC5C401C586160452A
:10022000A8BFC3E90421D869401CD861B0F57A7F22
:10023000A8BFC3E90621586A401C5862B0F5FA7F8E
:10024000A8BFC3E9082110BDF00200202DE9F0414C
:1002500004460DF0BDFD68B100688268002A1CBF2D
:10026000217A9047207E10F0020F74D110F0010F18
:1002700040F0BF80606801270026806828B1817E39
:1002800011F03F0F0CBF0020C06800252AE0016874
:1002900000291CBF017A11F0800F12D0802904D0F0
:1002A000227A21F0800191420BD14168E16001681E
:1002B00020468847207E10F0020F4CD110F0010F2D
:1002C0007CD161686D1C2846896821B18A7E02F064
:1002D0003F02824201D8002004E0C96805EB4500D6
:1002E00001EB8000002818BF002FD0D160680068A3
:1002F000D8B10169002908BF0068F9D0E660026939
:1003000021469047207E012610F0010F18BF0026DD
:1003100046B16068806830B1817E11F03F0F18BF30
:10032000C06800D1002000252EE00126F0E701681A
:10033000C1B1017A11F0800F14D100291CBF227ABB
:1003400091420FD14168E160016820468847207ED4
:1003500010F0020F03D04FF00100BDE8F08110F063
:10036000010F46D1616805F101052846896821B170
:100370008A7E02F03F02824201D8002004E0C96870
:1003800005EB450001EB800008B1C6B1CFE7B6B17F
:100390006068416899B1217E11F0040F2CD1217A57
:1003A000232918BF24291BD04FF4804112F040FCB0
:1003B00028B1207A11381C2812D201E019E01BE084
:1003C000DFE800F01A1A1A1A1A1A1A1A1A1A1A0E4A
:1003D0000E1A0E0E1A1A1A1A0E0E0E0E1A1A0E1ADD
:1003E0006068406860602046FFF730FF06460128DD
:1003F00002D00020BDE8F0813046BDE8F0817047B2
:1004000070B4DDE903C489B3050A15F0020F02D008
:100410001E462346344615F0040F02D06646A44615
:10042000344615F0060F05F0010626D016B11E461B
:100430006346B4468CF800206FEA010C0CF0FF0C08
:1004400012FB0CFC4FEA1C2C84F800C0C0B215F063
:10045000010F18BF11FB00F012D06FEA1020C0B2DC
:1004600012FB00F0000A187070BC7047FFE72270A2
:100470008CF800201A7070BC7047002EDAD1D6E7D5
:1004800000280FBF08024042C0B210FB01F0E4E7B1
:100490002DE9FF4F85B017460A460446DDE91301F2
:1004A0009388B2F800C0DDF84880A3EB0C035B1C16
:1004B0001DB2D38852889A1A521C16B20022D0B1AB
:1004C000BDF82020DFF8E49402EB0242B8F1FD0F02
:1004D000C0F00382A5F1040B4FF0000A002EDCBF30
:1004E00009B0BDE8F08F7B1B0193BDF82030A1EB74
:1004F000050E0021D2E0B8F1FD0F14D34FF0000833
:10050000002EDCBF09B0BDE8F08F2A4620460899CE
:1005100006F0BAF908F1010804EB47044645F4DC9B
:1005200009B0BDE8F08FBDF8000062F3040080B2AE
:1005300062F34A1080B262F3CF20ADF8000080B2BF
:100540000090BDF80000009001464246089806F071
:1005500081FA019008F10400C0080899C006000E55
:1005600089B2CA0A12FB00F2ADF80820C1F34512A5
:1005700012FB00F2ADF80A2001F01F0111FB00F19F
:10058000ADF80C10C0F1FF014FF0000C002EDCBFE5
:1005900009B0BDE8F08F0020002D44DDBDF800203B
:1005A00034F810309A4236D004EB4002BDF80830DF
:1005B0001288ADF80020ADF8042092B24FEAD2289C
:1005C00018FB0133DFF8E883C2F3451903FB08F396
:1005D0004FEAD368BDF8103068F3CF23BDF80A8026
:1005E00019FB0188DFF8CC9302F01F0208FB09F821
:1005F0004FEA986868F34A13BDF80C8012FB018239
:100600004FEA490802FB08F2D20E62F304039AB2E1
:10061000ADF81030019204EB4002BDF80430401CEC
:100620001380A842BADB0CF1010C04EB4704B4457B
:10063000B1DB09B0BDE8F08F90F800C0BCF1FF0F4E
:1006400008BF238027D0B4F80080ADF800800CF1FB
:10065000040C089F4FEADC08BDF800C0BFB24CEAAA
:100660000C4C47EA07470CEA090C07EA0907A7EB15
:100670000C0707FB08F70CEB571C0CEA090C4CEABB
:100680001C4CADF800C01FFA8CFCCDF800C0BDF8C2
:1006900000C0A4F800C0401C491CA41CA94202DAF6
:1006A00010F0030FC8D159457EDCD0F800C0BCF172
:1006B000FF3F7AD0BCF1000F78D090F800C0BCF1B9
:1006C000FF0F08BF238027D0B4F80080ADF800806A
:1006D0000CF1040C089F4FEADC08BDF800C0BFB263
:1006E0004CEA0C4C47EA07470CEA090C07EA0907F1
:1006F000A7EB0C0707FB08F70CEB571C0CEA090CDF
:100700004CEA1C4CADF800C01FFA8CFCCDF800C0C0
:10071000BDF800C0A4F800C004F1020C10F8014FAD
:10072000FF2C08BFACF8003023D0BCF80080ADF837
:100730000080241D089F4FEAD408BDF80040BFB2D6
:1007400044EA044447EA074704EA090407EA0907B8
:100750003F1B07FB08F704EB571404EA090444EABB
:100760001444ADF80040A4B20094BDF80040ACF8C9
:10077000004010F8014F0CF1020CFF2C08BFACF840
:10078000003027D0BCF80080ADF80080241D4FEA6F
:10079000D408089FBDF80040BFB244EA044404EA0C
:1007A000090447EA074702E055E044E04DE007EA64
:1007B00009073F1B07FB08F704EB571404EA090479
:1007C00044EA1444ADF80040A4B20094BDF80040DF
:1007D000ACF8004010F8014F0CF1020CFF2C08BFE0
:1007E000ACF8003023D0BCF80080ADF80080241DA8
:1007F000089F4FEAD408BDF80040BFB244EA044461
:1008000047EA074704EA090407EA09073F1B07FB11
:1008100008F704EB571404EA090444EA1444ADF859
:100820000040A4B20094BDF80040ACF800400CF1C8
:100830000204401C0BE014F0030F04BF226062604E
:1008400003D02380C4F80220E380001D0834091D72
:1008500059457FF72AAFA94233DA90F800C0BCF1BE
:10086000FF0F08BF238027D0B4F80080ADF80080C8
:100870000CF1040C089F4FEADC08BDF800C0BFB2C1
:100880004CEA0C4C47EA07470CEA090C07EA09074F
:10089000A7EB0C0707FB08F70CEB571C0CEA090C3D
:1008A0004CEA1C4CADF800C01FFA8CFCCDF800C01F
:1008B000BDF800C0A4F800C0401C491CA41CA942FB
:1008C000CBDB01990AF1010A04EB41047044B24503
:1008D000FFF60FAE09B0BDE8F08F4FF0000CB4F892
:1008E00000A0ADF800A06346E646002EC7BF491B36
:1008F000019109B0BDE8F08F0021002D4BDD027899
:10090000F2B3624505D0FF2A0EBF434602FB08F34F
:100910001B0A624504BF34F811B0DA452FD0FF2B13
:1009200008BFDDF820C025D004EB410CDDF820A085
:10093000BCF800C0ADF800C003F1040C4FEADC0BBA
:10094000BDF800C01FFA8AFA4CEA0C4C4AEA0A4A7F
:100950000CEA090C0AEA090AAAEB0C0A0AFB0BFAD0
:100960000CEB5A1C0CEA090C4CEA1C4CADF800C00C
:100970001FFA8CFCCDF800C0944634F811A000E0BA
:1009800005E004EB4102BDF800B0A2F800B0401C45
:10099000491CA942B3DB01990EF1010E04EB470497
:1009A0000844B645A8DB09B0BDE8F08F1FF8E007A2
:1009B00010080800080404000068096888420CBF99
:1009C00001200020704740680A6820F040409042B3
:1009D00038BF0860002070472DE9FF4F81B088467E
:1009E000DDE90EB400210122019811F049FF05B2A2
:1009F00000210422019811F043FF01B298F803008E
:100A000010F0020F0DD010F0010F42F2D17202D09F
:100A1000954202D009E0914209D120F0020088F805
:100A20000300C0B210F0010F01D07F4800E07F4802
:100A3000009098F8030010F0010F0CBFDFF8E8A158
:100A4000DFF8E8A100276780A78027612780A760DB
:100A5000E760039D0198294611F027F806007CD035
:100A60000398854206D04FF40001304612F0E0F8BA
:100A7000002872D16E49304612F0E1F800286DD19D
:100A80006C4800214289304611F0FAFE10F0FF094F
:100A90006CD02069401C2061A1885944A180217D2F
:100AA00011F0010F74D000EB800080000EF0AAFE60
:100AB000070020D0E16851B12069401E00EB8000A2
:100AC000820038460EF0BCFFE0680EF01DFF206982
:100AD0004FF0000100EB800007EB800040F8146C41
:100AE00098F8030010F0010F06D00222304611F0F2
:100AF000C7FE00B205E0FEE70522304611F0C0FE59
:100B000000B2216901EB810107EB810121F8100C92
:100B100098F803004FF0000110F0010F05D00322F8
:100B2000304611F0ADFE00B204E00622304611F06E
:100B3000A7FE00B2216901EB810107EB810121F8D9
:100B40000E0C2069002100EB800007EB800040F8CC
:100B5000089C206900EB800002E037E025E005E01A
:100B600007EB800040F8041CE76011E00099304674
:100B7000884798F8031011F0020F05D0B4F904105B
:100B80000A1804998A4221DCA18858440844A080AC
:100B90003046D0470146B4F900008142C4BF304618
:100BA000D0472080A068401CA06098F8030010F097
:100BB000040F14BF4FF0FF300120451906D4294619
:100BC000019810F072FF06007FF44AAFB4F90400F8
:100BD0000028C4BFA0EB0B00A0802069002814BF30
:100BE0000498B4F904006080CEB10398854216D110
:100BF00001988068016851F8256098F80310C1F3E6
:100C00008001002914BF6D1E6D1C46B13046D047CF
:100C1000208000993046884760800120A06005B0A0
:100C20002846BDE8F08F0000652B02087B1C0208F7
:100C300001000600840100202DE9F04FC44D93B05F
:100C4000044600216A8811F01BFE012121EA0002FE
:100C50009DF8171062F30001820862F34101C00899
:100C600060F382018DF817100021AA88204611F048
:100C700007FE8DF814000021EA88204611F000FEDE
:100C80008DF8150000212A89204611F0F9FD8DF814
:100C9000160000211622204611F0F2FDC0B20128F4
:100CA0000CBF4FF0010A4FF0000A9DF817004FF0FB
:100CB000000110F0010F12D01422204611F0E0FDC7
:100CC00006B29DF817004FF0000110F0010F0CD094
:100CD0001522204611F0D4FD0FFA80F90BE0152201
:100CE000204611F0CDFD06B2EBE71422204611F0AC
:100CF000C7FD0FFA80F99DF8170010F0010F20468C
:100D000002D010F067FF01E010F047FF0C900021C7
:100D10003222204611F0B4FD054600211022204663
:100D200011F0AEFDE18A28444718204611F07CF905
:100D3000381AADF8340000211222204611F0A0FD2F
:100D4000A18A28444518204611F066F9281AADF802
:100D50003C009DF817009DF8168010F0010F14BF9D
:100D60000DAD0FAD00210122204611F089FD00B22A
:100D7000119000210422204611F082FD00B2109053
:100D80009DF8170010F0010F0BD01099A1F51C521F
:100D9000D13A04BF618C11F4806F0BD010F0010FB9
:100DA0000AD11199A1F51C52D13A04BF618C11F4FA
:100DB000006F01D14FF00008BAF1000F0DD010F014
:100DC000010F0AD1B8F1000F08BF4FF0010804D09D
:100DD000B8F1010F08BF4FF000080027ADF83870D8
:100DE000BB46B8F1000F3CD09DF8170010F0040F7F
:100DF00008BF002215D0A0684068421E11E0002004
:100E00000B9006A8CDE9009005A920460C9BFFF7A2
:100E1000E3FDBDF81810BA1911440FB202460BF1E8
:100E2000010BA0684068824201DA002AE7DABBF1D0
:100E3000000F1CBFB81B07B29DF8170010F0010F80
:100E4000204602D010F0A9FE01E010F0C3FE0EA96A
:100E5000CDE9005101460FFA8BF33A46404619F0AE
:100E6000D1FE9DF8170010F0040F08BF4FF00008E6
:100E700003D0A1684968A1F10108BAF1000F05D0BB
:100E800010F0010F02D12888384428800DF1180B8A
:100E9000A0684068804548DAB8F1000F45DB0120C2
:100EA0000B90CDE9009B424605A920460C9BFFF71D
:100EB00093FD0746BAF1000F09D09DF8170010F016
:100EC000010F04D12888BDF81810401A28800C980A
:100ED000BDF93410CDE90110CDE9039BBDF93C000B
:100EE00000903B46424605A92046F8F70BFBB84662
:100EF00009980EF009FD00200990BAF1000F04D006
:100F00009DF8170010F0010F09D02888BDF81810BF
:100F10000844BDF83810314408442880B8E7BDF8CB
:100F2000381028883144401AF7E7119942F2D170FD
:100F300081421CBF1099814202D1204612F03CFD33
:100F400000222B2120460BF071F913B0BDE8F08F81
:100F5000840100202DE9F84F054600200090287FED
:100F600092468B4610F0010F62D14FF00108EC68F9
:100F70000026C14674B9287FC0F3C000401E30422D
:100F800056D1B9F1000F53D02846D8474FF000088A
:100F90000446C146002E08BFB4F1000648D0B8F19F
:100FA000000F05D021462846D0470446B0423FD026
:100FB0004FF00108002CDDD0206811F02DFC10F05E
:100FC000800FD7D127685FB10121384611F030FE7C
:100FD000B8B12FB10121384611F02AFE0028C9D13D
:100FE000E868A04224D0B0B1284600F00EFDE968C0
:100FF00002460B680F2118460BF018F9012806D09D
:1010000016E0384610F092FE0700DDD1E8E7E86808
:10101000006812F00FF92846EC6000F0F6FCE96871
:1010200002460B680E2118460BF000F9012802D089
:101030000098BDE8F88FE868006812F0FBF82969AD
:1010400000291CBF284688470120BDE8F88F000012
:10105000002808BF704738B590ED000A134C0025F2
:10106000BCEEC00A10EE100AC0F30C0040F4805031
:10107000ADF80000207890B10D4C002202212046EE
:10108000F0F73AFC4FF47A73012269460948F1F708
:10109000ACFD012202212046F0F72EFC38BD00F005
:1010A0000DF8054805700120207038BD8F00002024
:1010B000000802402C0A002084000020154810B5CA
:1010C000134901604FF48271416000214FF40062C6
:1010D000C0E902120222C0E9042112028261102238
:1010E000C0E90721416281620A21C162F1F7DAFB9E
:1010F000002818BFEFF7DAFC012220210648F0F79C
:10110000FBFB0122BDE8104002210448F0F7F4BBCC
:10111000003001402C0A002000100240000802406C
:10112000002814BF00297047027812B3164B4FF005
:10113000000202701B685A6243784EF6602C03FB73
:101140000CF300EE103AD0ED050A9FED101AB8EE40
:10115000400A30EE800AD0ED040A30EE600A80EDDD
:10116000020AC1EE000AC0ED030AC1ED000A427096
:10117000704710B50448F2F7CDF8BDE810400C21D7
:101180000148F2F7BFBA00007C0B0020002474492C
:10119000002908BF70472DE9F041934E04462DED1C
:1011A000068B0D4670799FED910A84427DD0904F59
:1011B0007471022C18BF032C4AD0042C1CBF052CC0
:1011C000072C45D00A2C1EBF81ED000ABDEC068B12
:1011D000BDE8F0816420F0F747FAF3F759FE642088
:1011E000F9F7F5F80220F3F7F5FDB078337900F060
:1011F000CF0040F02001F2780220F3F77DFE0220BC
:10120000F3F7E8FD0123F278B1780220F3F774FEDA
:101210000120F3F7DFFD307900F0BF0040F0360326
:10122000F07800F0F80040F00602B07800F07F019E
:101230000120F3F761FE00224FF480513846F0F7A9
:101240005BFBBDEC068B0220BDE8F041F9F7BFB8AF
:101250006420F0F709FAF3F71BFE6420F9F7B7F8FA
:101260000220F3F7B7FDB078337900F0CF0040F0FB
:101270002001F2780220F3F73FFE0B250220F3F75E
:10128000A9FD45EA0410C3B2F278B1780220F3F761
:1012900033FE00224FF480513846F0F72DFBBDECB1
:1012A000068B0220BDE8F04100E001E0F9F78FB8BD
:1012B00000210120F3F70EFD00EE100AB0EE041A33
:1012C000B8EE400A60EE010ADFED4A1A022C80EE09
:1012D000A10A53D0DFED480A032C59D0042C61D069
:1012E0009FED461A052C67D0072C6AD00A2C1CBF2C
:1012F000BDEC068BBDE8F08120EE200AC0EE010AAD
:10130000B7EE000A30EE60AA1AEE100AEFF7B1F954
:101310009FED3B8B53EC182BEFF7CAF89FED3A9BF0
:1013200053EC192BEFF7C1F841EC100BF4F7ABFAC3
:101330009FED371B51EC100B53EC112BEFF711F80D
:101340009FED351B53EC112BEFF724F9EFF7A4F9C0
:1013500004461AEE100AEFF78CF953EC182BEFF74E
:10136000A7F853EC192BEFF7A0F841EC100BF4F7AA
:101370008AFA2C60BDEC068BBDE8F081F3EE000A22
:1013800020EE200A85ED000ABDEC068BBDE8F08159
:101390009FED231A10EE201A85ED001ABDEC068B86
:1013A000BDE8F081F0EE000A10EE201A85ED001A7B
:1013B000BDEC068BBDE8F081C0EE011A21EEA00A5B
:1013C00009E020EE200ADFED170A20EE200AF6EEF3
:1013D000000A20EE200A85ED000ABDEC068BBDE870
:1013E000F0810000000000009000002000000000DC
:1013F0000004024000FEFF4600007A440000C8429C
:10140000F3F3C3E5889EC3BEBD81D0248683F03E3E
:10141000FEAED70D3E4170BFF3F3C3E5889EB3BE69
:10142000CDCC4C3E0AD7A33C30B583B00024054652
:10143000009403221E491F480194EFF7FFFC002887
:1014400018BFEFF733FB00216A46481C42F82140E1
:1014500010F0FF01F9D016480021009B30F811C0B0
:10146000491C6344C9B200930329F6D312480021F2
:101470000DF1040C52F82130A0FB03435B082CF85B
:101480001130491C11F0FF01F4D0BDF80400F3EE57
:101490000E0A00EE100AB8EE400A20EE200ADFED38
:1014A000070A80EE201A85ED001A03B030BD000057
:1014B000280000201C090020ABAAAAAA00F07F4542
:1014C00030B4426B818C12F0060F09D0C2F3410296
:1014D000022A04BFC08C084426D0012A04D024E08C
:1014E000008D084481B220E0B0F92C40458DA2B2B5
:1014F000AA423CBF02F5B47214B2B0F92830B0F879
:1015000026C09AB262453CBF02F5B47003B22819F6
:1015100000EBD07040108445B8BF0CEB010003DB3A
:101520009842B4BF5018084481B230BC08B270472A
:101530002DE9F34F87B0054602A910F068FB284655
:1015400011F010FB0490284610F097FB0590002145
:101550001222284611F094F907B2002113222846DE
:1015600011F08EF90FFA80F800211022284611F0B0
:1015700087F906B200211122284611F081F90FFAED
:1015800080F900211422284611F07AF904B20021D2
:101590001522284611F074F904F0010104EBD4720D
:1015A00001EB6201491C00B20FFA81FA00F001015F
:1015B00000EBD07001EB6000401C0FFA80FBBAF129
:1015C000100FA8BF4FF0100ABBF1100FA8BF4FF0CB
:1015D000100BB8F1100FA8BF4FF01008102EA8BFC5
:1015E0001026B9F1100FA8BF4FF010090024288E63
:1015F000002879D90498A0EB0800801E0490059873
:10160000A0EB0900801E0590A86A00EBC400B0F9A9
:101610000030ADF80030B0F90220ADF80220B0F98A
:101620000410ADF80410B0F90600ADF806009F42B2
:1016300017DBBDF908E0102FB4BFBC464FF0100C0B
:10164000AEEB0C0C6344ADF8003096421EDBBDF9E6
:101650000AC0102EB4BF33461023ACEB03031A4468
:1016600005E0BDF808C0ACEB0B0C6344EBE7ADF84C
:101670000220049A91421EDBBDF90820B8F1100F38
:101680000A44B4BF41461021114405E0BDF80A30B8
:10169000A3EB0A031A44EAE7ADF80410059988425F
:1016A00018DBBDF90A10B9F1100F0144B4BF484668
:1016B0001020084404E0BDF8082011445944EBE729
:1016C000ADF80600002268460899F4F7B9FB00B9A6
:1016D00005E009E0BDF80A1008445044F0E7601C3A
:1016E00084B2288EA0428FD8288EA04208BF4FF621
:1016F000FF74204609B0BDE8F08F2DE9F0474FF0A8
:1017000000081C46A3F8008016000F460546434615
:1017100008D0286B218830F813005B1C0844208017
:101720009E42F6D828460021162211F0A9F8C0B230
:10173000012818BF00200028284618D010F06CFCA3
:10174000218808442080284611F00CFA814628465A
:101750000021132211F094F82188A9EB0101081A45
:10176000A080296B31F81610401A208012E010F08A
:1017700053FC21881222081A20802846002111F0EB
:101780007FF8218808442080296B31F8161008441E
:10179000401EA0800022A4F80280002F08D9E86A29
:1017A000618830F81200521C084460809742F6D8D5
:1017B00028460021102211F063F8618808446080F7
:1017C000284610F031FC6188081A6080E96A31F817
:1017D00017100844401EE080BDE8F0872DE9F05F57
:1017E00091468A4604460021122211F049F806B2B9
:1017F00000211322204611F043F80FFA80F800214F
:101800001022204611F03CF805B20021112220469A
:1018100011F036F807B2204611F0A4F9801BA0EBB6
:10182000080B204610F029FA401BC01B83452046B8
:1018300005DA11F097F9801BA0EB080003E010F027
:101840001CFA401BC01B00EBD070401000B2A18AF4
:1018500082191144AAF80010E18A42191144AAF829
:101860000210B9F1000F18BFA9F80000BDE8F09F01
:10187000002904BF002070472DE9F04704690E4697
:1018800082B0616931B10868B04202BF486802B0F5
:10189000BDE8F0870022658AE805C00D1CBF04275B
:1018A000A36810D002EB820053F820C007EB800041
:1018B000185AA6EB0C0C60450ED2501C82B2C5F330
:1018C00008008242EED319B10E60616900204860C1
:1018D00002B00020BDE8F08702EB8205122000EB89
:1018E00085000027185C4FF0060802280AD04FF048
:1018F0000C0968B12B4B10220821032812D00128B3
:1019000029D046E008EB8500185A00EB0C0740E0B0
:1019100009EB850008EB85011858595A10F80C009E
:101920000F1836E0ADF804C00093A06801EB8509FC
:1019300002EB8502825A50F80910022301A8F5F73C
:1019400049FD30B3A16851F80920801A08EB8502DF
:101950004010895A1CE0ADF804C00093A06801EB68
:10196000850A02EB8502825A50F80A10022301A868
:10197000F5F730FD68B1A16808EB850351F80A203E
:10198000801A09EB850240108A58C95A32F81000B3
:101990000F18606910B106606069476002B0384690
:1019A000BDE8F087FB2603082DE9F0410546406AB3
:1019B0000E46002808BF002403D0002110F075F85F
:1019C0000446002C04BF0020BDE8F081E08A00211D
:1019D000371A5722204610F053FF0689002159225A
:1019E000204610F04DFF00B200EBD07107EB610113
:1019F000304409B200B291FBF0F0A98E80B281426E
:101A00009CBF481E80B2BDE8F0812DE9F041002660
:101A10000746354630460CF0E1F9040019D00CF0C9
:101A20001AFA616DB94205D1022817D0042808BFFF
:101A30002646254620460CF0D1F90400EFD1002EB1
:101A40001CBF3046BDE8F081002D1CBF2846BDE814
:101A5000F0810020BDE8F0410CF0C0B92046BDE89F
:101A6000F0812DE9F05F0C4683460021502220468C
:101A700010F006FF00B200EBD07045084FF4403183
:101A80001222204610F0FCFE82464FF44031132211
:101A9000204610F0F5FE81464FF4403110222046DA
:101AA00010F0EEFE80464FF440311122204610F037
:101AB000E7FE0246A08A218D638D0844411BA1EBFD
:101AC0000A0161F30F06E18A19444B1BA3EB0903DA
:101AD00063F31F4605EB0803184460F30F07A818CB
:101AE000084460F31F47CBF80060CBF80470BDE8F2
:101AF000F09F2DE9F84F90460F461E4605464FF4DD
:101B00000031502210F0BCFE00B200EBD070441047
:101B1000A8EB04082846FFF7D3FC82465A3000B2EF
:101B200017F0ECFC10FB08F04FEAE039504617F0D4
:101B3000E5FC10FB08F04FEAE0384FF44031122288
:101B4000284610F09DFE00904FF4403113222846A5
:101B500010F096FE83464FF440311022284610F0D4
:101B60008FFE82464FF440311122284610F088FE45
:101B70003988204401EB09020099511A091B318070
:101B800039880BEB040249441144B18079884144FF
:101B9000A1EB0A01091B7180798841440844F08057
:101BA000BDE8F88F2DE9F04105460E46B5F822C094
:101BB0000020CCF305110427EB68002910D907EBAE
:101BC000C0029A5812F0807F07D022F07F42B242C2
:101BD00003D153F83000BDE8F081401C8142EED8BB
:101BE0004FF0806000EBBC204FEAB0506884C0F337
:101BF0000510C10018460DF0E5FEE86080B1688C64
